:020000040800F2
:1000000000060020E10100086D0E0008ED0D00085B
:10001000450E0008ED0D0008190E0008E301000868
:10002000E3010008E3010008E301000841210008A2
:10003000E3010008E3010008E3010008E301000810
:10004000E3010008E3010008E3010008E301000800
:10005000E3010008E3010008093200083532000816
:10006000613200088D320008B9320008E30100084F
:10007000E3010008E3010008E3010008E3010008D0
:10008000E3010008E3010008E3010008E3010008C0
:10009000E3010008E3010008E3010008E53200087D
:1000A000E3010008E3010008E3010008E3010008A0
:1000B0007D300008E3010008E3010008E3010008C7
:1000C000E3010008E3010008E3010008E301000880
:1000D000E3010008E3010008E3010008E301000870
:1000E0004D330008E3010008E3010008E3010008C4
:1000F000E3010008E3010008E3010008E301000850
:10010000E3010008E3010008E3010008E30100083F
:10011000E3010008E3010008E3010008E30100082F
:10012000E3010008E3010008E3010008E30100081F
:10013000E3010008E3010008E3010008E30100080F
:10014000E3010008E3010008E30100087928000842
:10015000E3010008E3010008E3010008E3010008EF
:10016000E3010008E3010008E3010008E3010008DF
:10017000E3010008E3010008E3010008E3010008CF
:10018000E3010008E3010008E3010008E3010008BF
:10019000E3010008E3010008E3010008E3010008AF
:1001A000E3010008E3010008E3010008E30100089F
:1001B000E3010008E3010008E3010008E30100088F
:1001C000E3010008E3010008E3010008E30100087F
:1001D000E3010008E3010008E3010008E30100086F
:1001E00002E000F000F8FEE772B63A4880F30888B3
:1001F000394880F3098839484EF60851CEF200019B
:10020000086040F20000CCF200004EF63471CEF2ED
:1002100000010860BFF34F8FBFF36F8F40F2000003
:10022000C0F2F0004EF68851CEF200010860BFF334
:100230004F8FBFF36F8F4FF00000E1EE100A4EF6C4
:100240003C71CEF200010860062080F31488BFF3F1
:100250006F8F01F0F5FF01F0D1FF02F073FE4FF058
:1002600055301F491B4A91423CBF41F8040BFAE745
:100270001C49194A91423CBF41F8040BFAE71A495C
:100280001A4A1B4B9A423EBF51F8040B42F8040B2A
:10029000F8E700201749184A91423CBF41F8040B87
:1002A000FAE701F0AFFF02F0A1FE144C144DAC428E
:1002B00003DA54F8041B8847F9E700F041F8114CC1
:1002C000114DAC4203DA54F8041B8847F9E701F0FA
:1002D00097BF000000060020002200200000000858
:1002E00000000020000600207837000800220020CF
:1002F0004022002040220020A82D0020E00100081C
:10030000E0010008E0010008E00100082DE9F04FDD
:100310002DED108AC1F80CD0C3689D46BDEC108A43
:10032000BDE8F08F002383F311882846A047002002
:1003300001F012FBFEE701F08DFA00DFFEE700009E
:1003400038B501F0CDFE054601F0F0FE0446D8B9FF
:100350000F4B9D421AD001339D4218BF044641F213
:10036000883504BF01240025002001F0C3FE0CB134
:1003700000F076F800F010FD00F09EFB284600F03B
:10038000BFF800F06DF8F9E70025EDE70546EBE76B
:10039000010007B008B500F061FBA0F1200358424E
:1003A000584108BD07B541F21203022101A8ADF87A
:1003B000043000F071FB03B05DF804FB38B5202376
:1003C00083F311881748C3680BB101F04BFB164A41
:1003D000144800234FF47A7101F008FB002383F3E3
:1003E0001188124C236813B12368013B23606368B2
:1003F00013B16368013B63600D4D2B7833B96368BB
:100400007BB9022000F042FC322363602B78032B7F
:1004100007D163682BB9022000F038FC4FF47A73DF
:10042000636038BD40220020BD0300085C2300202B
:1004300054220020084B187003280CD8DFE800F085
:1004400008050208022000F017BC022000F00ABCD8
:10045000024B00225A607047542200205C23002087
:10046000234B244A10B51C46196801313FD0043390
:100470009342F9D16268A24239D31F4B9B6803F1C2
:10048000006303F540439A4231D2002000F02EFB76
:100490000220FFF7CFFF194B1A6C00221A64196E65
:1004A0001A66196E596C5A64596E5A665A6E5A69B0
:1004B00042F080025A615A6922F080025A615A69F8
:1004C0001A6942F000521A611A6922F000521A6148
:1004D0001B6972B64FF0E0232021C3F8084DD4E920
:1004E000003281F311889D4683F30888104710BDC0
:1004F00000C0000820C00008002200200038024090
:100500002DE9F04F93B0A94B00902022FF210AA8BB
:100510009D6800F0EBFBA64A1378A3B9A54801211A
:10052000C3601170202383F31188C3680BB101F0FD
:1005300099FAA14A9F4800234FF47A7101F056FAC4
:10054000002383F31188009B13B19C4B009A1A601F
:100550009B4A009C1378032B1EBF00231370974AFD
:100560004FF0000A18BF5360D3465646D1460120CB
:1005700000F082FB24B1914B1B68002B00F00F822E
:10058000002000F06BFA0390039B002BF2DB0120AC
:1005900000F068FB039B213B162BE8D801A252F820
:1005A00023F000BF0106000829060008BD06000868
:1005B0006F0500086F0500086F0500084507000873
:1005C000130900082D0800088F080008B708000864
:1005D000DD0800086F050008EF0800086F05000837
:1005E00061090008A10600086F050008A5090008B8
:1005F0000D060008A10600086F0500088F08000816
:100600000220FFF7C7FE002840F0F381009B022183
:10061000BAF1000F08BF1C4605A841F21233ADF82D
:10062000143000F039FAA2E74FF47A7000F016FAAD
:10063000071EEBDB0220FFF7ADFE0028E6D0013FEE
:10064000052F00F2D881DFE807F0030A0D101336FA
:1006500005230593042105A800F01EFA17E053486E
:100660000421F9E757480421F6E757480421F3E746
:100670004FF01C08404600F03BFA08F104080590D2
:10068000042105A800F008FAB8F12C0FF2D10120DE
:1006900000FA07F747EA0B0B5FFA8BFB4FF00009F4
:1006A00000F070FB26B10BF00B030B2B08BF0024EE
:1006B000FFF778FE5BE745480421CDE7002EA5D083
:1006C0000BF00B030B2BA1D10220FFF763FE0746B3
:1006D00000289BD0012000F009FA0220FFF7AAFEB3
:1006E00000265FFA86F8404600F010FA044688B10A
:1006F000404600F01BFA01360028F2D1BA46044603
:1007000041F21213022105A8ADF814303E4600F064
:10071000C3F92CE70120FFF78DFE2546234B9B688C
:10072000AB4207D9284600F0E3F9013040F066817A
:100730000435F3E7224B00251D70204BBA465D605F
:100740003E46ADE7002E3FF461AF0BF00B030B2BE1
:100750007FF45CAF0220FFF76DFE322000F07EF9DF
:10076000B0F10008FFF652AF18F003077FF44EAF68
:100770000E4A926808EB050393423FF647AFB8F57F
:10078000807F3FF743AF124B0193B84522DD4FF412
:100790007A7000F063F90390039A002AFFF636AFEF
:1007A000019B039A03F8012B0137EDE7002200209B
:1007B0005823002040220020BD0300085C230020B5
:1007C0005422002004220020082200200C220020B5
:1007D00058220020C820FFF7DDFD074600283FF41F
:1007E00015AF1F2D11D8C5F1200242450AAB25F0E7
:1007F000030028BF424683490192184400F050FA92
:10080000019A8048FF2100F071FA4FEAA8037D4960
:100810000193C8F38702284600F070FA06460028C4
:100820003FF46EAF019B05EB830539E70220FFF72C
:10083000B1FD00283FF4EAAE00F0A2F900283FF431
:10084000E5AE0027B846704B9B68BB4218D91F2FF6
:1008500011D80A9B01330ED027F0030312AA1344C8
:1008600053F8203C05934046042205A900F000FB04
:1008700004378046E7E7384600F03AF90590F2E79A
:10088000CDF81480042105A800F006F908E700233C
:10089000642104A8049300F0F5F800287FF4B6AEB4
:1008A0000220FFF777FD00283FF4B0AE049800F077
:1008B0004FF90590E6E70023642104A8049300F0B3
:1008C000E1F800287FF4A2AE0220FFF763FD0028C4
:1008D0003FF49CAE049800F04BF9EAE70220FFF7E2
:1008E00059FD00283FF492AE00F05AF9E1E70220EA
:1008F000FFF750FD00283FF489AE05A9142000F051
:1009000055F904210746049004A800F0C5F83946BB
:10091000B9E7322000F0A2F8071EFFF677AEBB075A
:100920007FF474AE384A926807EB090393423FF6AE
:100930006DAE0220FFF72EFD00283FF467AE27F0D2
:1009400003074F44B9453FF4ABAE484600F0D0F83A
:100950000421059005A800F09FF809F10409F1E7CA
:100960004FF47A70FFF716FD00283FF44FAE00F009
:1009700007F9002844D00A9B01330BD008220AA9AA
:10098000002000F0BBF900283AD02022FF210AA85D
:1009900000F0ACF9FFF706FD1C4800F0E3FF13B0D0
:1009A000BDE8F08F002E3FF431AE0BF00B030B2BA4
:1009B0007FF42CAE0023642105A8059300F062F8B3
:1009C000074600287FF422AE0220FFF7E3FC8046B2
:1009D00000283FF41BAEFFF7E5FC41F2883000F041
:1009E000C1FF059800F000FA464600F0CBF93C46FE
:1009F000BDE5064654E64FF0000907E6BA467FE635
:100A000037467DE65822002000220020A086010003
:100A100070B50F4B1B780133DBB2012B0C4611D89C
:100A20000C4D29684FF47A730E6AA2FB033201461B
:100A300022462846B047844204D1074B00221A7050
:100A4000012070BD4FF4FA7000F08CFF0020F8E731
:100A500010220020502500209023002007B50023FD
:100A6000024601210DF107008DF80730FFF7D0FF96
:100A700020B19DF8070003B05DF804FB4FF0FF3094
:100A8000F9E700000A4608B50421FFF7C1FF80F02E
:100A90000100C0B2404208BD30B4054C2368DD6996
:100AA000044B0A46AC460146204630BC604700BFB6
:100AB00050250020A086010070B501F003FA094E10
:100AC000094D3080002428683388834208D901F01A
:100AD000F3F92B6804440133B4F5404F2B60F2D393
:100AE00070BD00BF922300206423002001F0ACBA47
:100AF00000F1006000F540400068704700F10060C0
:100B0000920000F5404001F02BBA0000054B1A6836
:100B1000054B1B889B1A834202D9104401F0CCB9C3
:100B200000207047642300209223002038B5074D31
:100B300004462868204401F0C7F928B928682044F1
:100B4000BDE8384001F0D8B938BD00BF64230020AB
:100B500010F003030AD1B0F5047F05D200F1005074
:100B6000A0F51040D0F80038184670470023FBE786
:100B700000F10050A0F51040D0F8100A70470000B6
:100B8000064991F8243033B10023086A81F82430F3
:100B90000822FFF7B3BF0120704700BF6823002081
:100BA000014B1868704700BF002004E070B52A4B65
:100BB0001B68C3F30B0204461B0C62B140F21340E6
:100BC000824230D040F2194082422ED040F2214081
:100BD00082422CD10322214D0C2000FB0252556889
:100BE00042F20102934224D0B3F5805F23D041F258
:100BF0000102934221D041F2030293421FD041F2FD
:100C00000702934214BF3F233123013C0C44013DB2
:100C10000A46A24215D215F9016F501C9EB100F888
:100C2000016C0246F5E70122D5E70222D3E70C4D1D
:100C3000D6E73323E9E74123E7E75A23E5E75923DA
:100C4000E3E7104605E02C258442157001D9901C7D
:100C50005370401A70BD00BF002004E078340008D3
:100C60004C340008022802BF024B4FF080729A6198
:100C7000704700BF00080240022802BF024B4FF439
:100C800080729A61704700BF00080240022801BFCD
:100C9000024A536983F4807353617047000802402D
:100CA00010B50023934203D0CC5CC4540133F9E760
:100CB00010BD000010B5013810F9013F3BB191F9AA
:100CC00000409C4203D11AB10131013AF4E71AB154
:100CD00091F90020981A10BD1046FCE70346024621
:100CE000D01A12F9011B0029FAD1704702440346B9
:100CF000934202D003F8011BFAE770472DE9F8434D
:100D00001F4D144695F824200746884652BBDFF84D
:100D100070909CB395F824302BB92022FF214846CF
:100D20002F62FFF7E3FF95F82400C0F10802A2420A
:100D300028BF2246D6B24146920005EB8000FFF75D
:100D4000AFFF95F82430A41B1E44F6B2082E1744BA
:100D50009044E4B285F82460DBD1FFF711FF00284E
:100D6000D7D108E02B6A03EB82038342CFD0FFF791
:100D700007FF0028CBD10020BDE8F8830120FBE766
:100D800068230020024B1A78024B1A70704700BF8C
:100D9000902300201022002010B50F4C0F4800F0C7
:100DA000F7F821460D4800F01FF924680C48626DE1
:100DB000D2F8043843F00203C2F8043800F0D2FD40
:100DC0000849204600F016FA626DD2F8043823F084
:100DD0000203C2F8043810BD6C350008502500200D
:100DE00040420F00743500087047000000B59BB00A
:100DF000EFF3098168226846FFF752FFEFF305839E
:100E0000044B9A6BDA6A9A6A9A6A9A6A9A6A9A6A36
:100E10009B6AFEE700ED00E000B59BB0EFF30981AF
:100E200068226846FFF73CFFEFF30583044B9A6B9B
:100E30009A6A9A6A9A6A9A6A9A6A9B6AFEE700BFF5
:100E400000ED00E000B59BB0EFF309816822684631
:100E5000FFF726FFEFF30583034B5A6B9A6A9A6AF2
:100E60009A6A9A6A9B6AFEE700ED00E0FEE70000DE
:100E700030B5094D0A4491420DD011F8013B58405C
:100E8000082340F30004013B2C4013F0FF0384EAE5
:100E90005000F6D1EFE730BD2083B8ED026843681B
:100EA0001143016003B118477047000013B5446B4C
:100EB000D4F894341A681178042915D1217C0229B8
:100EC00012D11979128901238B4013420CD101A947
:100ED00004F14C0001F03CFFD4F89444019B2179CB
:100EE0000246206800F0CEF902B010BD143001F0C7
:100EF000BFBE00004FF0FF33143001F0B9BE000058
:100F00004C3001F091BF00004FF0FF334C3001F046
:100F10008BBF0000143001F08DBE00004FF0FF3198
:100F2000143001F087BE00004C3001F05DBF0000BE
:100F30004FF0FF324C3001F057BF000000207047E7
:100F400010B5D0F894341A6811780429044617D1E2
:100F5000017C022914D15979528901238B40134213
:100F60000ED1143001F020FE024648B1D4F894446A
:100F70004FF4807361792068BDE8104000F070B9CB
:100F800010BD0000406BFFF7DBBF000070470000A2
:100F90007FB5124B036000234360C0E90233012593
:100FA00002260F4B057404460290019300F184025F
:100FB000294600964FF48073143001F0D1FD094B9F
:100FC0000294CDE9006304F523724FF4807329463F
:100FD00004F14C0001F098FE04B070BDA834000884
:100FE000850F0008AD0E00080B68202282F31188DF
:100FF0000A7903EB820290614A79093243F82200B0
:101000008A7912B103EB8203986102230374C0F85A
:101010009414002383F311887047000038B5037FD0
:10102000044613B190F85430ABB9201D01250221BC
:10103000FFF734FF04F1140025776FF0010100F091
:10104000B9FC84F8545004F14C006FF00101BDE884
:10105000384000F0AFBC38BD10B501210446043063
:10106000FFF71CFF0023237784F8543010BD0000E5
:1010700038B504460025143001F08AFD04F14C0017
:10108000257701F059FE201D84F854500121FFF707
:1010900005FF2046BDE83840FFF752BF90F84430C6
:1010A00003F06003202B07D190F84520212A4FF050
:1010B000000303D81F2A06D800207047222AFBD13C
:1010C000C0E90E3303E0034A82630722C26303646C
:1010D000012070471122002037B5D0F894341A68E7
:1010E0001178042904461AD1017C022917D11979F3
:1010F000128901238B40134211D100F14C0528467F
:1011000001F0DAFE58B101A9284601F021FED4F819
:101110009444019B21790246206800F0B3F803B0A3
:1011200030BD0000F0B500EB810385B09E69044638
:101130000D46FEB1202383F3118804EB8507301D93
:101140000821FFF7ABFEFB685B691B6806F14C00EA
:101150001BB1019001F00AFE019803A901F0F8FD0E
:10116000024648B1039B2946204600F08BF8002335
:1011700083F3118805B0F0BDFB685A691268002A34
:10118000F5D01B8A013B1340F1D104F14402EAE798
:10119000093138B550F82140DCB1202383F31188A0
:1011A000D4F894241368527903EB8203DB689B69BB
:1011B0005D6845B104216018FFF770FE294604F10F
:1011C000140001F0FBFC2046FFF7BAFE002383F376
:1011D000118838BD7047000001F0A8B801230370E2
:1011E0000023C0E90133C36183620362C3624362C7
:1011F0000363704738B50446202383F31188002524
:10120000C0E90355C0E90555416001F09FF802238C
:10121000237085F3118838BD70B500EB8103054656
:101220005069DA600E46144618B110220021FFF70B
:101230005DFDA06918B110220021FFF757FD31466E
:101240002846BDE8704001F04BB90000826802F00A
:10125000011282600022C0E90422826101F0CCB94F
:10126000F0B400EB81044789E4680125A4698D404E
:101270003D43458123600023A2606360F0BC01F020
:10128000E7B90000F0B400EB81040789E4680125A8
:1012900064698D403D43058123600023A260636043
:1012A000F0BC01F061BA000070B5022300250446CD
:1012B0000370C0E90255C0E90455C564856180F832
:1012C000345001F0A9F863681B6823B12946204611
:1012D000BDE87040184770BD037880F85030052392
:1012E000037043681B6810B504460BB1042198478E
:1012F0000023A36010BD000090F8502043680270E6
:101300001B680BB1052118477047000070B590F8B5
:101310003430044613B1002380F8343004F1440221
:10132000204601F08BF963689B68B3B994F84430A8
:1013300013F0600535D00021204601F0DDFB0021CF
:10134000204601F0CFFB63681B6813B106212046DD
:101350009847062384F8343070BD2046984700280B
:10136000E4D0B4F84A30E26B9A4288BFE36394F960
:101370004430E56B002B4FF0200380F20381002DF9
:1013800000F0F280092284F8342083F311880021D0
:10139000D4E90E232046FFF775FF002383F311885D
:1013A000DAE794F8452003F07F0343EA022340F292
:1013B0000232934200F0C58021D8B3F5807F48D037
:1013C0000DD8012B3FD0022B00F09380002BB2D11F
:1013D00004F14C02A2630222E2632364C1E7B3F585
:1013E000817F00F09B80B3F5407FA4D194F8463014
:1013F000012BA0D1B4F84C3043F0020332E0B3F536
:10140000006F4DD017D8B3F5A06F31D0A3F5C063EE
:10141000012B90D8636894F846205E6894F84710D2
:10142000B4F848302046B047002884D04368A3630E
:101430000368E3631AE0B3F5106F36D040F602425A
:1014400093427FF478AF5C4BA3630223E3630023F2
:10145000C3E794F84630012B7FF46DAFB4F84C30FD
:1014600023F00203C4E90E55A4F84C30256478E754
:10147000B4F84430B3F5A06F0ED194F8463084F838
:101480004E30204601F020F863681B6813B101213B
:1014900020469847032323700023C4E90E339CE7BA
:1014A00004F14F03A3630123C3E72378042B10D176
:1014B000202383F311882046FFF7C8FE85F31188A7
:1014C0000321636884F84F5021701B680BB12046DC
:1014D000984794F84630002BDED084F84F30042330
:1014E000237063681B68002BD6D0022120469847E2
:1014F000D2E794F848301D0603F00F0120460AD5C4
:1015000001F08EF8012804D002287FF414AF2B4B91
:101510009AE72B4B98E701F075F8F3E794F846301B
:10152000002B7FF408AF94F8483013F00F01B3D0CC
:101530001A06204602D501F0F3FAADE701F0E6FA0B
:10154000AAE794F84630002B7FF4F5AE94F84830C3
:1015500013F00F01A0D01B06204602D501F0CCFAF3
:101560009AE701F0BFFA97E7142284F8342083F356
:1015700011882B462A4629462046FFF771FE85F33F
:101580001188E9E65DB1152284F8342083F31188CF
:101590000021D4E90E232046FFF762FEFDE60B2270
:1015A00084F8342083F311882B462A4629462046A6
:1015B000FFF768FEE3E700BFD8340008D034000826
:1015C000D434000838B590F834300446002B3ED0AF
:1015D000063BDAB20F2A34D80F2B32D8DFE803F0FB
:1015E0003731310822323131313131313131373710
:1015F000C56BB0F84A309D4214D2C3681B8AB5FB54
:10160000F3F203FB12556DB9202383F311882B46A7
:101610002A462946FFF736FE85F311880A2384F807
:1016200034300EE0142384F83430202383F31188FF
:1016300000231A4619462046FFF712FE002383F3C3
:10164000118838BD036C03B198470023E7E70021F8
:10165000204601F051FA0021204601F043FA636868
:101660001B6813B10621204698470623D7E70000E0
:1016700010B590F83430142B044629D017D8062B17
:1016800005D001D81BB110BD093B022BFBD80021AE
:10169000204601F031FA0021204601F023FA636868
:1016A0001B6813B1062120469847062319E0152B25
:1016B000E9D10B2380F83430202383F311880023F1
:1016C0001A461946FFF7DEFD002383F31188DAE797
:1016D000C3689B695B68002BD5D1036C03B1984745
:1016E000002384F83430CEE7024B0022C3E90033F4
:1016F0009A60704794230020002303748268054B8E
:101700001B6899689142FBD25A680360426010607E
:10171000586070479423002008B5202383F3118874
:10172000037C032B05D0042B0DD02BB983F3118838
:1017300008BD436900221A604FF0FF334361FFF791
:10174000DBFF0023F2E7D0E9003213605A60F3E7D1
:10175000002303748268054B1B6899689142FBD88B
:101760005A680360426010605860704794230020FC
:10177000054B19690874186802681A60536018618B
:1017800001230374FEF7C2BD9423002030B54B1C27
:101790000B4D87B0044610D02B690A4A01A800F00F
:1017A00025F92046FFF7E4FF049B13B101A800F0E0
:1017B00059F92B69586907B030BDFFF7D9FFF8E731
:1017C000942300201917000838B50C4D41612B698E
:1017D00081689A689142044603D8BDE83840FFF713
:1017E0008BBF1846FFF7B4FF01232C610146237419
:1017F0002046BDE83840FEF789BD00BF9423002095
:10180000044B1A681B6990689B68984294BF00203B
:10181000012070479423002010B5084C23682069EC
:101820001A6822605460012223611A74FFF790FF46
:1018300001462069BDE81040FEF768BD94230020F2
:1018400008B5FFF7DDFF18B1BDE80840FFF7E4BFBA
:1018500008BD0000FFF7E0BFFEE7000010B50C4C2C
:10186000FFF742FF00F0B4F80A498022204600F05A
:101870003BF8012344F8180C037400F071FC0023BA
:1018800083F3118862B60448BDE8104000F04CB8FC
:10189000BC230020DC340008EC34000800F01CB944
:1018A000EFF3118020B9EFF30583202282F3118832
:1018B0007047000010B530B9EFF30584C4F3080495
:1018C00014B180F3118810BDFFF7BAFF84F31188BB
:1018D000F9E70000034A516853685B1A9842FBD845
:1018E000704700BF001000E0826002220282704751
:1018F0008368A3F17C0243F80C2C026943F83C2C6A
:10190000426943F8382C074A43F81C2CC26843F854
:10191000102C022203F8082C002203F8072CA3F154
:10192000180070472503000810B5202383F31188A1
:10193000FFF7DEFF00210446FFF746FF002383F395
:101940001188204610BD0000024B1B6958610F2012
:10195000FFF70EBF94230020202383F31188FFF7A5
:10196000F3BF000008B50146202383F31188082047
:10197000FFF70CFF002383F3118808BD49B1064B24
:1019800042681B6918605A60136043600420FFF7C7
:10199000FDBE4FF0FF30704794230020036898424B
:1019A00006D01A680260506059611846FFF7A4BE5D
:1019B0007047000038B504460D462068844200D1C7
:1019C00038BD036823605C604561FFF795FEF4E76E
:1019D000054B03F11402C3E905224FF0FF31002249
:1019E000C3E90712704700BF9423002070B51C4E56
:1019F000C0E9032305460C4601F090FA334653F83C
:101A0000142F9A420DD13062C5E901242A600A2CB4
:101A10002CBF00190A30C6E90555BDE8704001F039
:101A20006BBA316A431AE31838BF1C469368A34265
:101A300002D9081901F06EFA73699A6894420CD8B9
:101A40005A68AC602B606A6015609A685D60121B12
:101A50009A604FF0FF33F36170BD1B68A41AECE786
:101A60009423002038B51B4C636998420DD0D0E90F
:101A7000003213605A6000228168C2609A680A448A
:101A80009A604FF0FF33E36138BD2246036842F8A5
:101A9000143F002193425A60C16003D1BDE8384031
:101AA00001F032BA9A688168256A0A449A6001F0A6
:101AB00035FA63699A68411B8A42E5D9AB181D1A49
:101AC000092D206A98BF01F10A02BDE83840104490
:101AD00001F020BA942300202DE9F041184C002792
:101AE00004F11406656901F019FA236AAA68C11A9B
:101AF0008A4215D813442362D5E9003213605A6034
:101B00006369D5F80C80EF60B34201D101F0FCF9B4
:101B100087F311882869C047202383F31188E1E700
:101B20006169B14209D013441B1ABDE8F0410A2B88
:101B30002CBFC0180A3001F0EDB9BDE8F08100BF3C
:101B40009423002000207047FEE70000704700004B
:101B50004FF0FF307047000002290CD0032904D059
:101B60000129074818BF00207047032A05D80548F7
:101B700000EBC2007047044870470020704700BF68
:101B8000D0350008202200208435000870B59AB0B6
:101B90000546084601A9144600F0C2F801A8FFF75F
:101BA0009DF8431C5B00C5E9003400222370032329
:101BB0006370C6B201AB02341046D1B28E4204F15A
:101BC000020401D81AB070BD13F8011B04F8021CFE
:101BD00004F8010C0132F0E708B5202383F31188E3
:101BE0000348FFF779FA002383F3118808BD00BF8B
:101BF0005025002090F8443003F01F02012A07D13D
:101C000090F845200B2A03D10023C0E90E3315E0DC
:101C100003F06003202B08D1B0F848302BB990F8BE
:101C20004520212A03D81F2A04D8FFF737BA222AD1
:101C3000EBD0FAE7034A82630722C2630364012000
:101C4000704700BF1822002007B5052917D8DFE824
:101C500001F0191603191920202383F31188104A63
:101C600001900121FFF7D8FA01980E4A0221FFF7EF
:101C7000D3FA0D48FFF7FCF9002383F3118803B072
:101C80005DF804FB202383F311880748FFF7C6F9AA
:101C9000F2E7202383F311880348FFF7DDF9EBE730
:101CA00024350008483500085025002038B50C4D73
:101CB0000C4C0D492A4604F10800FFF767FF05F1B7
:101CC000CA0204F110000949FFF760FF05F5CA7266
:101CD00004F118000649BDE83840FFF757BF00BFC0
:101CE000182A002020220020043500080E350008A4
:101CF0001935000870B5044608460D46FEF7EEFF9C
:101D0000C6B22046013403780BB9184670BD32467E
:101D10002946FEF7CFFF0028F3D10120F6E70000A7
:101D20002DE9F04705460C46FEF7D8FF2B49C6B211
:101D30002846FFF7DFFF08B10636F6B228492846E5
:101D4000FFF7D8FF08B11036F6B2632E0BD8DFF8D4
:101D50008C80DFF88C90234FDFF894A02E7846B962
:101D60002670BDE8F08729462046BDE8F04701F01F
:101D700065BB252E2ED1072241462846FEF79AFF45
:101D800070B9194B224603F10C0153F8040B42F8C9
:101D9000040B8B42F9D11B78137007350D34DDE746
:101DA000082249462846FEF785FF98B90F4BA21C2A
:101DB000197809090232C95D02F8041C13F8011BE5
:101DC00001F00F015345C95D02F8031CF0D118342E
:101DD0000835C3E704F8016B0135BFE7F0350008AB
:101DE0001935000806360008F8350008107AFF1F7C
:101DF0001C7AFF1FBFF34F8F024AD368DB03FCD46A
:101E0000704700BF003C024008B5094B1B7873B90E
:101E1000FFF7F0FF074B1A69002ABFBF064A5A6056
:101E200002F188325A601A6822F480621A6008BD92
:101E3000762C0020003C02402301674508B50B4B7F
:101E40001B7893B9FFF7D6FF094B1A6942F000429D
:101E50001A611A6842F480521A601A6822F4805299
:101E60001A601A6842F480621A6008BD762C00205D
:101E7000003C02400B28F0B516D80C4C0C492378D6
:101E80007BB90C4D0E460C234FF0006255F8047BD5
:101E900046F8042B013B13F0FF033A44F6D101232B
:101EA000237051F82000F0BD0020FCE7A82C002092
:101EB000782C002018360008014B53F8200070479A
:101EC000183600080C2070470B2810B5044601D9BD
:101ED000002010BDFFF7CEFF064B53F82430184406
:101EE000C21A0BB90120F4E712680132F0D1043BA9
:101EF000F6E700BF183600080B2838B5044628D886
:101F0000FFF7CEFCFFF776FFFFF77EFF124AF323C1
:101F1000D360E300DBB243F4007343F002031361C8
:101F2000136943F48033136105462046FFF762FFCF
:101F3000FFF7A0FF094B53F8241000F0E9F82846FA
:101F4000FFF77CFFFFF7B6FC2046BDE83840FFF7FF
:101F5000BBBF002038BD00BF003C0240183600085F
:101F600012F001032DE9F04105460E4614464BD10F
:101F70008218B2F1016F61D8314B1B6813F0010375
:101F80005CD0304FFFF78CFCFFF73EFFF323FB6084
:101F9000FFF730FF314640F20128032C18D824F017
:101FA0000104284E0C446D1A40F20118A142336915
:101FB00005EB01072AD123F001033361FFF73EFF50
:101FC000FFF778FC0120BDE8F081043C0435E4E72C
:101FD000AB07E4D13B6923F440733B613B6943EABF
:101FE00008033B6151F8046B2E60BFF34F8FFFF77E
:101FF00001FF2B689E42E8D03B6923F001033B615F
:10200000FFF71CFFFFF756FC0020DCE723F44073CA
:102010003361336943EA080333610B883B80BFF3C4
:102020004F8FFFF7E7FE3F8831F8023BBFB2BB425C
:10203000BCD0336923F001033361E1E71846C2E7FE
:1020400000380240003C0240084908B50B7828B12E
:102050001BB9FFF7D9FE01230B7008BD002BFCD084
:10206000BDE808400870FFF7E9BE00BF762C0020ED
:1020700010B50244064BD2B2904200D110BD441CB0
:1020800000B253F8200041F8040BE0B2F4E700BFBF
:10209000502800400F4B30B51C6F240407D41C6F30
:1020A00044F400741C671C6F44F400441C670A4C21
:1020B000236843F4807323600244084BD2B29042F9
:1020C00000D130BD441C00B251F8045B43F82050ED
:1020D000E0B2F4E7003802400070004050280040B1
:1020E00007B5012201A90020FFF7C2FF019803B044
:1020F0005DF804FB13B50446FFF7F2FFA04205D0DC
:10210000012201A900200194FFF7C4FF02B010BD15
:1021100070470000034B1A681AB9034AD2F87428B2
:102120001A607047AC2C00200030024008B5FFF761
:10213000F1FF024B1868C0F3407008BDAC2C0020C2
:10214000EFF3098305494A6B22F001024A636833C1
:1021500083F30988002383F31188704700EF00E0C0
:10216000202080F3118862B60C4B0D4AD96821F407
:10217000E0610904090C0A43DA60D3F8FC2009493C
:1021800042F08072C3F8FC200A6842F001020A6043
:102190001022DA7783F82200704700BF00ED00E0DC
:1021A0000003FA05001000E010B5202383F3118826
:1021B0000E4B5B6813F4006314D0F1EE103AEFF3AA
:1021C0000984683C4FF08073E361094BDB6B236645
:1021D00084F30988FFF714FB10B1064BA36110BD0F
:1021E000054BFBE783F31188F9E700BF00ED00E042
:1021F00000EF00E0370300083A03000870470000D2
:10220000FEE700000A4B0B480B4A90420BD30B4BE6
:10221000DA1C121AC11E22F003028B4238BF0022C0
:102220000021FEF763BD53F8041B40F8041BECE7E4
:10223000B8370008A82D0020A82D0020A82D0020C8
:102240007047000070B5D0E915439E6800224FF03A
:10225000FF3504EB42135101D3F800090028BEBF3B
:10226000D3F8000940F08040C3F80009D3F8000B10
:102270000028BEBFD3F8000B40F08040C3F8000B2D
:10228000013263189642C3F80859C3F8085BE0D2DC
:102290004FF00113C4F81C3870BD00001D4B03EB58
:1022A00080022DE9F043D2F80CC05D6DDCF81420FB
:1022B000461CD2F800E005EB063605EB40185168E5
:1022C00071450AD3D5F83438012202FA00F023EA26
:1022D0000000C5F83408BDE8F083BCF81040AEEB50
:1022E0000103A34228BF2346D8F81849A4B2B3EB90
:1022F000840FF0D89468A4F1040959F8047F37607A
:10230000A4EB09071F44042FF7D81C440B44946026
:102310005360D4E7B02C0020890141F02001016115
:1023200003699B06FCD41220FFF7D4BA10B5054C04
:102330002046FEF753FF4FF0A0436365024BA365B1
:1023400010BD00BFB02C00206C36000870B50378BB
:10235000012B054650D12A4B446D98421BD1294B85
:102360005A6B42F080025A635A6D42F080025A65FD
:102370005A6D5A6942F080025A615A6922F080020D
:102380005A610E2143205B6900F0D4FB1E4BE360D1
:102390001E4BC4F800380023C4F8003EC02323605D
:1023A0006E6D4FF40413A3633369002BFCDA012331
:1023B00033610C20FFF78EFA3369DB07FCD412205F
:1023C000FFF788FA3369002BFCDA0026A66028465E
:1023D000FFF738FF6B68C4F81068DB68C4F814684E
:1023E000C4F81C684BB90A4BA3614FF0FF3363611B
:1023F000A36843F00103A36070BD064BF4E700BF80
:10240000B02C00200038024040140040030020029D
:10241000003C30C0083C30C0F8B5446D0546002192
:102420002046FFF779FFA96D00234FF001128F6856
:10243000C4F834384FF00066C4F81C284FF0FF3061
:1024400004EB431201339F42C2F80069C2F8006BEB
:10245000C2F80809C2F8080BF2D20B686A6DEB6586
:10246000636210231361166916F01006FBD1122067
:10247000FFF730FAD4F8003823F4FE63C4F80038CC
:10248000A36943F4402343F01003A3610923C4F874
:102490001038C4F814380A4BEB604FF0C043C4F84E
:1024A000103B084BC4F8003BC4F81069C4F800396D
:1024B000EB6D03F1100243F48013EA65A362F8BDEB
:1024C0004836000840800010426D90F84E10D2F857
:1024D000003823F4FE6343EA0113C2F80038704762
:1024E0002DE9F84300EB8103456DDA68166806F0C4
:1024F0000306731E022B05EB41130C4680460FFAB0
:1025000081F94FEA41104FF00001C3F8101B4FF062
:10251000010104F1100398BFB60401FA03F39169B5
:102520008EBF334E06F1805606F5004600293AD09C
:10253000578A04F15801490137436F50D5F81C18E8
:102540000B43C5F81C382B180021C3F81019536928
:102550000127611EA7409BB3138A928B9B08012A17
:1025600088BF5343D8F85C20981842EA034301F12E
:10257000400205EB8202C8F85C0021465360284601
:10258000FFF7CAFE08EB8900C3681B8A43EA84533D
:10259000483464011E432E51D5F81C381F43C5F83A
:1025A0001C78BDE8F88305EB4917D7F8001B21F428
:1025B0000041C7F8001BD5F81C1821EA0303C0E747
:1025C00004F13F0305EB83030A4A5A60284621467B
:1025D000FFF7A2FE05EB4910D0F8003923F40043C1
:1025E000C0F80039D5F81C3823EA0707D7E700BF41
:1025F0000080001000040002826D1268C265FFF7BF
:1026000021BE00005831436D49015B5813F400406E
:1026100004D013F4001F0CBF0220012070470000FB
:102620004831436D49015B5813F4004004D013F462
:10263000001F0CBF022001207047000000EB810149
:10264000CB68196A0B6813604B68536070470000D1
:1026500000EB810330B5DD68AA691368D36019B94E
:10266000402B84BF402313606B8A1468426D1C4466
:10267000013CB4FBF3F46343033323F0030302EBA5
:10268000411043EAC44343F0C043C0F8103B2B68F9
:1026900003F00303012B09B20ED1D2F8083802EB84
:1026A000411013F4807FD0F8003B14BF43F08053F7
:1026B00043F00053C0F8003B02EB4112D2F8003B5C
:1026C00043F00443C2F8003B30BD00002DE9F04167
:1026D000244D6E6D06EB40130446D3F8087BC3F817
:1026E000087B38070AD5D6F81438190706D505EB44
:1026F00084032146DB6828465B689847FA071FD5A4
:10270000D6F81438DB071BD505EB8403D968CCB9A0
:102710008B69488A5A68B2FBF0F600FB16228AB928
:102720001868DA6890420DD2121AC3E900242023F7
:1027300083F311880B482146FFF78AFF84F3118841
:10274000BDE8F081012303FA04F26B8923EA020356
:102750006B81CB68002BF3D021460248BDE8F041E5
:10276000184700BFB02C002000EB810370B5DD6876
:10277000436D6C692668E6604A0156BB1A444FF403
:102780000020C2F810092A6802F00302012A0AB2E6
:102790000ED1D3F8080803EB421410F4807FD4F86C
:1027A000000914BF40F0805040F00050C4F8000908
:1027B00003EB4212D2F8000940F00440C2F80009CD
:1027C000D3F83408012202FA01F10143C3F83418A6
:1027D00070BD19B9402E84BF4020206020682E8A29
:1027E0008419013CB4FBF6F440EAC44040F00050C8
:1027F0001A44C6E7F8B504461E48456D05EB441378
:10280000D3F80869C3F80869F10717D5D5F8103867
:10281000DA0713D500EB8403D9684B691F68DA68BF
:10282000974218D2D21B00271A605F60202383F3DF
:1028300011882146FFF798FF87F31188330617D5D3
:10284000D5F834280123A340134211D02046BDE817
:10285000F840FFF723BD012303FA04F2038923EABA
:10286000020303818B68002BE8D021469847E5E7F7
:10287000F8BD00BFB02C00202DE9F74F984C666DD5
:102880007569B3691D4015F48058756107D02046FD
:10289000FEF70AFD03B0BDE8F04FFFF785BC002D41
:1028A00012DAD6F8003E8E489F071EBFD6F8003ECB
:1028B00023F00303C6F8003ED6F8043823F00103E2
:1028C000C6F80438FEF718FD280505D58448FFF73B
:1028D000B9FC8348FEF700FDA9040CD5D6F80838EA
:1028E00013F0060FF36823F470530CBF43F4105336
:1028F00043F4A053F3602A0704D56368DB680BB187
:1029000077489847EB0274D4AF0227D5D4F8549097
:10291000DFF8CCB100274FF0010A09EB4712D2F8DB
:10292000003B03F44023B3F5802F11D1D2F8003BD4
:10293000002B0DDA62890AFA07F322EA03036381A6
:1029400004EB8703DB68DB6813B1394658469847C8
:10295000A36D01379B68FFB29F42DED9E80617D509
:10296000676D3A6AC2F30A1002F00F0302F4F01224
:10297000B2F5802F00F08880B2F5402F08D104EB2B
:1029800083030022DB681B6A07F5805790426DD1F4
:102990002903D6F8184813D5E20302D50020FFF723
:1029A00095FEA30302D50120FFF790FE670302D531
:1029B0000220FFF78BFE260302D50320FFF786FED9
:1029C0006D037FF567AFE00702D50020FFF712FF28
:1029D000A10702D50120FFF70DFF620702D50220F3
:1029E000FFF708FF23077FF555AF0320FFF702FF2E
:1029F00050E7636DDFF8E8B0019300274FF0010A5C
:102A0000A36D9B685FFA87F999453FF67DAF019BFF
:102A100003EB4913D3F8002902F44022B2F5802FCA
:102A200022D1D3F80029002A1EDAD3F8002942F077
:102A30009042C3F80029D3F80029002AFBDB606D1F
:102A40004946FFF769FC22890AFA09F322EA0303DF
:102A5000238104EB8903DB689B6813B14946584620
:102A600098474846FFF71AFC0137C9E7910708BFA6
:102A7000D7F80080072A98BF03F8018B02F1010202
:102A800098BF4FEA182881E7023304EB830207F569
:102A900080575268D2F818C0DCF80820DCE9001C26
:102AA000A1EB0C0C002188420AD104EB830463687B
:102AB0009B699A6802449A605A6802445A6067E7C0
:102AC00011F0030F08BFD7F800808C4588BF02F8CB
:102AD000018B01F1010188BF4FEA1828E3E700BF2D
:102AE000B02C0020436D03EB4111D1F8003B43F4BF
:102AF0000013C1F8003B7047436D03EB4111D1F85F
:102B0000003943F40013C1F800397047436D03EBFB
:102B10004111D1F8003B23F40013C1F8003B70478A
:102B2000436D03EB4111D1F8003923F40013C1F8D0
:102B30000039704700F1604303F561430901C9B2F0
:102B400083F80013012200F01F039A4043099B0001
:102B500003F1604303F56143C3F880211A607047B5
:102B600030B5039C0172043304FB0325C0E906530E
:102B7000049B03630021059BC160C0E90000C0E91C
:102B80000422C0E90842C0E90A11436330BD0000D5
:102B9000416A0022C0E90411C0E90A22C2606FF054
:102BA0000101FEF707BF0000D0E90432934201D1D2
:102BB000C2680AB9181D7047002070470369196080
:102BC000C2680132C260C2691344826903619342E0
:102BD00024BF436A03610021FEF7E0BE38B5044616
:102BE0000D46E3683BB16269131D1268A36213448A
:102BF000E362002007E0237A33B929462046FEF736
:102C0000BDFE0028EDDA38BD6FF00100FBE70000E3
:102C1000C368C269013BC36043691344826943616D
:102C2000934224BF436A436100238362036B03B171
:102C30001847704770B52023044683F31188866ACD
:102C40003EB9FFF7CBFF054618B186F31188284639
:102C500070BDA36AE26A13F8015BA362934202D3D8
:102C60002046FFF7D5FF002383F31188EFE700002C
:102C70002DE9F84F04460E46174698464FF02009B6
:102C800089F311880025AA46D4F828B0BBF1000FBB
:102C900009D141462046FFF7A1FF20B18BF31188EF
:102CA0002846BDE8F88FD4E90A12A7EB050B521AA3
:102CB000934528BF9346BBF1400F1BD9334601F122
:102CC000400251F8040B43F8040B9142F9D1A36A76
:102CD00040334036A3624035D4E90A239A4202D3F6
:102CE0002046FFF795FF8AF31188BD42D8D289F3B9
:102CF0001188C9E730465A46FDF7D2FFA36A5B4404
:102D00005E44A3625D44E7E710B5029C01720433A0
:102D100004FB0321C0E906130023C0E90A33039B27
:102D20000363049BC460C0E90000C0E90422C0E959
:102D30000842436310BD0000026AC260426AC0E9F3
:102D400004220022C0E90A226FF00101FEF732BE20
:102D5000D0E904239A4201D1C26822B9184650F83A
:102D6000043B0B607047002070470000C368C269D5
:102D70000133C3604369134482694361934224BFB2
:102D8000436A43610021FEF709BE000038B50446DE
:102D90000D46E3683BB123691A1DA262E269134440
:102DA000E362002007E0237A33B929462046FEF784
:102DB000E5FD0028EDDA38BD6FF00100FBE700000B
:102DC00003691960C268013AC260C269134482692A
:102DD0000361934224BF436A036100238362036B50
:102DE00003B118477047000070B520230D46044614
:102DF000114683F31188866A2EB9FFF7C7FF10B119
:102E000086F3118870BDA36A1D70A36AE26A01335C
:102E10009342A36204D3E16920460439FFF7D0FF4F
:102E2000002080F31188EDE72DE9F84F04460D46A8
:102E3000904699464FF0200A8AF311880026B3463F
:102E4000A76A4FB949462046FFF7A0FF20B187F394
:102E500011883046BDE8F88FD4E90A073A1AA8EB82
:102E60000607974228BF1746402F1BD905F140039C
:102E700055F8042B40F8042B9D42F9D1A36A403346
:102E8000A3624036D4E90A239A4204D3E16920467A
:102E90000439FFF795FF8BF311884645D9D28AF3A1
:102EA0001188CDE729463A46FDF7FAFEA36A3B446E
:102EB0003D44A3623E44E5E7D0E904239A4217D19A
:102EC000C3689BB1836A8BB1043B9B1A0ED013601D
:102ED000C368013BC360C3691A44836902619A42B3
:102EE00024BF436A036100238362012318467047AD
:102EF0000023FBE700F088B84FF0804300225863BE
:102F00001A610222DA6070474FF080430022DA60D3
:102F1000704700004FF08043586370474FF0804384
:102F2000586A70474B6843608B688360CB68C360A6
:102F30000B6943614B6903628B6943620B680360F1
:102F40007047000008B5264B26481A6940F2FF1169
:102F50000A431A611A6922F4FF7222F001021A610F
:102F60001A691A6B0A431A631A6D0A431A651E4AD4
:102F70001B6D1146FFF7D6FF02F11C0100F58060C2
:102F8000FFF7D0FF02F1380100F58060FFF7CAFFBC
:102F900002F1540100F58060FFF7C4FF02F17001F7
:102FA00000F58060FFF7BEFF02F18C0100F5806044
:102FB000FFF7B8FF02F1A80100F58060FFF7B2FF4C
:102FC00002F1C40100F58060FFF7ACFF02F1E001FF
:102FD00000F58060FFF7A6FFBDE8084000F09AB852
:102FE00000380240000002407836000808B500F0C2
:102FF00007FAFEF733FCFFF78DF8BDE80840FEF74F
:1030000055BE000070470000104B1A6C42F00102E0
:103010001A641A6E42F001021A660D4A1B6E93681A
:1030200043F0010393604FF0804353229A624FF0C4
:10303000FF32DA6200229A615A63DA605A60012232
:103040005A6108211A601C20FFF774BD0038024045
:10305000002004E04FF0804208B51169D3680B40AE
:10306000D9B2C9439B07116107D5202383F3118887
:10307000FEF714FC002383F3118808BD08B5FFF7A1
:10308000E9FFBDE80840FFF78FB800001F4B1A6941
:103090006FEAC2526FEAD2521A611A69C2F3080289
:1030A0001A614FF0FF301A695A69586100215A6954
:1030B00059615A691A6A62F080521A621A6A02F0F9
:1030C00080521A621A6A5A6A58625A6A59625A6A6D
:1030D0001A6C42F080521A641A6E42F080521A66DC
:1030E0001A6E0B4A106840F480701060186F00F47C
:1030F0004070B0F5007F1EBF4FF48030186719672D
:10310000536823F40073536000F05AB9003802404A
:1031100000700040334B4FF080521A64324A4FF433
:10312000404111601A6842F001021A601A68910762
:10313000FCD59A6822F003029A602A4B9A6812F032
:103140000C02FBD1196801F0F90119609A601A6844
:1031500042F480321A601A689203FCD55A6F42F02A
:1031600001025A671F4B5A6F9007FCD51F4A5A60DD
:103170001A6842F080721A601B4A53685904FCD5E1
:10318000184B1A689201FCD5194A9A60194B1A68B3
:10319000194B9A42194B21D1194A1168194A914287
:1031A0001CD140F205121A60144A136803F00F0391
:1031B000052BFAD10B4B9A6842F002029A609A688A
:1031C00002F00C02082AFAD15A6C42F480425A6486
:1031D0005A6E42F480425A665B6E704740F2057246
:1031E000E1E700BF0038024000700040085440078B
:1031F00000948838002004E011640020003C024064
:1032000000ED00E041C20F41084A08B5516913685A
:103210000B4003F00103536123B1054A13680BB15E
:1032200050689847BDE80840FEF7BEBF003C01402B
:10323000282D0020084A08B5516913680B4003F097
:103240000203536123B1054A93680BB1D0689847D4
:10325000BDE80840FEF7A8BF003C0140282D002033
:10326000084A08B5516913680B4003F00403536121
:1032700023B1054A13690BB150699847BDE808406E
:10328000FEF792BF003C0140282D0020084A08B5F7
:10329000516913680B4003F00803536123B1054AD9
:1032A00093690BB1D0699847BDE80840FEF77CBF31
:1032B000003C0140282D0020084A08B551691368D8
:1032C0000B4003F01003536123B1054A136A0BB19D
:1032D000506A9847BDE80840FEF766BF003C0140D1
:1032E000282D0020174B10B55A691C68144004F4AF
:1032F00078725A61A30604D5134A936A0BB1D06A57
:103300009847600604D5104A136B0BB1506B984771
:10331000210604D50C4A936B0BB1D06B9847E2059C
:1033200004D5094A136C0BB1506C9847A30504D51A
:10333000054A936C0BB1D06C9847BDE81040FEF77E
:1033400033BF00BF003C0140282D00201A4B10B5B0
:103350005A691C68144004F47C425A61620504D521
:10336000164A136D0BB1506D9847230504D5134AC7
:10337000936D0BB1D06D9847E00404D50F4A136EDE
:103380000BB1506E9847A10404D50C4A936E0BB153
:10339000D06E9847620404D5084A136F0BB1506F82
:1033A0009847230404D5054A936F0BB1D06F984713
:1033B000BDE81040FEF7F8BE003C0140282D00207B
:1033C000062108B50846FFF7B5FB06210720FFF7E1
:1033D000B1FB06210820FFF7ADFB06210920FFF70E
:1033E000A9FB06210A20FFF7A5FB06211720FFF7FE
:1033F000A1FBBDE8084006212820FFF79BBB000089
:1034000008B5FFF743FE00F00BF8FDF7E5FEFDF70A
:10341000BDFDFFF7F7FDBDE80840FFF76BBD0000FD
:103420000023054A19460133102BC2E9001102F1AD
:103430000802F8D1704700BF282D0020034611F87C
:10344000012B03F8012B002AF9D1704753544D3357
:1034500032463F3F3F00000053544D333246343034
:10346000780053544D3332463432780053544D3340
:103470003246343436585800000000004C340008FE
:103480003F00000013040000583400083F00000013
:1034900019040000623400083F000000210400000D
:1034A0006C3400083F00000000000000090F000815
:1034B000F50E0008310F00081D0F0008290F000845
:1034C000150F0008010F0008ED0E00083D0F000861
:1034D0000000000001000000000000006D61696E46
:1034E0000000000069646C6500000000E43400081E
:1034F000D8230020502500200100000059180008A2
:10350000000000004172647550696C6F74002542C0
:103510004F415244252D424C002553455249414CC0
:103520002500000002000000000000002511000836
:103530009111000840004000E8290020F8290020EF
:103540000200000000000000030000000000000076
:10355000D51100080000000010000000082A00201B
:10356000000000000100000000000000B02C00205E
:1035700001010200491C0008591B0008F51B000846
:10358000D91B0008430000008C35000809024300E5
:10359000020100C0320904000001020201000524FA
:1035A0000010010524010001042402020524060084
:1035B00001070582030800FF09040100020A000058
:1035C00000070501024000000705810240000000DD
:1035D00012000000D835000812011001020000405E
:1035E000091241570002010203010000040309040B
:1035F00025424F41524425007370656564796265C8
:103600006566347633003031323334353637383905
:103610004142434445460000004000000040000095
:103620000040000000400000000001000000020017
:103630000000020000000200000002000000020082
:103640000000020000000200000000000D1300084E
:10365000C51500087116000840004000102D00201C
:10366000102D002001000000202D0020800000000F
:103670004001000003000000000180420000000043
:10368000AAAAAAAA00010040FFFF00000000000053
:1036900000A00A000000000100000000AAAAAAAAD7
:1036A00000000001FFFF000000000000000000001B
:1036B0000000010000000000AAAAAAAA0000000061
:1036C000FFFE0000000000000000000000000000FD
:1036D00000000000AAAAAAAA00000000FFFF000044
:1036E00000000000000000000000000000000000DA
:1036F000AAAAAAAA00000000FFFF00000000000024
:10370000000000000000000000000000AAAAAAAA11
:1037100000000000FFFF00000000000000000000AB
:103720000000000000000000AAAAAAAA00000000F1
:10373000FFFF00000000000000000000000000008B
:10374000000000000A00000000000000030000006C
:103750000000000000000000000000000000000069
:103760000000000000000000000000000000000059
:1037700000000000000000003A040000000000000B
:1037800000400F0000000000FF009600000000084D
:10379000009600000000080004000000EC3500085E
:1037A0000000000000000000000000000000000019
:1037B0000000000000000000FFFFFFFFFFFFFFFF11
:1037C000FFFFFFFFFFFFFFFFFFFFFFFFFFFFFFFF09
:1037D000FFFFFFFFFFFFFFFFFFFFFFFFFFFFFFFFF9
:1037E000FFFFFFFFFFFFFFFFFFFFFFFFFFFFFFFFE9
:1037F000FFFFFFFFFFFFFFFFFFFFFFFFFFFFFFFFD9
:10C000000006002099D200089D6F0608F96E060808
:10C01000656F0608F96E0608316F06089BD20008A6
:10C020009BD200089BD200089BD2000841640808FC
:10C030009BD200089BD200089BD200089BD200082C
:10C040009BD200089BD200089BD200089BD200081C
:10C050009BD200089BD20008D96F0808017008081D
:10C06000297008085170080879700808D91808085C
:10C07000011908082D190808591908088519080810
:10C08000AD190808D91908085D1808089BD20008DE
:10C090009BD200089BD200089BD20008A170080820
:10C0A0009BD200089BD200089BD200089BD20008BC
:10C0B0009BD20008ED710808017208089BD20008A5
:10C0C0009BD20008651F08080D2108089BD20008B4
:10C0D0009BD2000875710808897108089D710808CD
:10C0E000057108089BD200089BD200082572080839
:10C0F000297208083D72080841720808051A0808E4
:10C100009BD200089BD20008157208089BD2000839
:10C11000B1710808C57108089BD200089BD20008BD
:10C12000311A0808591A0808851A0808B11A0808A7
:10C13000DD1A08089BD200089BD200089BD2000899
:10C140009BD200089BD200089BD200086D6B0808A8
:10C15000051B0808311B08085D1B0808D971080871
:10C160009BD200089BD200089BD200089BD20008FB
:10C170009BD200089BD200089BD200089BD20008EB
:10C180009BD200089BD200089BD200089BD20008DB
:10C190009BD200089BD200089BD200089BD20008CB
:10C1A0009BD200089BD200089BD200089BD20008BB
:10C1B0009BD200089BD200089BD200089BD20008AB
:10C1C0009BD200089BD200089BD200089BD200089B
:10C1D0009BD200089BD200089BD200089BD200088B
:10C1E0002DE700080DF70008B95B010859AD0208FA
:10C1F000692E0408014D040875AB040839B304081E
:10C2000071B60408B915050835310508CDA3050830
:10C2100025B1050865610608256606083DF3060890
:10C22000911307086D680708858E07082D99070880
:10C230003DC5070805CB070800000000000000000E
:10C2400081F0004102E000BF83F0004330B54FEAC7
:10C2500041044FEA430594EA050F08BF90EA020F34
:10C260001FBF54EA000C55EA020C7FEA645C7FEAC7
:10C27000655C00F0E2804FEA5454D4EB5555B8BFEA
:10C280006D420CDD2C4480EA020281EA030382EA5B
:10C29000000083EA010180EA020281EA0303362DED
:10C2A00088BF30BD11F0004F4FEA01314FF4801CC0
:10C2B0004CEA113102D0404261EB410113F0004FD2
:10C2C0004FEA03334CEA133302D0524263EB430389
:10C2D00094EA050F00F0A780A4F10104D5F1200E27
:10C2E0000DDB02FA0EFC22FA05F2801841F1000182
:10C2F00003FA0EF2801843FA05F359410EE0A5F156
:10C3000020050EF1200E012A03FA0EFC28BF4CF086
:10C31000020C43FA05F3C01851EBE37101F000453C
:10C3200007D54FF0000EDCF1000C7EEB00006EEB49
:10C330000101B1F5801F1BD3B1F5001F0CD34908D3
:10C340005FEA30004FEA3C0C04F101044FEA44522A
:10C3500012F5800F80F09A80BCF1004F08BF5FEAB1
:10C36000500C50F1000041EB045141EA050130BD91
:10C370005FEA4C0C404141EB0101013C28BFB1F5A3
:10C38000801FE9D291F0000F04BF01460020B1FAEE
:10C3900081F308BF2033A3F10B03B3F120020CDAC1
:10C3A0000C3208DD02F1140CC2F10C0201FA0CF09F
:10C3B00021FA02F10CE002F11402D8BFC2F1200C04
:10C3C00001FA02F120FA0CFCDCBF41EA0C019040BA
:10C3D000E41AA2BF01EB0451294330BD6FEA040403
:10C3E0001F3C1CDA0C340EDC04F11404C4F12002EE
:10C3F00020FA04F001FA02F340EA030021FA04F300
:10C4000045EA030130BDC4F10C04C4F1200220FA56
:10C4100002F001FA04F340EA0300294630BD21FA94
:10C4200004F0294630BD94F0000F83F4801306BF5A
:10C4300081F480110134013D4EE77FEA645C18BF4E
:10C440007FEA655C29D094EA050F08BF90EA020FE5
:10C4500005D054EA000C04BF1946104630BD91EADD
:10C46000030F1EBF0021002030BD5FEA545C05D1E0
:10C470004000494128BF41F0004130BD14F580041F
:10C480003CBF01F5801130BD01F0004545F0FE4193
:10C4900041F470014FF0000030BD7FEA645C1ABFC8
:10C4A000194610467FEA655C1CBF0B46024650EAFF
:10C4B000013406BF52EA033591EA030F41F400212B
:10C4C00030BD00BF90F0000F04BF0021704730B5B1
:10C4D0004FF4806404F132044FF000054FF0000186
:10C4E00050E700BF90F0000F04BF0021704730B547
:10C4F0004FF4806404F1320410F0004548BF40421C
:10C500004FF000013EE700BF42004FEAE2014FEA70
:10C5100031014FEA02701FBF12F07F4393F07F4F4B
:10C5200081F06051704732F07F4208BF704793F04E
:10C530007F4F04BF41F40021704730B54FF4607461
:10C5400001F0004521F000411CE700BF50EA010264
:10C5500008BF704730B54FF000050AE050EA01020D
:10C5600008BF704730B511F0004502D5404261EB7D
:10C5700041014FF4806404F132045FEA915C3FF4BE
:10C58000D8AE4FF003025FEADC0C18BF03325FEA5B
:10C59000DC0C18BF033202EBDC02C2F1200300FA0C
:10C5A00003FC20FA02F001FA03FE40EA0E0021FA31
:10C5B00002F11444BDE600BF70B54FF0FF0C4CF41F
:10C5C000E06C1CEA11541DBF1CEA135594EA0C0FD1
:10C5D00095EA0C0F00F0DEF82C4481EA030621EA0C
:10C5E0004C5123EA4C5350EA013518BF52EA033547
:10C5F00041F4801143F4801338D0A0FB02CE4FF0F9
:10C600000005E1FB02E506F00042E0FB03E54FF028
:10C610000006E1FB03569CF0000F18BF4EF0010E20
:10C62000A4F1FF04B6F5007F64F5407404D25FEA1C
:10C630004E0E6D4146EB060642EAC62141EA5551CF
:10C640004FEAC52040EA5E504FEACE2EB4F1FD0C11
:10C6500088BFBCF5E06F1ED8BEF1004F08BF5FEA8F
:10C66000500E50F1000041EB045170BD06F0004641
:10C6700046EA010140EA020081EA0301B4EB5C04EE
:10C68000C2BFD4EB0C0541EA045170BD41F48011E6
:10C690004FF0000E013C00F3AB8014F1360FDEBF0B
:10C6A000002001F0004170BDC4F10004203C35DAE7
:10C6B0000C341BDC04F11404C4F1200500FA05F36A
:10C6C00020FA04F001FA05F240EA020001F000420B
:10C6D00021F0004110EBD37021FA04F642EB060181
:10C6E0005EEA430E08BF20EAD37070BDC4F10C04AB
:10C6F000C4F1200500FA04F320FA05F001FA04F26F
:10C7000040EA020001F0004110EBD37041F100015A
:10C710005EEA430E08BF20EAD37070BDC4F1200565
:10C7200000FA05F24EEA020E20FA04F301FA05F2CD
:10C7300043EA020321FA04F001F0004121FA04F275
:10C7400020EA020000EBD3705EEA430E08BF20EA45
:10C75000D37070BD94F0000F0FD101F0004640007F
:10C7600041EB010111F4801F08BF013CF7D041EA01
:10C77000060195F0000F18BF704703F00046520005
:10C7800043EB030313F4801F08BF013DF7D043EAD6
:10C790000603704794EA0C0F0CEA135518BF95EA8C
:10C7A0000C0F0CD050EA410618BF52EA4306D1D113
:10C7B00081EA030101F000414FF0000070BD50EA32
:10C7C000410606BF1046194652EA430619D094EABC
:10C7D0000C0F02D150EA013613D195EA0C0F05D1A6
:10C7E00052EA03361CBF104619460AD181EA0301FA
:10C7F00001F0004141F0FE4141F470014FF00000B2
:10C8000070BD41F0FE4141F4780170BD70B54FF04C
:10C81000FF0C4CF4E06C1CEA11541DBF1CEA1355CC
:10C8200094EA0C0F95EA0C0F00F0A7F8A4EB0504AE
:10C8300081EA030E52EA03354FEA013100F08880A5
:10C840004FEA03334FF0805545EA131343EA12636E
:10C850004FEA022245EA111545EA10654FEA002623
:10C860000EF000419D4208BF964244F1FD0404F5DC
:10C87000407402D25B084FEA3202B61A65EB030538
:10C880005B084FEA32024FF480104FF4002CB6EBF5
:10C89000020E75EB030E22BFB61A754640EA0C0075
:10C8A0005B084FEA3202B6EB020E75EB030E22BFB5
:10C8B000B61A754640EA5C005B084FEA3202B6EBF6
:10C8C000020E75EB030E22BFB61A754640EA9C00B5
:10C8D0005B084FEA3202B6EB020E75EB030E22BF85
:10C8E000B61A754640EADC0055EA060E18D04FEA43
:10C8F000051545EA16754FEA06164FEAC30343EAE3
:10C9000052734FEAC2025FEA1C1CC0D111F4801FAF
:10C910000BD141EA00014FF000004FF0004CB6E7A8
:10C9200011F4801F04BF01430020B4F1FD0C88BF47
:10C93000BCF5E06F3FF6AFAEB5EB030C04BFB6EB52
:10C94000020C5FEA500C50F1000041EB045170BD45
:10C950000EF0004E4EEA113114EB5C04C2BFD4EB72
:10C960000C0541EA045170BD41F480114FF0000EF6
:10C97000013C90E645EA060E8DE60CEA135594EA72
:10C980000C0F08BF95EA0C0F3FF43BAF94EA0C0F75
:10C990000AD150EA01347FF434AF95EA0C0F7FF4EA
:10C9A00025AF104619462CE795EA0C0F06D152EA3E
:10C9B00003353FF4FDAE1046194622E750EA410622
:10C9C00018BF52EA43067FF4C5AE50EA41047FF433
:10C9D0000DAF52EA43057FF4EBAE12E74FF0FF3C98
:10C9E00006E000BF4FF0010C02E000BF4FF0010C69
:10C9F0004DF804CD4FEA410C7FEA6C5C4FEA430CE2
:10CA000018BF7FEA6C5C1BD001B050EA410C0CBF30
:10CA100052EA430C91EA030F02BF90EA020F002092
:10CA2000704710F1000F91EA030F58BF994208BFF9
:10CA300090422CBFD8176FEAE37040F001007047B6
:10CA40004FEA410C7FEA6C5C02D150EA013C07D10D
:10CA50004FEA430C7FEA6C5CD6D152EA033CD3D058
:10CA60005DF8040B704700BF8446104662468C4652
:10CA70001946634600E000BF01B5FFF7B7FF002885
:10CA800048BF10F1000F01BD4DF808EDFFF7F4FFAE
:10CA90000CBF012000205DF808FB00BF4DF808ED39
:10CAA000FFF7EAFF34BF012000205DF808FB00BF5C
:10CAB0004DF808EDFFF7E0FF94BF012000205DF87E
:10CAC00008FB00BF4DF808EDFFF7CEFF94BF012033
:10CAD00000205DF808FB00BF4DF808EDFFF7C4FF2C
:10CAE00034BF012000205DF808FB00BF4FEA410C75
:10CAF0007FEA6C5C02D150EA013C0AD14FEA430C58
:10CB00007FEA6C5C02D152EA033C02D14FF0000094
:10CB100070474FF0010070474FEA410212F50012D2
:10CB200015D211D56FF47873B3EB625212D94FEA74
:10CB3000C12343F0004343EA505311F0004F23FA5E
:10CB400002F018BF404270474FF00000704750EAB3
:10CB5000013005D111F0004008BF6FF00040704770
:10CB60004FF00000704700BF4A0011D212F50012CA
:10CB700011D20DD56FF47873B3EB62520ED44FEA35
:10CB8000C12343F0004343EA505323FA02F07047B5
:10CB90004FF00000704750EA013002D14FF0FF30F3
:10CBA00070474FF0000070474FEA4102B2F1E04396
:10CBB00024BFB3F5001CDCF1FE5C0DD901F0004C84
:10CBC0004FEAC0024CEA5070B2F1004F40EB8300D4
:10CBD00008BF20F00100704711F0804F21D113F100
:10CBE0003872BCBF01F00040704741F480114FEA39
:10CBF0005252C2F11802C2F1200C10FA0CF320FAC2
:10CC000002F018BF40F001004FEAC1234FEAD323DE
:10CC100003FA0CFC40EA0C0023FA02F34FEA430348
:10CC2000CCE77FEA625307D150EA01331EBF4FF0D1
:10CC3000FE4040F44000704701F0004040F0FE40EC
:10CC400040F40000704700BF80F0004002E000BFE9
:10CC500081F0004142001FBF5FEA410392EA030FE7
:10CC60007FEA226C7FEA236C6AD04FEA1262D2EB31
:10CC70001363C1BFD218414048404140B8BF5B4236
:10CC8000192B88BF704710F0004F40F4000020F0CF
:10CC90007F4018BF404211F0004F41F4000121F0E5
:10CCA0007F4118BF494292EA030F3FD0A2F101022F
:10CCB00041FA03FC10EB0C00C3F1200301FA03F16D
:10CCC00000F0004302D5494260EB4000B0F5000F90
:10CCD00013D3B0F1807F06D340084FEA310102F14F
:10CCE0000102FE2A51D2B1F1004F40EBC25008BF01
:10CCF00020F0010040EA03007047490040EB0000CB
:10CD0000013A28BFB0F5000FEDD2B0FA80FCACF1CB
:10CD1000080CB2EB0C0200FA0CF0AABF00EBC250F8
:10CD200052421843BCBFD0401843704792F0000FE6
:10CD300081F4000106BF80F400000132013BB5E739
:10CD40004FEA41037FEA226C18BF7FEA236C21D0AF
:10CD500092EA030F04D092F0000F08BF0846704714
:10CD600090EA010F1CBF0020704712F07F4F04D1E2
:10CD7000400028BF40F00040704712F100723CBFF5
:10CD800000F50000704700F0004343F0FE4040F41F
:10CD9000000070477FEA226216BF08467FEA2363DD
:10CDA0000146420206BF5FEA412390EA010F40F4C8
:10CDB000800070474FF0000304E000BF10F0004314
:10CDC00048BF40425FEA000C08BF704743F09643FB
:10CDD00001464FF000001CE050EA010208BF704716
:10CDE0004FF000030AE000BF50EA010208BF70479D
:10CDF00011F0004302D5404261EB41015FEA010CB2
:10CE000002BF84460146002043F0B64308BFA3F1A9
:10CE10008053A3F50003BCFA8CF2083AA3EBC2538B
:10CE200010DB01FA02FC634400FA02FCC2F12002AA
:10CE3000BCF1004F20FA02F243EB020008BF20F0E1
:10CE40000100704702F1200201FA02FCC2F1200247
:10CE500050EA4C0021FA02F243EB020008BF20EA3C
:10CE6000DC7070477BB972B90029BEBF00204FF05B
:10CE7000004106E008BF00281CBF6FF000414FF0E2
:10CE8000FF3000F007BAADF1080C6DE904CE0029BF
:10CE900009DB002B1ADB00F095F8DDF804E0DDE992
:10CEA000022304B07047404261EB4101002B1BDBC1
:10CEB00000F088F8DDF804E0DDE9022304B0404228
:10CEC00061EB4101524263EB43037047524263EB13
:10CED000430300F077F8DDF804E0DDE9022304B055
:10CEE000404261EB41017047524263EB430300F063
:10CEF00069F8DDF804E0DDE9022304B0524263EB97
:10CF00004303704753B94AB9002908BF00281CBF22
:10CF10004FF0FF314FF0FF3000F0BCB9ADF1080C1D
:10CF20006DE904CE00F04EF8DDF804E0DDE90223FF
:10CF300004B07047430803F05533C01A830803F068
:10CF4000333300F03330184400EB101000F00F3092
:10CF500000EB002000EB0040000E704707EE900A47
:10CF6000F5EEC07AF1EE10FA01D400F00BB8F1EE54
:10CF7000677A08B517EE900A00F004F8404261EBBA
:10CF8000410108BDD0B5FFF7BFFA0C4B00220646A1
:10CF90000F46FFF711FBFFF7E7FD0446FFF792FA94
:10CFA000074B0022FFF708FB02460B463046394686
:10CFB000FFF74AF9FFF7D8FD2146D0BD0000F03D4C
:10CFC0000000F0412DE9F047089D04468E46002BF5
:10CFD0004DD18A42944669D9B2FA82F252B101FA2D
:10CFE00002F3C2F1200120FA01F10CFA02FC41EA3D
:10CFF000030E94404FEA1C48210CBEFBF8F61FFAC2
:10D000008CF708FB16E341EA034306FB07F199425C
:10D010000AD91CEB030306F1FF3080F01F8199420F
:10D0200040F21C81023E63445B1AA4B2B3FBF8F0E9
:10D0300008FB103344EA034400FB07F7A7420AD970
:10D040001CEB040400F1FF3380F00A81A74240F298
:10D0500007816444023840EA0640E41B00261DB103
:10D06000D4400023C5E900433146BDE8F0878B4238
:10D0700009D9002D00F0EF800026C5E900013046F7
:10D080003146BDE8F087B3FA83F6002E4AD18B42D1
:10D0900002D3824200F2F980841A61EB030301207B
:10D0A0009E46002DE0D0C5E9004EDDE702B9FFDE67
:10D0B000B2FA82F2002A40F09280A1EB0C014FEA12
:10D0C0001C471FFA8CFE0126200CB1FBF7F307FB6F
:10D0D000131140EA01410EFB03F0884208D91CEB12
:10D0E000010103F1FF3802D2884200F2CB804346AF
:10D0F000091AA4B2B1FBF7F007FB101144EA01448E
:10D100000EFB00FEA64508D91CEB040400F1FF311C
:10D1100002D2A64500F2BB800846A4EB0E0440EA0A
:10D1200003409CE7C6F12007B34022FA07FC4CEA13
:10D13000030C20FA07F401FA06F31C43F9404FEA06
:10D140001C4900FA06F3B1FBF9F8200C1FFA8CFE1B
:10D1500009FB181140EA014108FB0EF0884202FA6F
:10D1600006F20BD91CEB010108F1FF3A80F0888030
:10D17000884240F28580A8F102086144091AA4B2ED
:10D18000B1FBF9F009FB101144EA014100FB0EFE6E
:10D190008E4508D91CEB010100F1FF346CD28E459D
:10D1A0006AD90238614440EA0840A0FB0294A1EB2E
:10D1B0000E01A142C846A64656D353D05DB1B3EB8B
:10D1C000080261EB0E0101FA07F722FA06F3F140BB
:10D1D0001F43C5E9007100263146BDE8F087C2F162
:10D1E0002003D8400CFA02FC21FA03F391400143DA
:10D1F0004FEA1C471FFA8CFEB3FBF7F007FB103613
:10D200000B0C43EA064300FB0EF69E4204FA02F4BE
:10D2100008D91CEB030300F1FF382FD29E422DD911
:10D22000023863449B1B89B2B3FBF7F607FB163346
:10D2300041EA034106FB0EF38B4208D91CEB0101C6
:10D2400006F1FF3816D28B4214D9023E6144C91A46
:10D2500046EA004638E72E46284605E70646E3E656
:10D260001846F8E64B45A9D2B9EB020864EB0C0E60
:10D270000138A3E74646EAE7204694E74046D1E76F
:10D28000D0467BE7023B614432E7304609E764441D
:10D29000023842E7704700BF02E000F000F8FEE706
:10D2A00072B6374880F30888364880F309883648D4
:10D2B0003649086040F20000CCF200004EF63471AE
:10D2C000CEF200010860BFF34F8FBFF36F8F40F2C3
:10D2D0000000C0F2F0004EF68851CEF20001086066
:10D2E000BFF34F8FBFF36F8F4FF00000E1EE100AD6
:10D2F0004EF63C71CEF200010860062080F31488DF
:10D30000BFF36F8F79F0FAF878F0D2F94FF055301B
:10D310001F491B4A91423CBF41F8040BFAE71D49E3
:10D32000184A91423CBF41F8040BFAE71A491B4ADC
:10D330001B4B9A423EBF51F8040B42F8040BF8E72E
:10D3400000201849184A91423CBF41F8040BFAE703
:10D3500079F0D8F878F000FA144C154DAC4203DAA5
:10D3600054F8041B8847F9E701F0D0F9114C124D2D
:10D37000AC4203DA54F8041B8847F9E779F0C0B8E7
:10D38000000600200022002000C0000808ED00E098
:10D39000000000200006002080620A080022002011
:10D3A000E8250020E8250020F8240120E0C100083D
:10D3B00038C2000838C2000838C200082DE9F04F12
:10D3C0002DED108AC1F80CD0C3689D46BDEC108AC3
:10D3D000BDE8F08F002383F311882846A047002082
:10D3E00077F0ECFEFEE777F059FD00DFFEE7000086
:10D3F00001F0FF01102A2BDB10F0070F08D010F806
:10D40000013B013A8B422DD010F0070F42B3F6D109
:10D41000F0B441EA012141EA014122F007047FF022
:10D4200000070023F0E80256083C85EA010586EA79
:10D43000010685FA47F5A3FA87F586FA47F6A5FAB5
:10D4400087F68EB9EED1F0BC01F0FF0102F00702C1
:10D4500032B110F8013B013A83EA010313B1F8D16C
:10D460000020704701387047002D06BF354603384D
:10D47000073815F0010F07D1013015F4807F02BF86
:10D48000013015F4C03F0130F0BC0138704700BFD7
:10D4900010F8012B11F8013B012A28BF9A42F7D05E
:10D4A000D01A7047034613F8012B002AFBD1181A33
:10D4B0000138704738B50022002304460D46FFF7B7
:10D4C000EDFA28B920462946BDE8384000F00AB8F0
:10D4D000204605F1004100F005F8404261EB4101B2
:10D4E00038BD00BFD0B50C4B002206460F46FFF7F3
:10D4F00063F8FFF739FB0446FEF7E4FF074B002211
:10D50000FFF75AF802460B4630463946FEF79CFEB6
:10D51000FFF72AFB2146D0BD0000F03D0000F0419E
:10D5200000207047704700007047000070470000FF
:10D53000002070470020704700207047012070478E
:10D54000002070477047000000207047002070479F
:10D5500070470000704700000020704700207047AF
:10D5600070B5154ED6F8900203681B6898470428DA
:10D570001ADC01281DDC002814BF012441240F4BB4
:10D580001D68E86A0368DB69984701280AD0D6F865
:10D5900090220B4B9A4205D0EB6A93F89C300BB16A
:10D5A00044F08004204670BD0A2814BF01241924C9
:10D5B000E5E71924E3E700BFF0550020EC25002043
:10D5C00088580020044BD3F8900203F5267290424D
:10D5D00014BF042002207047F0550020014B93F83F
:10D5E000A0017047F04500207047000038B5C578AD
:10D5F0000B461C2D044628BF1C251C220021184662
:10D600007CF08AFE2A4604F10C01BDE838407CF02B
:10D6100039BE000038B5C5780B46102D044628BF2A
:10D6200010251022002118467CF076FE2A4604F1CF
:10D630000C01BDE838407CF025BE000008B53FF085
:10D64000D9FE30B9034A92F8243343F0040382F838
:10D65000243308BDF055002038B591ED000AF7EEEF
:10D66000000A0D4618F066FB20B10B4801F0D8FE09
:10D67000002038BDD5ED007A9FED087AF0EEE77A0C
:10D68000F4EEC77AF1EE10FA03D5034801F0DAFEA2
:10D69000EEE70320EDE700BFF02500200000003496
:10D6A00010B5044608F096FA204610BD13B58B8BD2
:10D6B000B72B0C4607D0B3F5967F22D002B0BDE859
:10D6C000104043F019BB12491E22A1F54B5001F046
:10D6D000E1FED4ED017A94ED007A0D48FCEEE77A94
:10D6E000BCEEC77A17EE903A8DED017A9DF80410E2
:10D6F0009AB201F071FB002814BF0020042002B090
:10D7000010BD04480449022201F0C4FE0020F6E7DF
:10D71000B0580020F02500208458002000B51F4A92
:10D72000DFED1F6AD2EDC77A92EDC67AD2F80C13FC
:10D73000007CA2F580538BB093F9C2310491002B89
:10D7400018BFB0EE677AD2EDC17A8DED057AFDEEA5
:10D75000E77A3E2117EE903AD2EDC27AF4EEE67AFD
:10D76000F1EE10FA58BFF0EE667AFCEEE77A1BB2E3
:10D77000ADF82030ADF8223017EE903A0022039237
:10D7800006920792ADF82430B7221A23CDE9003271
:10D7900003AA3DF0B3F80BB05DF804FBF055002090
:10D7A00000FF7F4770B5154C94F82A238AB022B940
:10D7B0000AB0BDE870403EF06DBB057C59F024FC1A
:10D7C000D4E9A261D4F88432A4F50054CDE905135C
:10D7D000B4F8C024ADF826200023CDE90733ADF816
:10D7E000243068221C23CDE90306CDE90032212133
:10D7F00003AA28463DF082F80AB070BDF05500201B
:10D80000F0B53B4CB4F8E431DE078DB0054637D5B2
:10D81000D4F89832089302238DF82430D4F8A83233
:10D82000D4F89C02CDF82530D4F8A432D4F8901264
:10D83000D4F894220590CDF8293062202123D4F821
:10D840008862D4F884720691CDE90030C221192390
:10D85000287C079203AA049603973DF04FF8287C92
:10D860003CF0E2FF0646287C3DF0E2FE00F1210399
:10D870009E4205D2287C0DB0BDE8F0403CF050BA85
:10D88000B4F8E431990731D5D4F8803308930323F1
:10D890008DF82430D4F89033D4F87C23CDF825309B
:10D8A000D4F88C33D4F88403D4F878130792CDF8E5
:10D8B000293062222123D4F87063D4F86C73059068
:10D8C000CDE90032287C0691192303AAC2210397CF
:10D8D00004963DF013F8287C3CF0A6FF0446287C13
:10D8E0003DF0A6FE00F121039C42C3D30DB0F0BD74
:10D8F000F045002005207047024BD3F890020368E2
:10D900001B681847F055002030B5CD788BB0272D17
:10D9100028BF27250C462722002168467CF0FCFC06
:10D920002A4604F10C0168467CF0ACFC1A4BD3F893
:10D93000901203F5287291422BD1DDED057A9FED0F
:10D94000177AF0EEE77AF4EEC77AF1EE10FA20D506
:10D950009DF8262002F0410141291AD1110618D460
:10D9600002F01801182914D00199C3F8A41282F00A
:10D9700004020299C3F8A812C2F380020399C3F803
:10D98000AC1283F8B4220499079AC3F8B012C3F812
:10D99000B8220BB030BD00BFF055002000000034AD
:10D9A00030B5194D95F8293385B00C464BBBCA7874
:10D9B0008DF80C30092A28BF09220C3101A8CDE9C5
:10D9C00001337CF05FFC9DF808305A1F012A18D9FA
:10D9D00003F0F703122B14D0A5F58053B3F9A2215D
:10D9E00012B9E279A3F8A221227AE179074800F07E
:10D9F000B1F9227AE179054800F0E4F9012385F8CC
:10DA0000293305B030BD00BFF0550020285100205B
:10DA1000F0B51B4BB3F9A23189B005460E4614464A
:10DA20003BB1D779BB4204D009B0BDE8F04041F02A
:10DA3000EDBCA27A637A43EA0223E27A43EA024324
:10DA40001D2B13D0212B08D01BB921462846FFF7E8
:10DA5000A7FF224631462846E6E701A92046FFF700
:10DA6000C5FD084801A901F093FFF2E701A920468E
:10DA7000FFF7D0FD034801A901F0E0FFE9E700BF8F
:10DA8000F0450020F025002013B5CA78072A4FF092
:10DA90000003044628BF07220C3168460093CDF8E6
:10DAA00003307CF0EFFBBDF900304BB901231C21A2
:10DAB000204684F80F3302B0BDE8104043F0D4B8DC
:10DAC00002B010BD30B5CD7889B01E2D28BF1E25FF
:10DAD0000C461E22002168467CF01EFC2A4604F1FA
:10DAE0000C0168467CF0CEFB0248694601F0F2FF6B
:10DAF00009B030BDF025002000B589B0084601A965
:10DB0000FFF774FD034801A901F042FF09B05DF879
:10DB100004FB00BFF02500201FB508466946FFF74B
:10DB200079FD0348694601F089FF05B05DF804FB03
:10DB3000F02500202DE9F041CC7894B0262C28BFA8
:10DB4000262488462622002107460AA87CF0E4FB0A
:10DB500002AD224608F10C010AA87CF093FB28468E
:10DB600007F062FD9DF84A30022B06AC03D0032B70
:10DB700044D0002B66D1DFED357ADDED106A9FEDE4
:10DB8000346A9DED0F7A66EEA76ADDED0E7A27EE18
:10DB9000067A67EE867A0023FDEEE66ABDEEC77A66
:10DBA000FDEEE77A17EE102A17EE901A0093204642
:10DBB00016EE903A07F058FD94E80F0085E80F0044
:10DBC00097F80F3363BB012698F8083098F80720C0
:10DBD0008DF8193000238DF818208DF81B3099220C
:10DBE0000423CDE90032387C8DF81A6003232246E5
:10DBF0002F213CF083FE14B0BDE8F081DFED137AF5
:10DC0000DDED106A9FED126A9DED0F7A66EEA76A50
:10DC1000DDED0E7A27EE067A67EE867A0123BBE702
:10DC2000BDF8446086B90B483246294601F0D2FB64
:10DC30000028C8D0084A062138463FF06FF887F818
:10DC40000F63C1E70226BFE70026BDE70000C84218
:10DC50008096184BF0250020C0E6080838B58A7A6F
:10DC60004B7A43EA0223CA7A43EA0243272B05464A
:10DC70000C460CD81C2B10D91D3B0A2B0DD8DFE805
:10DC800003F01E0C0C0C1B0C0C0C0C121500452B7D
:10DC90000FD0522B01D1FFF737FE21462846BDE8B1
:10DCA000384041F0C1BEFFF7EFFEF6E7FFF742FF55
:10DCB000F3E7FFF707FFF0E7FFF71EFFEDE7FFF7DA
:10DCC0002BFFEAE700207047C8207047012070470B
:10DCD00000207047002070470120704790F8903076
:10DCE0008B4286BF00EB8100D0F894000020704783
:10DCF00090F890308B4286BF00EB8100D0F8940002
:10DD000000207047014B93F89E017047F0450020BA
:10DD1000036A43F4E0530362436A43F4E05343620B
:10DD2000836A43F4E05383627047000013B54FF4F5
:10DD30004470CDE9002107F045FF044628B1DDE934
:10DD4000002142F0D5FB024B2360204602B010BDFB
:10DD50005CE808082DE9F04FDFF8649085B00646CE
:10DD60000F46904600254FF4837A96F89030ECB237
:10DD7000A34222D920463CF057FD834620463DF081
:10DD800057FC031D9B4514D399F9C331ADF80830F6
:10DD900094220623CDE90032422102AA20468DF8C2
:10DDA0000A708DF80B80ADF80CA03CF0A7FD013592
:10DDB000DBE720463BF0B4FFF9E705B0BDE8F08FA4
:10DDC000F04500202DE9F04FDFF8649085B006465D
:10DDD0000F469046002540F2011A96F89030ECB2BA
:10DDE000A34222D920463CF01FFD834620463DF049
:10DDF0001FFC031D9B4514D399F9C331ADF80830BE
:10DE000094220623CDE90032422102AA20468DF851
:10DE10000A708DF80B80ADF80CA03CF06FFD013559
:10DE2000DBE720463BF07CFFF9E705B0BDE8F08F6B
:10DE3000F04500201FB500F540530021D3F80C2316
:10DE40000191D3F80433029201A900F5965003938F
:10DE500001F0A0FF03F06CFB03F036F905B05DF8AC
:10DE600004FB000070B586B006461322002101A80D
:10DE700010EE105A10EE904A7CF04EFAA3238DF863
:10DE8000043095238DF8053059F0C6F81322CDF8EB
:10DE90000700CDF80B1006F57C6001A9CDF80F50F6
:10DEA000CDF8134037F032FE06B070BD2DE9F041D9
:10DEB0008AB00446884617460021232201A8109DF7
:10DEC0001E467CF029FAA3238DF8043095238DF8A3
:10DED000053001238DF8063059F09EF82B68CDF8F7
:10DEE0001B306B68CDF80700CDF80B10CDF81F3054
:10DEF0002322AB68CDF80F8001A904F57C60CDF832
:10DF00001370CDF81760CDF8233037F0FFFD0AB05D
:10DF1000BDE8F0819720704710B500F540530446E6
:10DF2000D3F8900203681B6898471A22C1B204F51F
:10DF30007C6037F0ABFF04F59070BDE810400FF047
:10DF4000F3BF000037B500F50651044601221C312D
:10DF500036F0AEFB012504F50151104A009500236F
:10DF60000831DA2033F0B4FD0D4A0095002304F5A2
:10DF70007C61FD2033F0ACFD0A4B1A68D20705D452
:10DF8000094A1D6004F58F540834146006480121C5
:10DF900003B0BDE8304033F0EDBD00BF24200A08D7
:10DFA00024A00908E8250020002200200020704756
:10DFB000002070470069C0F3401070470F299DBFD3
:10DFC000302303FB010050300020704700207047D1
:10DFD0000120704770470000036800221B68184743
:10DFE00000207047002070470020704700207047D5
:10DFF00000207047002070470020704700207047C5
:10E0000000207047002070477047000010207047C4
:10E0100000207047704700000320704701207047C0
:10E0200070470000012070470020704770470000D3
:10E0300000F507502C30704700487047880C0908DD
:10E0400008B500F54050D0F8900203681B68984767
:10E05000C0B208BD034808600F2111704FF0FF32B5
:10E060001A60704718240908002070470020704784
:10E070007047000015F0FEBE37F0AEBE43F024B985
:10E0800041F016BB05F0C0BB06F04EBA00F0D2BEA0
:10E0900000F0CCBE00F0EABE01F018BC00F0B8BE43
:10E0A00000F0BEBE00F026BF70B51F4B036000F548
:10E0B00000530446D3F8E80C1C4AC3F8382B08B1C7
:10E0C00007F08CFD1A4B236004F5805393F8842EDF
:10E0D00042B9D3F8805E2DB1284614F0FDFD2846E4
:10E0E00007F078FD04F58E500C3056F011F804F569
:10E0F0008650143045F0BAF904F6C44504F6644677
:10E10000B54204D0183D284614F054FAF8E7094BFC
:10E11000C4F8983804F694103AF04EFE04F51060F6
:10E120003AF04AFE204670BD4C25090868BA090835
:10E1300000990908106E090838B5474B044640F8A5
:10E14000043B45F00BFB04F1100006F013FB04F157
:10E15000680035F007FB04F590700FF0C7FA04F57E
:10E16000866005F0C1F904F2545007F039FD04F659
:10E17000980015F033FD04F5446045F077FA04F596
:10E18000516035F011F804F57C6037F0F3FB04F5CD
:10E190008650143045F052F904F58850103006F0DE
:10E1A000F7FB04F58E500C3055F09EFF04F58F50B0
:10E1B000083035F0E3FD04F591501C3046F0ACFC1E
:10E1C00004F5805304F593520025104683F86052FD
:10E1D000224B10301A6030F06FFF294604F596503C
:10E1E00001F0CEFE04F5C85010304EF0CBFE04F521
:10E1F000E850143052F0D6FF04F5F1500C3055F0D1
:10E20000CDF804F5F450103055F002FD04F5F75048
:10E21000083001F015FD04F5015008304FF0D6FA32
:10E2200004F5025020304BF0D3FA04F5005304F506
:10E23000055083F85C510A4D343056F0A5FA2B682E
:10E2400013B1084858F0AEFE2046074934F0A6F84E
:10E250002C60204638BD00BF0099090848640020A2
:10E26000C45B0020182209083898090810B59FEDF2
:10E27000225A9FED224A9FED222ADFED221A9FEDBE
:10E28000221A9FED220A86B00446F0EE453AB0EE1F
:10E29000453AF0EE452AF0EE450AF7EE004A5430D2
:10E2A0008DED054A8DED042ACDED031A8DED021A90
:10E2B0008DED015A8DED000A4EF004FC9DED015AE2
:10E2C0009DED054A9DED042ADDED031A9DED021A30
:10E2D0009DED000AF7EE004AF0EE453AB0EE453A01
:10E2E000F0EE452AF0EE450A04F59E704EF0EAFB8A
:10E2F000204606B010BD00BF00000000CDCCCC3DD4
:10E3000000007A450AD7A33CCDCC4C3DCDCC4C3E49
:10E31000F0B500F50055224BB5F89E211A7087B074
:10E32000044644F001FF44F0B7FC204601F002FC33
:10E3300004F5805393F83C2512F001020FD102A896
:10E34000019207F071F902A904F5965002F0D2FE8D
:10E3500028B12368019ADB6C02A920469847114E28
:10E360003368DB6A93F89C7037B195F85E311BB95E
:10E3700058F04AFEC5F86001336885F85E71DB6AC3
:10E3800093F89C20084B5A7135F05EFC35F0B0F9DB
:10E3900004F50B50183007B0BDE8F0404EF0E2BB7A
:10E3A00028230020EC250020ED5A0020FFF7B0BF05
:10E3B00010B50821044601F0A5F918B117F0BAF814
:10E3C00015F010FB0121204601F09CF910B1204608
:10E3D000FFF730FD0421204601F094F918B104F54F
:10E3E0007C6036F045FF1021204601F08BF928B102
:10E3F00004F57C60BDE8104036F0D4BF10BD0000CD
:10E40000FFF7D6BF102925D8DFE801F0090D111953
:10E410001524242424241C2424242424200000F54E
:10E420004A501C30704700F54B500430704700F5DF
:10E430004A503C30704700F54A502030704700F594
:10E440004B50704700F54A501430704700F54A5061
:10E45000183070470020704708B54FF0BBFA044BE6
:10E460001B68DB6A93F89C10BDE808404FF08EBA39
:10E47000EC250020FFF7F0BF2DE9FF410446FFF730
:10E480005BFE884B236004F5065004F500551C30F4
:10E49000FFF7ECFE002304F50F50C5F8C03304303D
:10E4A00043F030F9DFF860827F4BC5F8C43342F2A5
:10E4B000144642F21477A01943F0B2FA44F80680E9
:10E4C0003036BE42F7D1A01944F00EFD04F52C50B1
:10E4D0001C303AF0B3FE04F52C5028303AF0AEFE72
:10E4E0000023A5F8343B714BC5F8383B04F52D509B
:10E4F00057F0C6FC04F52D5604F52F57243608377F
:10E50000304614363FF002FBBE42F9D10723C5F86E
:10E51000EC3C0023A5F8F03C4FF4CB7007F058FB1F
:10E52000C5F8E80C04F53350343057F0A9FC04F575
:10E530003450383057F0A4FC5D4A13681BB904F519
:10E540002C53383313605B4BC5F8383B00265A4BCD
:10E5500003930294009604AB04F5355013E90C00C4
:10E560004021143005F06EFC04F54A5007F05CF8C9
:10E5700004F5405504F54A531833C5F890324F4B13
:10E58000C5F894324E4BC5F898324E4BC5F89C32C4
:10E590004D4BC5F8A0324FF07E53C5F8A4324B4B1B
:10E5A000C5F8BC3204F54B58494BC5F8C0320027BA
:10E5B000484BC5F8C43208F10808C5F8B072C5F870
:10E5C000AC72C5F8A87208F1040007F02DF808F144
:10E5D000140007F029F8404B4048C5F8F47204F5E0
:10E5E0004C52C5F8F872C5F8FC72186028323346F0
:10E5F0004FF6FF774FF0140C9EB20CFB060101336F
:10E60000097C0029F8D1364B36491E800B6813B1BE
:10E61000354858F0C7FC85F8293304F54C500123E0
:10E6200085F82A332C300A6056F05CF92F4BC5F878
:10E630002C332F4BC5F88043C5E9E1342D4B04F54D
:10E640004E50C5E9E3342C4BC5F89433283006F01E
:10E65000EBFF04F54F50043006F0E6FF04F54F5091
:10E66000203006F0E1FF04F54D56244BC5F8F43395
:10E67000A5F8F87306F1BC0006F0D6FF4FF0FF33A3
:10E680002436C5F858341E4B1E491E60304633F000
:10E6900085FE2046A5F8A073A5F8BC7304B0BDE8BC
:10E6A000F08100BF4C250908FC21090868BA090857
:10E6B000E05E002030E90808A5E00008C025090850
:10E6C000A422090808260908F42509081C260908B7
:10E6D000B8220908CC220908885B0020341C0908EC
:10E6E000865B0020445B00202C2209086422090874
:10E6F00069E000086DE0000871E000080000FFFF1D
:10E70000BC5A0020447A09085022090838B5054B44
:10E710001C6823680A461D68034B01462046A8472B
:10E72000002038BDEC250020F025002010B557F062
:10E7300075FF064C064B18602046FFF79DFE2046ED
:10E74000044A0549BDE8104079F0B8B8F02500202A
:10E75000EC250020E8BB0020A9E0000838B52DED2D
:10E76000028B0D46F0EE608AB0EE408A144602F04D
:10E77000DFFE90ED937AD0ED957A67EE877A90ED93
:10E78000927A67EEA87AE7EE087AC5ED007AD0EDC6
:10E79000920AD0ED937A90ED957A67EEA07A67EEC3
:10E7A000A80AE7EE480ABDEC028BC4ED000A38BDAA
:10E7B00030B52DED068B83B0F0EE409AB0EE60AA36
:10E7C0000D46044602F0B4FED0ED7F7AD0F8000288
:10E7D000B8EEE79A17F07AFB07EE900AF8EEE78AB0
:10E7E00079EEC9AA3AEE688AFDEEEAAAB0EE480AC6
:10E7F00017F04EFBBDEEC00A5DB110EE103ADFED32
:10E80000190A002BCCBF38EE608A38EE208ABDEEA4
:10E81000C80AF8EEC00A01AAB8EEEA0A694620461C
:10E82000FFF79CFFDFED107A104B009AC3F810231E
:10E8300069EEA79A019AC3F8142329EE279A2AEEC3
:10E8400027AA68EEA78AA3F58053C3EDA19A83EDAA
:10E85000A29A83EDDBAAC3EDDC8A03B0BDEC068B84
:10E8600030BD00BF00A00C470AD7233CF055002064
:10E8700038B52DED028B0D46B0EE408AF0EE608A81
:10E88000144602F055FED0ED937A9FED147AF0EE27
:10E89000E77AF4EEC77AF1EE10FA1DD4D0ED957A4E
:10E8A00090ED927A67EEE87AE8EE077AC5ED007AA5
:10E8B00090ED937AD0ED957A90ED926AC7EE876AE3
:10E8C0000120C6EE077A67EEA80AE6EE880AC4EDD4
:10E8D000000ABDEC028B38BD0020FAE700000034CE
:10E8E00030B55F4C2DED068BB4F9DC31DFED5D8A80
:10E8F0005B4285B008EE103A054604F61C303AF04B
:10E90000A1FCB8EEC88A90ED00AAB4F9DC3128EE7B
:10E91000288AF6EE009A98EE29AA04F61C3008EE32
:10E92000103A3AF08FFCB8EEC88A90ED009AB4F92C
:10E93000E03128EE288A04F6283098EE299A08EE6D
:10E94000103A3AF07FFCB4F9E231D0ED009A04F6C7
:10E9500028300AEE903A3AF075FCB8EEC88AF8EE24
:10E96000EAAAD8EE289A6A4602A990ED008A8DEDAF
:10E9700000AA9AEEA88A2846F0EE4A0AB0EE690A82
:10E980008DED038A8DED019ACDED029AFFF770FFB0
:10E9900001AA03A9F0EE490AB0EE480A2846FFF79B
:10E9A00067FF02F0C5FDD0F8000217F08FFA04F5FA
:10E9B0008053D4ED757A93EDC10A30EE270A08EE44
:10E9C000100A20EE280A17F063FAB8EEC88A30EE73
:10E9D000480A17F05DFADFED247A9DED007AB5EE76
:10E9E000C00AF1EE10FAACBF70EE676AF0EE406A52
:10E9F000B4EEE67AB4BF70EE277AF0EE407AF1EE2C
:10EA000010FA2ADD9DED016AB4EEE76AF1EE10FA24
:10EA100023D5B5EEC00AF1EE10FA08DD77EE665A9E
:10EA200037EEC65AF4EEC55AF1EE10FA13D4B5EE2D
:10EA3000C00AF1EE10FA10D537EE667A77EEC67A94
:10EA4000B4EEE77AF1EE10FACCBF0120002005B059
:10EA5000BDEC068B30BD0120F9E70020F7E700BFD1
:10EA6000F04500200000C84200A00C4770B5314CB2
:10EA70002DED028BA4F58055D5ED757A94EDC10A84
:10EA8000DFED2D8A30EE270A84B020EE280A0646F4
:10EA900017F0FEF9B5F9E231D5ED767A01EE103ACC
:10EAA000B5F9E031B0EE408A00EE903A94EDC30A39
:10EAB000B8EEC11A30EE270AF8EEE00A0C2017F083
:10EAC0003BFA20EE280A30468DED010AFFF708FFD9
:10EAD0009DED010A0146F0EE480A3046FFF768FE58
:10EAE0009DED010A03AA02A9F0EE480A3046FFF79D
:10EAF00035FEB5F9DE31002B0DDD07EE903A94EDD1
:10EB0000C27AF8EEE77AB4EEE77AF1EE10FA02DABA
:10EB100094F8C8324BB99DED020A084800F00AFB90
:10EB20009DED030A054800F0E3FB04B0BDEC028B49
:10EB300070BD00BFF05500200000C842F025002045
:10EB400038B5484C94F8243313F00101054643D1FD
:10EB5000A4F580529FED447AB2F9B02194EDC10A38
:10EB600007EE902AF8EEE77A13F0100F67EE877A37
:10EB7000F7EE006ABFEE007A08BFB0EE667AA7EE45
:10EB8000270AC3F30012DFED397A84EDC10AB5EE2E
:10EB9000C00AF1EE10FA0AD51AB161F3041384F831
:10EBA0002433B4EEE70AF1EE10FA06DC0BE0B4EE23
:10EBB000E70AF1EE10FA06DD2AB994F8243343F09F
:10EBC000100384F824339FED291ADFED290A2C2045
:10EBD00017F0B2F984EDC10A94F824339807C3F30F
:10EBE00040012ED4234A9FED207AB2F9B20107EEFC
:10EBF000900AB2F9E001B2F9E221F8EEE77A01EE0B
:10EC0000102A00EE900A1A0767EE877AF8EEE00AFB
:10EC100094EDC37AB8EEC11A18D577EE677AF4EEA0
:10EC2000E07AF1EE10FAC4EDC37A03D561F3C303C1
:10EC300084F8243394EDC30A3C2017F07DF984ED69
:10EC4000C30A2846BDE83840FFF710BF77EE877A41
:10EC5000F4EEC17AF1EE10FAC4EDC37AEADD43F0C6
:10EC60000803E5E7F05500200AD7A33C0000B443B1
:10EC700000000000F04500200A2070470120704786
:10EC8000094B93F8C812024609B1FFF7EFBE93F89B
:10EC9000291329B9A3F5805393F8E831DB0702D58E
:10ECA0001046FFF74DBF7047F05500200420704715
:10ECB0000120704730B52DED028B8BB0044658F023
:10ECC000A3F907AB054606AA05A9201D18F03AFED0
:10ECD000274A9FED288A136841F28831EB1A8B424C
:10ECE0001CD9156041F0E6FBDDED067A67EE887A07
:10ECF000054617EE900AFDF707FCDDED077A67EE93
:10ED0000887ACDE9020117EE900AFDF7FDFB1A4A59
:10ED1000CDE90001062128463AF0F8FDDDED067A3E
:10ED2000DDED070A9FED150A60EE880A27EE888A56
:10ED300060EE800A204628EE000A0021FFF738FD29
:10ED4000DDED070A9DED060A09AA08A92046FFF78E
:10ED500005FD9DED080A0A4800F0ECF99DED090A51
:10ED6000074800F0C5FA0BB0BDEC028B30BD00BF08
:10ED7000505A0020E02E6542CC2509080000C84208
:10ED8000F02500200020704701207047024B01460B
:10ED90001868026812681047E85E002008B5002075
:10EDA000FFF7F4FFC188472044F02AF8472043F0DA
:10EDB000F3FE0120FFF7EAFFC188482044F020F865
:10EDC000BDE80840482043F0E7BE0000022070473D
:10EDD00001207047FFF7B4BE08B50B46013BDBB21C
:10EDE000012B114611D85BB9472044F009F84720A0
:10EDF00043F0D2FE44F0C8F843F0AEFD012008BD58
:10EE0000482043F0FDFF4820F2E70020F7E700002C
:10EE100008B542F0D1FDBDE8084042F0ADBC0000AD
:10EE2000002100F5965002F009BB000000F254509A
:10EE300007F060BB10B5044607F04CFC90F9213098
:10EE40008BB190F8403373B194F978355BB1064BD0
:10EE50001B68DB6A93F89C302BB904F25450BDE870
:10EE6000104007F05FB910BDEC25002070B50446D6
:10EE700000F590700FF0B0FF94F8E4331B4904EBF9
:10EE80000312D2F894010A68824210D0B02202FB29
:10EE9000034294F8285492F8C12145B9022A06D9B0
:10EEA000134E08603278012A02D9013A327070BDDF
:10EEB000FDD104F54052D2F8881229B9D2F88C223B
:10EEC00012B905233370F2E7B02202FB034303F5C6
:10EED000E6730FCB04F54A5585E80F00236800223E
:10EEE000DB6C2946204698470023EBE7545A002064
:10EEF0000C2200207047000037B5044644F014F996
:10EF000043F0CAFE04F500554721002043F0C6FF38
:10EF10004821012043F0C2FFB5F8DC1101EB81016B
:10EF200001EB8101490089B2472043F01FFEB5F98A
:10EF3000E031B5F9E2110F4DC91A01EB810101EB86
:10EF40008101490089B2482043F010FE44F01CF8CA
:10EF500043F002FD04F52C5001A91C3001953AF054
:10EF6000CFF904F52C5001A9283001953AF0C8F9E1
:10EF700003B030BDCDCCCC3DF0B52DED028B00F50E
:10EF8000005785B0B7F8E021B7F8E23104466425B0
:10EF9000482012FB05F613FB05F543F0D7FD04F5F9
:10EFA000405304F507503030B0EE408ADFED230ABD
:10EFB00093EDC40A019000214DF03EFF07EE906AE8
:10EFC00038EE000AF8EEE77A0198B4EEE70AF1EEBF
:10EFD00010FA25D98DED020A07EE905A9DED027ABE
:10EFE000F8EEE77AF4EEC77AF1EE10FA03D8CDED39
:10EFF000027A4DF015FE48209DED020A43F092FD85
:10F0000097F8353B04F52C50283083B10C4B039313
:10F0100003AA02A93AF078F905B0BDEC028BF0BD65
:10F020000190CDED027A4DF0FBFD0198D4E702A9E5
:10F030003AF00AF9012387F8353BEDE70AD7A33CFC
:10F040000AD7A33C00F5405300F50050D0ED727A8A
:10F0500090ED746A93EDC47A67EE867AF0EEC76A33
:10F06000F4EEE76AF1EE10FA04D59FED180A482095
:10F0700043F058BDDFED167AB5EEC07AF1EE10FA26
:10F0800020EE270A10DDB0F8E031642213FB02F312
:10F0900007EE903AF8EEE77AF4EEC07AF1EE10FA65
:10F0A00002D59FED0C0AE2E7B0F8E231642213FBCF
:10F0B00002F307EE903AF8EEE77AF4EEC07AF1EE5A
:10F0C00010FA02DD9FED040AD1E77047000000004E
:10F0D0000000C84200A00CC600A00C4610B50446B3
:10F0E00000F5405304F5005400F50750DFED100A19
:10F0F00093EDC40A002130304DF09EFEB4F9E201D8
:10F10000B4F9E0313221C21A1B1A4A434B4301EED3
:10F11000102A00EE903A8020B8EEC11AF8EEE00A0C
:10F1200016F00AFFBDE81040482043F0FBBC00BFCA
:10F130000AD7A33C00F5005393F9C031012B03D04B
:10F14000022B03D0FFF718BFFFF77CBFFFF7C6BF46
:10F15000F0B52DED028B00F500573223B7F8DC51E6
:10F16000DFED310A00F50B5615FB03F5183600F5F7
:10F17000405393EDC50A83B00021044630464DF05C
:10F180005BFE9FED2A1ADFED2A0ABF2016F0D4FE9F
:10F190004720B0EE408A43F0D9FC9FED241ADFED02
:10F1A000240A30EE080AC02016F0C6FE6B4207EEB5
:10F1B000903AF8EEE77AB4EEE70AF1EE10FA26D9C3
:10F1C0008DED000A07EE905A9DED007AF8EEE77A91
:10F1D000F4EEC77AF1EE10FA04D83046CDED007A9D
:10F1E0004DF01EFD47209DED000A43F09BFC97F873
:10F1F000343B04F52C501C307BB10E4B019301AA1B
:10F2000069463AF081F803B0BDEC028BF0BD3046A0
:10F21000CDED007A4DF004FDD4E769463AF014F8DC
:10F22000012387F8343BEEE70AD7A33C00A08C46C5
:10F2300000A08CC60AD7A33C00F540539FED117A7D
:10F24000D3EDC57A00F5005067EE877A90ED736ACA
:10F2500090ED717A27EE067AF0EEE76AF4EEC76A6F
:10F26000F1EE10FA04D59FED080A472043F05ABC8E
:10F27000F5EEC07AF1EE10FACCBF9FED040A9FEDD7
:10F28000040AF2E70AD7233C0000000000A08C46E5
:10F2900000A08CC610B5044600F5405304F5005498
:10F2A00000F50B50DFED110A93EDC50A002118306F
:10F2B0004DF0C2FDB4F9DC314FF6CE71322213FBB2
:10F2C00002F213FB01F301EE102A00EE903AF12056
:10F2D000B8EEC11AF8EEE00AB1EE400A16F02CFEC4
:10F2E000BDE81040472043F01DBC00BF0AD7A33C37
:10F2F00000F5005393F9C131012B03D0022B03D049
:10F30000FFF726BFFFF798BFFFF7C4BFFEF704BEA5
:10F3100070B500F5005088B090F9E9010C46D8B1FD
:10F3200005210E4843F0BEFF092106460B4843F075
:10F33000B9FF01210390094843F0B4FF04AD002157
:10F340000346039A00912846314606F08DF995E868
:10F350000F0084E80F00012008B070BD585A00204B
:10F3600037B50C460022054611460F4843F0A6FF6C
:10F3700062680D48012143F0B9FFA2680A480521DF
:10F3800043F0B4FFE2680848092143F0AFFF05F5F8
:10F39000075001240DF1070129308DF8074033F0A3
:10F3A000FDFD204603B030BD585A002037B5036834
:10F3B0000191DD6C04460FF04DFD90F8C412019AE6
:10F3C000B02303FB0101AC3120462B4603B0BDE85E
:10F3D000304018477FB5044604F5965668460D46FA
:10F3E00006F022F96946304601F0A8FE48B92946E0
:10F3F0002046FFF7B5FF064650B90026304604B058
:10F4000070BD2946304601F063FD0028EFD1F4E7D6
:10F4100095E80F0004F54A5484E80F00EEE7000079
:10F4200010B5074B1B680446D86A036801211B68A6
:10F43000984704F57C600121BDE8104036F04ABBD6
:10F44000EC25002010B5074B1B680446D86A0368FA
:10F4500000211B68984704F57C600021BDE810403E
:10F4600036F038BBEC25002010B5044657F0CCFD33
:10F4700004F500540021C4F8C003472043F0DEFC2B
:10F480000021482043F0DAFC43F07EFDBDE8104047
:10F4900043F062BA70B5044604F5005304F54055D4
:10F4A00083F85C21D5F890328B420846164625D069
:10F4B000C5F890120B685B68984700B32046FFF7C9
:10F4C000AFFFD5F8900203681B6898473246C1B277
:10F4D00004F57C6036F0DAFC04F52C50002138305D
:10F4E00041F0E2FB04F5A653D3ED007A9FED067AD6
:10F4F000F8EEE77A67EE877AC5EDC17A70BD2046EF
:10F50000FFF7A0FFDDE700BF0AD7233CF7B50446AD
:10F5100000F5935010302FF05FFF5E4B04F535502F
:10F52000012214309A71DA7104F5866604F036FD12
:10F5300004F52C550823C4F844343046383504F01B
:10F54000E3FB28463EF02CFB284641F0BDFE07F0C9
:10F55000C1F82023036307F0BDF808F033F9022354
:10F56000C4F8743104F5907004F596570EF03AF92A
:10F57000384600F073FE04F58053002283F8C92555
:10F58000B4F9A43004F698001BB9B4F8A230A4F87A
:10F59000A430B4F8A41016F03FF8384600F058FF35
:10F5A0003046012104F040FA3B4B00933B4B019362
:10F5B00002AB13E9060004F57C6036F07FFA42F0F6
:10F5C000FBF99922292143F007F942F0F5F942F0BD
:10F5D0009BF904F500562046FFF78EFC96ED6D7AF8
:10F5E000DFED2F7AF0EEC76AF4EEE76AF1EE10FA7B
:10F5F00004F5405746D8D6ED6E7ADFED2A6AB0EEB4
:10F60000E76AB4EEE66AF1EE10FA3BD8DFED266A5F
:10F6100027EE267A67EEA67ABDEEC77AFDEEE77A88
:10F6200087EDA27AC7EDA37AD7F888323BB9D7F82D
:10F630008C3223B904F54A512046FFF769FE1B4B73
:10F640001B68986A03684FF47A715B68984796F96B
:10F65000E6112046FEF7D6FE014610B904F54A51E0
:10F660001C311F222046FFF715FFD6ED6F7AF5EE0D
:10F67000C07AF1EE10FA0BDD204603B0BDE8F04091
:10F68000FFF7F2BE0A4A052128463AF03FF9CBE7D8
:10F6900003B0F0BDED5A0020F02500200DF3000866
:10F6A0000000B442000034438096184BEC25002043
:10F6B0002826090808B50A2921D8DFE801F00D1825
:10F6C00011151C2020202020060000F54A5114317D
:10F6D000FFF7E0FE012008BD00F54A511C31F7E7B5
:10F6E00000F54A513C31F3E700F54B51F0E700F5E6
:10F6F0004B510431ECE700F54A512031E8E7002096
:10F70000E9E7000000F57C6036F0FABF014803210C
:10F7100043F02ABD585A002070B505462DED028BE6
:10F7200005F5405457F064FCD4F8EC32DFED1D7A57
:10F73000C31A08EE103AB8EE488A28EE278AF1EE8E
:10F74000047AB4EEE78AF1EE10FA29D504F53373A2
:10F750000FCB04F5377686E80F00D4EDBE0A94EDA2
:10F76000BD0A05F54B5068EE200A28EE000A1C3051
:10F7700006F01CFADFED0C7A94EDBF7A27EE277ABB
:10F78000D4EDB87AF8EEE77A0123E7EE087AFDEED9
:10F79000E77AC4EDB87A84F8C832BDEC028B70BD4C
:10F7A0000023F8E7BD3786350000C84230B585B084
:10F7B0006D460446284605F037FF294604F5965065
:10F7C00001F098FC50B104F54053002283F82A233D
:10F7D00095E80F0004F54A5484E80F0005B030BDE9
:10F7E00070B52DED028B00F5405482B094F8C8320C
:10F7F0000546002B5BD000F54A50D4F89022034612
:10F800003C3305F54B569A4206F11C0618D094F885
:10F810002433DA0714D43146019006F0B5F89FED91
:10F82000277A0198F6EE007AE0EE077A9FED247AC7
:10F83000FDEEE77AF8EEE77A67EE877AC4EDC17AF3
:10F84000314606F043F905F5005584EDC20A95F9F5
:10F85000C231DFED1C6AD4F89002012B05BFD4F849
:10F86000E032D4F88422D4EDC07A9B1A08BF07EEA8
:10F87000903AF8EEE77A87EEA67A84EDC77A0368C5
:10F880001B689847022812D094F824339B070ED4A3
:10F8900095F9C231D4EDC20A9FED0B8A5BB994EDA4
:10F8A000C60A78F053FB20EE080A84EDC30A02B0C2
:10F8B000BDEC028B70BD94EDC70AF2E7A00CB34516
:10F8C0000AD7233C0000C842E02E654273B50446C7
:10F8D000FFF722FF2046FFF769FF04F50055204699
:10F8E000FFF77EFFD5ED6F7AF5EEC07AF1EE10FAF4
:10F8F00009DC244B1E68F06A0368DB69984701281D
:10F9000016D102B070BD57F07FFBD5F8C03395ED2E
:10F910006F7ADFED1D6AC01A07EE900A27EE267A8D
:10F92000F8EE677AF4EEC77AF1EE10FAE1D5E8E77F
:10F93000F36A93F89C10E9B995F9E731012B10D1DE
:10F940009FED120A472043F0EDF89FED100A482082
:10F9500043F0E8F843F018FB02B0BDE8704042F015
:10F96000FBBF4720019143F04BFA0199482043F037
:10F9700047FAEFE704F54054D4F8900203689B6817
:10F980009847E7E7EC25002000007A4400000000DB
:10F9900037B54B68054613B98A68002A49D005F582
:10F9A00040540A20C4F8D4328B68C4F8D832CA68EC
:10F9B00092FBF0F2C4F8D0220B6993FBF0F3C4F889
:10F9C0000033B1F91630DFED1C7A07EE103AB1F9C9
:10F9D0001830B8EEC77A87EE276A07EE103AB1F909
:10F9E000143084EDBE6AB8EEC77AC7EE276A07EE18
:10F9F000103AB8EEC77AC4EDBF6AC7EE275AC4ED15
:10FA0000BD5A57F0F5FAC4F8EC0257F0FDFA02219E
:10FA1000C4F8F0022846FFF775FE50B105F54B53C8
:10FA200034330093D4E9B512D4F8D0322846FEF727
:10FA30003DFA03B030BD00BF0000C84210B52DED47
:10FA4000028B044691ED018ADFED207A94F841346F
:10FA500028EE278A00F58660242202FB0303F0EEDD
:10FA6000480A93ED090A03F087FCB4EE400AF1EE70
:10FA700010FAF0EE400A1FD69FED157AF0EEC07A2C
:10FA8000F4EE477AF1EE10FA16DC04F54053D3EDAC
:10FA9000C87A93F8242377EE807A5107C3EDC67AAB
:10FAA0000AD5F1EE407A00216FF38202C3EDC87AE5
:10FAB000C3F8181383F82423B0EE480ABDEC028B78
:10FAC0002046BDE81040FEF7CDB900BF0000C84297
:10FAD000FFFF7F7FB1F9003007EE903AF8EEE77A4A
:10FAE00000F5405010B5C0EDC17AB1F9023007EE13
:10FAF000903AF8EEE77A0023C0F80833C0EDC37AF5
:10FB0000B1F9002090F8243347F6FF74121B18BF98
:10FB1000012262F3000380F82433B1F9023090F837
:10FB200024231B1B18BF012363F3410280F8242305
:10FB300010BD000010B500F54054D4F8F00250B1EB
:10FB400057F062FAD4F8F032C01A41F28733984283
:10FB50008CBF00200120014B187110BDED5A002010
:10FB600070B52DED028B00F500541646B4F9E22174
:10FB700094ED760A01EE102AB4F9E02100F5405325
:10FB8000D3EDC37AD3EDC18A00EE902ADA20B8EE25
:10FB9000C11AF8EEE00A30EE270A0D4616F0CCF94D
:10FBA000B4F9E021B4F9E23107EE902AF8EEE77AF1
:10FBB0009B1A30EE670A07EE903A30EE000AF8EE34
:10FBC000E77AB7EE008A80EE277A37EE487A86ED3C
:10FBD000007A94ED750A38EE800A16F019F9B4F936
:10FBE000DC3107EE103A30EE000AB8EEC77A012099
:10FBF000C0EE077A77EEC87ABDEC028BC5ED007ACD
:10FC000070BD000070470000002070477047000082
:10FC10000020704700207047002070470020704788
:10FC20009FED010A704700BF000000009FED010A30
:10FC3000704700BF000000000020704770470000C0
:10FC400010B50446143000F019F804F12C0000F04F
:10FC500015F804F1740057F0E3F904F1F40057F0DB
:10FC6000DFF94FF0FF33C4F85031204610BD0000DB
:10FC7000014B1868704700BF5C5A002070470000B5
:10FC8000F0B52DED048B91B004466D46284605F085
:10FC9000CBFC94F8BC33002B72D004F57A730FCBF5
:10FCA00085E80F0094F8F833D4EDEC8A94EDED8AF2
:10FCB00094EDEE9A002B63D094F8D033002B5FD0F4
:10FCC0002D22002104A8D4F8C073D4F8C463D4F85A
:10FCD000C853D4F8CC437AF01FFBA3238DF810301F
:10FCE00095238DF8113046238DF8123057F094F992
:10FCF0009FED250A9FED257ACDF8171068EE807AE2
:10FD0000CDF8130067EE877AFDEEE77A17EE903AAA
:10FD100068EE007A29EE000A67EE877AADF81B30AC
:10FD2000FDEEE77A20EE070A17EE903AADF81D30A7
:10FD300016F098F8DDED017A9FED157ACDF82D706B
:10FD4000BCEEC00AF8EEE77A10EE103A67EE877A5A
:10FD5000ADF81F3017EE903ACDF82130029BCDF868
:10FD60002530039BCDF82930CDF83160CDF83550E2
:10FD7000CDF8394036F09EFE2D2204A935F0C6FE9E
:10FD800011B0BDEC048BF0BDE02E65420000C8420E
:10FD90000AD7233C30B52DED028B8BB004462422CC
:10FDA0000D4601A800217AF0B7FAA3238DF804309C
:10FDB00095238DF8053048239FED1F8A8DF8063076
:10FDC00057F02AF9D4ED817A2B68CDF80F3067EE21
:10FDD000887A95ED020ACDF80B1017EE903AD4ED23
:10FDE000827ACDF8133067EE887A6B68CDF81730D9
:10FDF00017EE903ACDF80700CDF81B3016F008F852
:10FE000010EE103A94ED830ACDF81F3020EE080A68
:10FE100015F0FEFF10EE103ACDF8233094F80C33B5
:10FE20008DF8273036F046FE242201A935F06EFE0B
:10FE30000BB0BDEC028B30BDE02E654230B587B013
:10FE400014460D461822002168467AF065FAA3236D
:10FE50008DF8003095238DF8013049238DF802305C
:10FE600057F0DAF8A3680393E36804936368CDF866
:10FE700007100593CDF803008DF80B5036F01AFEED
:10FE80001822694635F042FE07B030BD10B58EB07D
:10FE9000044602A805F0C8FB02A9204601F02AF991
:10FEA000002845D001F044FB694600F0BBFF1F224B
:10FEB000002106A87AF030FAA3238DF81830952394
:10FEC0008DF819304A238DF81A3057F0A5F8DDED7A
:10FED000037A9FED1B7A049BCDF82330F8EEE77A86
:10FEE000059BCDF8273067EE877ACDF81B0017EE1B
:10FEF000903ADDED007ACDF82B30F1EE677A17EE0F
:10FF0000903ACDF81F10204601A9CDF82F3000F00F
:10FF1000FDFB78B1DDED017AF1EE677A17EE903AEC
:10FF2000CDF8333036F0C6FD1F2206A935F0EEFDC0
:10FF30000EB010BD36F0BEFDDFED027AEEE700BF79
:10FF40000AD7233C5241C07F002303604360836093
:10FF5000C360036143618361C36103627047000052
:10FF600090F8C432B02202FB030390F8082393F800
:10FF7000A13012B1012B28BF0123184670470000A1
:10FF80002DE9F04F04468BB04FF0000A0D461BF0F0
:10FF9000CFFF84F814A204F506704FF07E5755F099
:10FFA0006FFF4FF47A73A4F8623284F86852C4F891
:10FFB0004872C4F84C72C4F8507204F51B700025E6
:10FFC00005F032FB04F52B790323C4F8803204F5E5
:10FFD0003476C4F89452C4F89852C4F89C52C4F8C9
:10FFE000A052C4F8A452C4F8A8524846FFF7ACFF88
:10FFF00004F5487B3046FFF7A7FFC4F81453C4F854
:020000040801F1
:100000001853C4F81C535846FFF79EFFC4F84453D6
:10001000C4F84853C4F84C53C4F85053C4F854536C
:10002000C4F85853C4F85C53C4F86053C4F864531C
:10003000C4F86853C4F86C53C4F87053C4F88C53B4
:10004000C4F89053C4F89453C4F8A853C4F8A45304
:10005000C4F8A053C4F8B053C4F8B453C4F8B853A8
:10006000C4F8CC53C4F8C853C4F8C453C4F89C7340
:10007000C4F8C07304F5757005F0D6FA04F57A700B
:1000800005F0D2FA04F58063C4F8FC531D6004F552
:10009000816304F583601D605D609D6005F0C4FAB6
:1000A00004F22C4304F264481D605D609D60684B5F
:1000B000C4F83C3404F50D73C4F8403404F50E73F1
:1000C000C4F8443404F50F73C4F8483404F51073CD
:1000D000C4F84C3404F24523C4F8503404F51173C9
:1000E000C4F8543404F58B6340461D605D609D6028
:1000F000FFF72AFF04F59160FFF726FF04F59763E9
:1001000004F23C421D605D609D6004F2C44304F251
:10011000A4501D605D609D6004F59A631D605D6084
:100120009D6004F2DC431D605D609D6004F2EC4361
:100130001D605D609D6004F2FC431D605D609D601C
:1001400004F5A463C2F8D470C2F8D8701D605D6075
:100150009D6004F22C531D605D609D6004F5A963F1
:100160001F605D6004F26C531D605D609D6004F56E
:10017000AF631D605D609D6004F5B2631D605D60EE
:100180009D6005F051FA04F2B45324221D605D60B5
:1001900004F2BC5351461D605D6004F2C4534046F6
:1001A0001D605D607AF0B8F804F2E450C8F8207081
:1001B000C8F81070C8F80070FFF7C6FE04F5C163F8
:1001C00004F5C7601D605D609D6004F214631D60EE
:1001D0005D609D6004F5C4631D605D609D6004F218
:1001E0002C631D605D609D6005F01EFA194B1A4975
:1001F0001C60204632F0D2F85146242258467AF04C
:100200008BF8C4F84073C4F83073C4F8207304F555
:10021000257207CA04F5287383E80700484694ED61
:10022000AA1AD4EDA90A94EDA80A16F031FA3546B7
:10023000494668466E4616F04DF90FCE0FC50FCEF3
:100240000FC533682B6020460BB0BDE8F08F00BFB0
:1002500068280908605A00201827090810B50446C4
:1002600088B001F0EFF994F93232012B02D127481E
:1002700004F070FB022B0AD1032384F8323204A964
:10028000012304F111008DF8103032F049FE94F88A
:10029000323284F8903204F23C4001F089F994F94A
:1002A0003132642B30D1652304A904F231208DF85A
:1002B000103032F073FE04A9204631F0A9F918B3CA
:1002C00004238DF818300023CDE9013303930F2365
:1002D0000593694604A831F01BFB059B28B108AAC9
:1002E00002EB8302009942F8581C0133112B05934D
:1002F000EFD954F0DBFA9DED031ADDED020A9DED16
:10030000010A652154F090FA08B010BD782609085A
:1003100070B500F5257600F528758CB00446314699
:10032000284617F0A1FDE0B996E8070085E8070028
:1003300004F52B7194EDAA1AD4EDA90A94EDA80A3C
:100340000191084616F0A4F902AD019902A816F031
:10035000C1F80FCD04F534740FC40FCD0FC42B6852
:1003600023600CB070BD000013B540F2411200F5DF
:100370000671044601A812F069FA04F23C4001F04B
:10038000FFFA20461BF0B2FF01A812F081FA02B07A
:1003900010BD0000F8B50B68C0F804324B68C0F817
:1003A00008328B68C0F80C3201F10C0607460C4687
:1003B00000F548750FCE0FC50FCE0FC533682B6003
:1003C00004F1300207CA07F5457383E8070004F11A
:1003D0003C0207CA07F5517383E8070004F148029D
:1003E00007CA07F5547383E80700543494E80700FC
:1003F00007F5577383E80700384601F037FA3846A7
:10040000BDE8F84001F01ABA13B5044600F23C40CA
:10041000019002F0ABFE04F5BB610198009102F07F
:1004200003FA0099204602B0BDE81040FFF7B2BFC2
:100430004A78064BC2F340121A754A78C2F380120A
:100440005A750A78C2F300129A757047ED5A002067
:1004500013B540F2F522044600F5067101A812F02A
:10046000F5F9002104F23C4001F0FCFC94F8603204
:1004700023B120461CF0E6F884F8600201A812F0CF
:1004800007FA02B010BD000038B590F80C330546ED
:100490000C462BB1032B0BD095F86832DB070CD43C
:1004A00005F5C7630FCB84E80F0095F8480603E015
:1004B0001BF072FF0028EFD038BD0020FCE70000E1
:1004C00000F23C4090ED350A7047000000F23C40DD
:1004D00090ED360A7047000010B490F80C230C46DB
:1004E0002AB1032A0AD000205DF8044B704700F5BA
:1004F000B26007C884E807000120F5E75DF8044B07
:100500001BF032BF90F88403431E58425841704795
:1005100038B590F80C330D468BB900F23C4001F031
:10052000A1FA044610B90024204638BD01F0EEF9C6
:10053000D5ED007A27EE800A85ED000AF4E7D0EDCC
:10054000E07AC1ED007A90F87C43002CEBD090ED7E
:10055000DE7ADFED086AB4EEE67AF1EE10FAF7EE35
:10056000006AB8BFB0EE667A67EE877AC1ED007AAE
:10057000DAE700BF0000003490F80C33032B01D100
:100580001BF072BE0020704790F80C23032A01D1A3
:100590001BF08CBF00F23C4001F0C6BE30B590F8B5
:1005A0000C3385B004460D468BB1032B18D004F5EF
:1005B000257017F093FC284601A98DED010ACDEDB9
:1005C000020A8DED031A17F0E3FA012006E000F2AB
:1005D0003C4001F0F1F90028E9D1002005B030BD20
:1005E00090F86032002BF8D01BF048FFDFE70000E6
:1005F0007FB590F80C2332B1032A4FF0000309D0E5
:10060000039304930CE000F23C4007B05DF804EB68
:1006100001F0ACBA03A90393049305931BF01AFEEF
:100620009DED030ADDED040A07B05DF804FB000050
:1006300007B590F80C3333B100F57F7003B05DF867
:1006400004EB17F0B1BB00F23C4001F08FFA6846B2
:100650008DED000ACDED010A17F0A6FB03B05DF8A1
:1006600004FB000090F80C03003818BF012070470D
:1006700008B590F80C23032A05D0BDE8084000F225
:100680003C4001F05DBA1BF0E5FD012008BD000013
:1006900010B590F80C230C461AB1032A07D000209D
:1006A00010BDBDE8104000F23C4001F0EDB91BF078
:1006B000E7FD012084ED000AF2E7000030B590F874
:1006C0000C3385B005460C4623B1032B09D000201E
:1006D00005B030BD00F23C4005B0BDE8304002F04E
:1006E000D3B8002302A9029303931BF09BFD0028BB
:1006F000EDD001A928461BF0A1FD0028E7D0029B00
:100700002360039B6360019BA360E1E790F80C23E7
:100710001AB1032A05D00020704700F23C4002F0D5
:10072000D9B81BF08BBD000090F932323BB990F87C
:10073000683213F0010F14BF03200020704703201C
:1007400070470000F7B50446FFF7EEFF05460028A6
:1007500062D0032839D194F860326BB394F86832D0
:10076000D8072BD501A920461CF096F8BDF8043017
:10077000002B18BF002594F8146206F0FD06012E28
:100780004AD10023032D019307D101A920461CF073
:100790008FF820461BF096FE064604F23C4002F01D
:1007A00025F908B994F809039DF80430D90703D551
:1007B0005A0701D59F0632D400252DE020461BF0B4
:1007C0000BFD002808BF0025D5E70025D3E713F06F
:1007D000020F2EE094F9443223B99DF80430DB096E
:1007E0002FD0E9E7002EF8D00EF034FBFFF7B8FB6E
:1007F000022807D99DF805309806DDD59DF804300C
:10080000D906D9D5FB6A93F89C30002BE5D118E0C6
:10081000DA0601D41B0718D5284603B0F0BD00281E
:10082000FAD094F80923B4F94C36002ACFD013F04B
:10083000010FF1D1154B1F68FB6A93F89C30002B18
:10084000C8D19DF804309C07E2D405F043FF05F0C1
:100850003FFE0028B0D10EF0FDFAFFF781FB022821
:10086000AAD90EF0F7FA90F8C432B02202FB0300C6
:1008700090ED2F7AF0EE007AB4EEE77AF1EE10FA0E
:100880009AD59DF80530DB09C6D195E7EC25002007
:100890002DE9F04790F8603292B00446002B00F04A
:1008A000948020461CF004F92046FFF74BFF0328F4
:1008B0007BD104F5487800274146204600970197F0
:1008C00002971BF0D1FD694620461BF0C3FD009B3B
:1008D000C4F80432019BC4F80832029BC4F80C32FD
:1008E000204600F0C3FF204600F0A8FF14F022FECF
:1008F000054620461BF088FC0028A8BFC6B203AA04
:100900004FF0FF312046BCBF95F8129395F8136362
:100910000397A8BFB146049705971BF0BFFC03A837
:1009200017F0DCFA4FF00C0A0AFB095084EDD10AEB
:10093000C4EDD20A84EDD31A04F5517100F511709B
:1009400017F0DCFA04F557770AFB065584EDC50A63
:10095000C4EDC60A84EDC71A3A464FF0FF3120466F
:1009600005F5C4751BF0AEFC95E8070006AE86E8F9
:1009700007003946304617F027FB04F52B72414635
:1009800009A815F037FD314609A815F0B5FC09A9ED
:10099000204684EDD40AC4EDD50A84EDD61A1BF0A6
:1009A00087FF09A92046FFF743FD94F84E36002B38
:1009B0003AD109A804F038FE09A920461BF0F8FC3A
:1009C00090B3012384F84E362EE0D0F864321BB980
:1009D00056F01AFBC4F86402154B1B68D86A03680A
:1009E0005B68984788B156F00FFBD4F86432C01AA0
:1009F000B4F86232984204D920461BF023FE84F8F2
:100A0000600294F860327BB14BE756F0FDFAD4F8FF
:100A10006432C01A41F287339842E4D836F04AF87B
:100A200035F08AFE0028DED112B0BDE8F08700BFA5
:100A3000EC25002090F80C3323B1032B4FF000007D
:100A400007D0704790F93222032A04D10A7001209E
:100A500070470870FBE718467047000073B50D46F5
:100A60000DF107010446FFF7E5FF064628B19DF8A2
:100A700007302BB1032B09D00026304602B070BDE1
:100A800004F5C7630FCB85E80F00F6E7294620463B
:100A90001BF082FC94F86062EFE700007FB50E4621
:100AA0000DF103010446FFF7C5FF054618B90025FF
:100AB000284604B070BD9DF8033083B1032B16D0D7
:100AC00004F5257017F00AFA01A930468DED010AE8
:100AD000CDED020A8DED031A17F05AF8E8E731461A
:100AE00004F23C4000F068FF0028E9D1DFE794F809
:100AF0006032002BDBD0314620461BF0BFFCDFE725
:100B000037B50D460DF107010446FFF793FF28B1F5
:100B10009DF8073023B1032B0FD0002003B030BD68
:100B200004F5BB631B682B6004F2DC5304F5BC6462
:100B30001B686B602368AB60F0E7204629461BF01A
:100B400089FC94F86002E9E710B50446FFF7ECFD74
:100B500018B1032807D0002010BD04F23C40BDE8C6
:100B6000104000F053BF94F86032002BF3D02046C1
:100B70001BF032FB0028EED094F8143203F0FD0392
:100B8000012BE9D194F80C03C31E58425841E3E706
:100B900010B50446FFF7C8FD80B1032810D194F8C2
:100BA000600250B156F030FAD4F86432C01A44F6FC
:100BB0002063984294BF0020012010BD0120FCE773
:100BC0000020FAE708B50246FFF7AEFD032804D17E
:100BD00010461BF06DFE012008BD0020FCE7000060
:100BE00030B585B004460191FFF742F801990546FA
:100BF00010B9002005B030BD0191FFF70BF8019945
:100C00000028F6D02846FFF709F80028F1D0B4F8FC
:100C10004C365907EED494F80933002BEAD00B4A2E
:100C20001268D26A92F89C506DB103A92046FFF772
:100C3000C9FF30B19DF80E309A07DBD5C3F38000B1
:100C4000D8E72846D6E71846D4E700BFEC250020B1
:100C50002DE9F04190F80C338CB00027032B0646A9
:100C60000C46154600970197029719D11BF0CCFA54
:100C70006A4680464FF0FF3130461BF023FBB8F147
:100C8000FF3FA760676027600DD114F053FC2B462F
:100C900090F81313224613F0DBFC0CB0BDE8F08192
:100CA0004FF0FF38EBE714F045FC2B4622465FFA85
:100CB00088F113F0CDFC95ED000A684617F04AF96B
:100CC00003A920468DED051A8DED030ACDED040A2A
:100CD00017F07AF906F52B7206F5487103A815F09E
:100CE00089FB214603A815F007FB84ED021A84ED69
:100CF000000AC4ED010A95ED007ADFED037AA7EE54
:100D0000271A84ED021AC8E70AE81C4137B50546E0
:100D100000F5067140F6033201A811F097FD284650
:100D2000FFF702FD044640B103280AD0002401A8C1
:100D300011F0AEFD204603B030BD28461BF0F0FA9E
:100D4000F5E728461BF0ECFA0446F0E708B5024642
:100D5000FFF7EAFC10B1032806D008BDBDE8084043
:100D600002F23C4000F01CBEBDE8084010461BF0FB
:100D7000ABBD00000B4610B411462BB1032B09D0BC
:100D800000205DF8044B70475DF8044B00F23C40D6
:100D900000F01CBE5DF8044B1BF00ABB13B5044603
:100DA000FFF7C2FC0A46014620460192FFF7E2FF28
:100DB00070B9084B019A1B68DB6A93F89C0038B144
:100DC00094F80C13204602B0BDE81040FFF7D2BFE4
:100DD00002B010BDEC25002037B504460D4640F2A8
:100DE000B25200F5067101A811F030FD29462046E7
:100DF0001BF0FCFA94F80C33032B054610D148B1D4
:100E000004F583612046FFF7C9FF84F828042046D3
:100E100000F05CFD01A811F03BFD284603B030BD99
:100E20000025F7E770B590F87C32DB0786B0044602
:100E30000D460CD402F04EFF437C242202FB03003B
:100E4000D0ED0B7AF1EE677AC5ED007A3BE002A8AF
:100E500004F0EAFB01A92046FFF758FCE8B90DF0C1
:100E6000F9FF94F94432022B0646E3D1FFF778F8F4
:100E70000228DFD996F8C4029FED147AB02303FB51
:100E80000066D4F87032D6F8B0209B1A07EE903A7C
:100E9000F8EEE77A67EE877AD6E702A92046FFF7F1
:100EA0007DFF0028DBD0D4F87022039BDFED076ABA
:100EB0009DED017A9B1A07EE903AF8EEE77AA7EEDD
:100EC000E67A85ED007A06B070BD00BF0AD7233CF4
:100ED000F0B50C4687B000F50671064640F686323E
:100EE00001A811F0B3FCA36853B9E36843B9636880
:100EF00033B9002701A811F0CBFC384607B0F0BD8C
:100F0000204604F099FC0028F3D094E80F0002ADCD
:100F100085E80F000021284604F050FC0746002811
:100F2000E7D096F87C32DB0704D435F0C3FD1921F5
:100F300035F058FB95E80F0006F51B7C8CE80F0098
:100F400096F87C3243F0010386F87C32304600F09C
:100F5000BDFC3FF0AFFA46213FF0A6FE3FF0AAFAF3
:100F600045213FF0A1FE054BA2681B68DB6A1A61B0
:100F7000E2685A6162689A61BCE700BFEC25002014
:100F800038B5144B1B68DD6A2B6804465B6828463D
:100F90009847F0B12B690BB96A69D2B1C4F87432C1
:100FA0006B69C4F87832A969002204F51B7004F05B
:100FB00041FB94F87C3223F0030343F0030384F8ED
:100FC0007C323FF077FABDE83840034A062138F01A
:100FD0009DBC38BDEC250020A026090810B588B0BE
:100FE00004460593FFF7A0FB0328059B4FF0000084
:100FF0000AD10690079006A802900B9801900A98D3
:10100000009020461BF044FA08B010BD38B50446E5
:10101000FEF72EFE0546D0B194F80C33032B03D017
:1010200095F84E41204638BD20461BF0A9F9FF280F
:101030000446F5D001462846FEF7F0FD0028EFD023
:1010400021462846FEF7E6FD0028E9D0EAE70446F7
:10105000E8E7000008B590F80C33032B05D014F036
:1010600069FA90F91203C0B208BD1BF0CDF8431C19
:10107000F9D1F4E708B590F80C3383B1032B03D111
:10108000BDE808401BF0B8B833F0A6FF40F6ED42CB
:101090004FF4801133F058FF4FF0FF3008BD184671
:1010A000FCE7000090F80C33032B01D11BF04CBE81
:1010B0007047000090F80C33032B01D11AF0EABFFF
:1010C000704700001BF070B810B504461DF07EFE9E
:1010D0002046FEF7D5FD2046BDE81040FEF7D6BEFF
:1010E00090F80C330BB1032B01D11BF0A9BE0020EB
:1010F0007047000030B500F5757304460D460FCB00
:1011000085E80F0094F8E40330BD0000D0F8803388
:101110000B6090F87C037047D0F888330B6090F830
:101120008503704730B500F5677304460D460FCB55
:1011300085E80F0094F8AC0330BD000030B500F531
:10114000836304460D460FCB85E80F0094F828040E
:1011500030BD000010B500F22C4203460C4607CA11
:1011600084E8070093F8380410BD00002DE9F0432F
:101170002DED028B8BB005460E461746FFF746FF56
:10118000014680462846FFF72BFD0446002848D03C
:10119000FEF76EFD4146FEF743FD86ED000A95F928
:1011A0003032002B3ADD0DF055FEFEF7D9FE012856
:1011B00034D90DF04FFE90F8C432D5EDDE7ADFED74
:1011C0005D8A96ED000AB02202FB030095F93032E9
:1011D000D0ED2F0A07EE103AF4EEE87AB8EEC77AAF
:1011E000F1EE10FAB7EE008AB8BFF0EE487A37EEAB
:1011F000201A20EE270A70EEC70A40F2B63014F02B
:101200009BFED5EDDE7AF4EEE87AF1EE10FAB8BF87
:10121000F0EE487A80EE277A86ED007A01233B7063
:1012200003E095F8083333B9387020460BB0BDECB5
:10123000028BBDE8F08395F80C334FF00009CDF830
:101240000490CDF80890CDF80C9043B1032B10D04A
:10125000CDF81090CDF81490CDF818907CB90223F9
:101260003B703246414605F23C4001F083FB0446A8
:10127000DBE701A928461BF077F80446E8E795F874
:101280000C33002BEBD004A92846FFF763FF04467C
:101290000028E4D001A904A816F046FE07A8CDED69
:1012A000080A8DED091A8DED070A17F051FA04A806
:1012B000B0EE408A17F04CFA95F93032002B30DD51
:1012C00007EE903AF8EEE77A4FF47F7070EE670A17
:1012D00037EE801AF5EEC00AF1EE10FA48BFDFEDE6
:1012E000160AF4EE410AF1EE10FAB0EE480AC8BF51
:1012F000B0EE601A14F020FEB0EE408AD5EDDE7A32
:101300009FED0C7AF4EEC77AF1EE10FAB7EE007AA0
:10131000B8BFF0EE477A88EE277A032386ED007A8D
:101320007DE7B5EEC08AF1EE10FA48BF9FED028A64
:10133000E4E700BF000000340000000010B50446E0
:10134000FFF788FE84F80D032046FFF783FE84F83C
:101350000E032046FFF77EFE84F80F032046FFF7BA
:1013600089FE04F55A7184F810032046FFF7B4F89B
:1013700084F8740300F0CAFA04F5617284EDDE0AA1
:1013800004F560712046FFF7F1FE04F5627184F800
:101390007C032046FFF7BCF804F5637184F88503ED
:1013A0002046FFF7E9F804F5677184F898032046B2
:1013B000FFF7F4F804F56C7184F8AC032046FFF7EE
:1013C0009FFB04F5707184F8BC032046FFF766FBB1
:1013D00004F5757184F8D0032046FFF755F804F53D
:1013E0007A7184F8E4032046FFF738FB84F8F803A9
:1013F0002046FFF7FDF804F5806384EDFF0A2046E0
:10140000C3ED000AFFF714F904F2044383ED000A68
:1014100004F2144204F581612046FFF719FC04F53B
:1014200083612046FFF7BAFC04F22C4184F82804BB
:101430002046FFF71DF984F8380410BD37B50D4676
:10144000044600F0FFF81DB914F074F813F030F8FA
:101450004FF4BE7204F5067101A811F0F7F994F883
:1014600069322BB92046FFF78BFD012384F86932DE
:10147000224B1D68A86A03689B6998472046FEF7BF
:1014800047FF2046FEF7C0FF204600F051FA2046F5
:10149000FFF7FEF9286B30B10368D4EDD20ADB68A0
:1014A00094EDD10A9847D4F8100208B156F01AFD0D
:1014B000204600F07DF82046FFF744F994F890327A
:1014C00084F80C0383420ED084F8900298B10C4D3E
:1014D0000C4B032808BF1D463EF0ECFF0A4A2B4682
:1014E000062138F013FA2046FFF728FF01A811F073
:1014F000CFF903B030BD054DEEE700BFEC2500206D
:10150000E7F9080897260908B82609089C2609085B
:10151000D0EDDE7A9FED057AF4EEC77AF1EE10FA9F
:10152000B7EE000AA8BFB0EE670A704700000034AB
:10153000014B1868704700BF605A00204FF0FF3021
:10154000704700000120704770470000002070477E
:10155000002070477047000070470000002070476F
:10156000002070470020704700207047002070471F
:101570000020704700207047012070470368D3F8AF
:1015800094301847002070470020704700207047B3
:1015900000207047002070470020704700207047EF
:1015A00000207047002070470020704770470000FF
:1015B0007047000008B513F0BDFF90F8130308BD95
:1015C00008B513F0B7FF90F8120308BD30B52DED44
:1015D000028B9FED1A1ADFED1A0A91ED000A87B00F
:1015E00005462D200C468DED011ACDED000A14F0B4
:1015F000A3FC9DED011ADDED000AF0EE408A2E20DD
:1016000094ED010A14F098FC9DED011ADDED000A3D
:10161000B0EE408A2F2094ED020A14F08DFC03A94D
:1016200005F52570CDED038A8DED048A8DED050A53
:1016300031F098FD07B0BDEC028B30BDC2B8323E30
:10164000C2B832BE10B5044655F0DEFCD4F8F43210
:101650001BB1C21AB2F57A7F12D30A4A1268D26A53
:1016600092F89C2002B15BB9C4F8F40294F83142BC
:1016700013F060FF80F80D4305F02CF880F825404A
:1016800010BD00BFEC2500202DE9F0432DED028BAD
:1016900091ED007AD1ED037A87B08DED047AB0EE4A
:1016A000C77AB5EEC07AF1EE10FADDE91087DDF801
:1016B0004C90CDED057A0C4615461E4606DCF0EE44
:1016C000E77AF5EEC07AF1EE10FA02DD04A816F022
:1016D000BDFB6B20B7EE001AFFEE000A9DED050A78
:1016E00014F02AFC6C2089ED000AB7EE001AFFEE18
:1016F000000A9DED040A14F01FFC04A888ED000AFE
:1017000016F02CFBB7EE008A002852D00023C9F84F
:10171000003088ED008AD4ED067A67EEA77AF4EE01
:10172000C87AF1EE10FA4ADB0023336085ED008AB7
:10173000DFED3F0A96ED000A7C20B7EE001A14F0A8
:10174000FBFB86ED000A95ED000A7D20B7EE001A3E
:10175000FFEE000A14F0F0FB85ED000AD4ED067AE6
:10176000129BDFED346AF1EE677AC3ED007A96EDF5
:10177000007AF0EEC77AF4EEE67AF1EE10FA2BD5A5
:1017800003AB02AA01A9204614F0E2FF9DED018AF5
:10179000B0EE480A76F0B8F985ED000AB0EE480AD6
:1017A00076F008FB87ED000A07B0BDEC028BBDE8C0
:1017B000F08304A816F0BEFA0028A7D1ABE738EEF4
:1017C000670A14F0EBFA86ED000A94ED087AC7EE8A
:1017D000007AC5ED007AABE794ED076AC6EE077AAA
:1017E000C7ED007A96ED007AB0EEC77AB4EEE67AED
:1017F000F1EE10FAC4D495ED007ADFED0F6AB0EE89
:10180000C76AB4EE666AF1EE10FAB9DCB4EE477A54
:10181000F1EE10FAB4D6B0EEE77AB4EE667AF1EEF5
:1018200010FAADDCF4EE677AF1EE10FABCD7A7E758
:101830000000000000000034FFFF7F7F1FB500F5AF
:101840001773039300F51673029300F51573019354
:1018500000F51473009300F5127200F5137300F590
:101860004871FFF711FF05B05DF804FB9FED156AA5
:1018700090ED817ADFED146AD0ED837A27EE067A57
:1018800067EE867A27EE267A67EEA67ABDEEC77AED
:10189000FDEEE77A80ED7E7A90ED827A27EE067A89
:1018A00017EE903A27EE267A002BB8BF03F50C43CB
:1018B000BDEEC77AB8BFA03380ED7F7AC0F80032A2
:1018C000704700BFE02E65420000C8421FB50E4BB6
:1018D0001B680446B3B1684603F0A6FE694620467D
:1018E000FFF72CFC20B16A4600212046FEF7A6FA3D
:1018F00094F87C32DB0705D504F51B7201212046E4
:10190000FEF79CFA04B010BD105D002008B502F08F
:10191000E1F9BDE8084001F06FBD000010B580F8A6
:10192000F812044655F070FBC4F8FC0210BD00002C
:1019300010B590F8F832044653B155F065FBD4F871
:10194000FC32C01AB0F57A7F84BF002384F8F832E5
:1019500094F8003353B155F057FBD4F80433C01A50
:10196000B0F57A7F84BF002384F8003310BD0000F7
:1019700000F5AA700B4607C883E8070001207047EE
:101980000023C0F89C30C0F89830C0F89430C0F8FC
:10199000A830C0F8A430C0F8A030C0F8AC30704710
:1019A00070470000024B0B604FF07C531360704790
:1019B000000048427047000008B50B4600F12801BE
:1019C000184615F02FFD012008BD000010B500F5E8
:1019D000B4700C460FC884E80F00204603F014FED4
:1019E00030B1FFF7A5FD00F51B700FC884E80F00AC
:1019F000204603F009FE80F00100C0B210BD0000D7
:101A000010B5044604F0E6F8204610BD10B5D0F835
:101A1000603104465BB155F0F7FAD4F86031C01A72
:101A200041F28833984294BF0020012010BD01206C
:101A3000FCE7000013B5009303680192D3F89030DF
:101A40009847DDE90021044628B90448044B0068A2
:101A5000C06A11F0DBF8204602B010BDEC25002072
:101A6000D827090813B504460191FEF701F9236848
:101A7000019A1B6D014608B190F84E11204602B044
:101A8000BDE810401847000030B585B00023019331
:101A90000293039303680D46DB6D01A99847044642
:101AA00020B1039B2B60204605B030BD02F012F937
:101AB000417C01F0DDFD04460028F4D002F00AF973
:101AC00001F03CFDB1EE400A85ED000AEBE70000B5
:101AD00090ED007ADFED0F7AB0EEC77AB4EEE77AD8
:101AE000F1EE10FA14D590ED017AB0EEC77AB4EEAB
:101AF000E77AF1EE10FA0BD590ED027AB0EEC77AE4
:101B0000B4EEE77AF1EE10FA4CBF012000207047E6
:101B1000002070470000003410B5FEF7A9F8044615
:101B200058B190F84E11FEF775F830B194F84E1197
:101B30002046BDE81040FEF771B8002010BD00003F
:101B400038B50D460DF086F90446FEF709FA02286D
:101B500081BF94F8C402B02303FB0040D43089BF96
:101B600007C8002085E80700012038BD2DE9F043B3
:101B70002DED028B8FB003680025DB6C0395049577
:101B800005950695029502A904469847064638B180
:101B9000FFF7BCFEDDED027A27EE800A8DED020A2A
:101BA0000DF058F9FEF7DCF90746002E50D0DDEDB8
:101BB000027AD4ED646A94ED657A23680B9527EE7A
:101BC000877A67EEA67A8DED097ACDED0A7A0C95C3
:101BD0000D959B6C0BA9204609AD98470BA928468B
:101BE00016F032F8012F8DED030ACDED040A40F214
:101BF000B3800DF02FF990F8C432DFED5B7AB02599
:101C000005FB030090ED308A28EE278AB0EE480AE3
:101C100075F07AFFF0EE408AB0EE480A76F0CAF826
:101C2000CDED0B8A8DED0C0A0DF014F990F8C4324D
:101C300005FB030090ED2F0A0BA816F025F809AD5F
:101C40008DED050ACDED060A05A896BB03C885E013
:101C50000128CED89DED020AB5EEC00AF1EE10FAC9
:101C60007FDD07AED4F89421D4F890310792304646
:101C7000089316F027F823680B950C950D959B6C2F
:101C80000BA920469847DDED077A9DED0B7A77EE9C
:101C9000877A9DED0C7ACDED077ADDED087A77EE47
:101CA000877A09ABCDED087A96E8030083E8030054
:101CB00049E0236993ED000AB7EE008A38EE408AC6
:101CC00015F0E2FF04F5BC798DED090A4846B0EE47
:101CD000480ACDED0A0A15F0D7FF0BA92846CDED2D
:101CE0000C0A8DED0B0A15F0AFFF04F5C47603AFB7
:101CF000C4ED5F0A314684ED5E0A384615F0B4FF44
:101D000004F5C0788DED090A4046B0EE480ACDEDE5
:101D10000A0A15F0B9FF0BA928468DED0B0ACDED87
:101D20000C0A15F091FF97E8030084ED600AC4EDFA
:101D3000610A86E803004946404615F085FF8DEDAF
:101D4000090ACDED0A0A9DED090ADDED0A0A0FB078
:101D5000BDEC028BBDE8F083DDE9030185E80300FB
:101D6000F1E709950A95EEE735FA8E3C10B590F843
:101D70004213044604F0C8F87C23C0B203FB0044BD
:101D8000D4F8A00010BD0000044B026F1B68DB6A92
:101D90005A60426F9A60826FDA607047EC250020CB
:101DA000F0B58FB0044613F0C5FB002302930393F4
:101DB000049390F8121301AB02AA054612F0EEFB51
:101DC00004F19407D8B39DED010AB5EEC00AF1EE17
:101DD00010FA34DD02A816F0CDF804F1B00684ED57
:101DE0002C0AC4ED2D0A84ED2E1A3946304616F021
:101DF000D1F804F17C01304616F080F804F1880136
:101E000005A88DED050ACDED060A8DED071A16F031
:101E100075F808A88DED080A9DED010ACDED090AB7
:101E20008DED0A1A16F096F80BA904F128008DED35
:101E30000B0ACDED0C0A8DED0D1A14F035FD95F859
:101E400012030C2303FB0050394600F5117016F005
:101E500055F884ED2C0AC4ED2D0A84ED2E1A0FB02E
:101E6000F0BD00002DE9F047824B00251F682DEDE5
:101E7000028BC0F89C50C0F89850C0F89450C0F83D
:101E80008450C0F88050C567C0F89050C0F88C509E
:101E9000C0F88850C0F8B850C0F8B450C0F8B0507E
:101EA0000446F86A03688AB05B680E46984704F1F6
:101EB0002809002854D055F0A7F842F20F73984231
:101EC0004ED8FB6A9FED6C8A93ED010A84ED1C0AE3
:101ED000D3ED020AC4ED1D0A93ED031A484684EDC2
:101EE0001E1A14F0D5FB3EF0E5FAD4ED1E7A67EE2B
:101EF000887A054617EE900AFAF706FBD4ED1D7AAC
:101F000067EE887ACDE9040117EE900AFAF7FCFA39
:101F1000D4ED1C7A67EE887ACDE9020117EE900ABB
:101F2000FAF7F2FA554ACDE900010621284637F0C2
:101F3000EDFC94ED1E8AB0EE480A75F0E5FD84EDE7
:101F4000650AB0EE480A75F035FF84ED640A55F075
:101F50005BF8C4F864010AB0BDEC028BBDE8F08701
:101F6000A6B194ED1C0AB4EE400AF1EE10FA0DD6BB
:101F7000D4ED1D0AF4EE600AF1EE10FA06D694EDE7
:101F80001E1AB4EE411AF1EE10FA52D713F0D2FA3B
:101F900090F813334FF00C0A0AFB030303F5C473E4
:101FA000074693E8070007AE86E807004FF01508DC
:101FB000B2EE028AF2EE068A304616F0C9FBB4EEA3
:101FC000C80AF1EE10FA38D508F1FF3818F0FF080A
:101FD0003CD1304616F0BCFBF1EE047AB4EEE70AD1
:101FE000F1EE10FA43DD9DED090ADDED087A9DED75
:101FF000078A20EE000AA7EEA70A76F0F1F8F0EEC5
:10200000400AB0EE480A75F0A1FFDDED090A84ED43
:102010001D0A9DED080AF1EE600AB1EE400A75F066
:1020200095FF84ED1C0A9FED161AD4ED1D0A94ED60
:102030001C0A484614F02CFB7BE7304616F088FB60
:10204000B4EEE80AF1EE10FABEDCC2E7384612F050
:1020500067F9384612F02CFA97F813330AFB03732A
:1020600003F5C47393E8070086E80700A4E7256733
:102070006567D8E7EC250020E02E6542E4270908D3
:10208000000000000021FFF7EDBE000037B5044658
:1020900008461546019116F05BFBB7EE007AC7EED5
:1020A000007AB4F8D03001980133A4F8D03094ED20
:1020B000337A37EE277A84ED337AB0EE007AF4EE95
:1020C000C77AF1EE10FA06D5B6EE007AF4EEC77ACA
:1020D000F1EE10FA0DDC9FED0E7AF4EEC77AF1EE18
:1020E00010FA13D59FED0B7AF4EEC77AF1EE10FAE1
:1020F0000CDDB0EE670A15F02DFF012085ED000A1A
:10210000C5ED010A85ED021A03B030BD0020FBE7E2
:1021100000247449BD37863570B52DED028B00F172
:10212000280600F134058AB029460446304615F0E9
:102130008DFFB6EE008A20EE088A2846B0EE480AE7
:1021400015F008FF07A93046CDED080A8DED091AF4
:102150008DED070A15F0E8FE30468DED010AB0EE70
:10216000480ACDED020A8DED031A15F0F3FE07A91A
:1021700028468DED070ACDED080A8DED091A15F0F8
:10218000D3FE04A901A88DED040ACDED050A8DED5D
:10219000061A15F06FFF324601A920468DED070A99
:1021A000CDED080A8DED091AFFF770FF58B954F00C
:1021B0002BFF0121C4F860012046FFF753FE0AB04F
:1021C000BDEC028B70BD2A4604A92046FFF75EFFD6
:1021D0000028ECD004F1400207A92046FFF756FF83
:1021E0000028E4D0EBE7000030B52DED028B0D4662
:1021F00083B091F842130446284603F085FEC1B22D
:102200007C2000FB0151903104F1280014F0D0F83B
:1022100068468DED000ACDED010A15F0C5FDDFED34
:102220001C7AB4EEE70AF1EE10FA05D59FED190A13
:1022300003B0BDEC028B30BD684615F007FE684662
:1022400015F08CFD0028F1D1284694ED428A03F068
:10225000CFFFF0EE400AB0EE480A13F06BFD80B9F4
:10226000284603F0C5FF84ED420AB0EE408A75F0BF
:102270004BFC84ED430AB0EE480A75F09BFD84EDFB
:10228000440A04F58671684615F046FDD0E700BFA4
:1022900000000034000000009FED0C7AB4EEC70A85
:1022A000F1EE10FA0BD4DFED0A7AB4EEE70AF1EEA4
:1022B00010FA07DCC0EE077AB0EE670A7047F7EE57
:1022C000007AF9E7F2EE047AF6E700BFF3665F3FC3
:1022D00058A00B4108B51C3015F066FDF1EE007AF0
:1022E000B4EEE70AF1EE10FA9DBFF1EE027A37EE96
:1022F000C00ADFED047A9FED040A98BF20EE270A9A
:1023000008BD00BFCDCC4C3ECDCCCC3D08B58369DB
:1023100093F9000038B10CF09DFDFDF721FE012876
:1023200094BF0020012008BDF8B52DED028B0546B5
:1023300004F0D0F904F0CCF80446B8B3FFF7F8F88D
:1023400090F8093393B32846FFF7E0FF064668B3D9
:102350000CF080FD90F8C432B02707FB030090ED2D
:102360002F7AF0EE087AB4EEE77AF1EE10FA1DD487
:1023700095ED1E8A0CF06EFD90F8C432DFED1E7AEA
:1023800007FB030090ED300A98EE270A13F056FD84
:10239000DFED1A7AB0EEC00AB4EEE70AF1EE10FAF9
:1023A00008DC54F031FE3446C5F85001BDEC028B18
:1023B0002046F8BD05F5AA7016F0CAF9B0EE408ABD
:1023C0000CF048FD90F8C4329FED0D7A07FB030333
:1023D000D3ED2F7A67EE877AB4EEE78AF1EE10FA42
:1023E000DFD554F011FED5F85041001BB0F5FA6F5F
:1023F0008CBF00240124D9E7E02E6542000034425E
:10240000CDCC4C3F10B50A4B1B68DB6A93F89C306F
:1024100004465BB954F0F8FDD4F86431C01A44F6B0
:102420001F6398428CBF0020012010BD0020FCE7F4
:10243000EC250020F8B52DED068B04460CF00AFDC6
:10244000054604F047F9064606F030FE002840F045
:10245000AA802046FFF768FF002800F0A7803046DA
:10246000FFF784FCD4F8DC30984200F01881304645
:10247000FFF77CFCD4F8DC30DFED8E7AC31A08EE6F
:10248000903AF8EE688A304668EEA78AFFF76EFC4D
:1024900094F8BC30C4F8DC00F3B9304604F02AF8F4
:1024A000D0B104F1280796F842233946304603F0AC
:1024B000A3FED4ED1D0AB0EE401A384694ED1C0A76
:1024C00014F0E6F80023C4F89030C4F88C30C4F857
:1024D0008830012384F8BC3020463146FFF784FE63
:1024E00095F8C40205EB0015B0EE408A2B6FC4F8D6
:1024F000E03004F1B000D4ED129A16F029F96368C7
:10250000DFED6D7A93ED007AB4EEE77AF1EE10FA32
:1025100068EE299AB0EE40AA01D5C3ED007A2046B4
:10252000B0EE4A0AFFF7B8FE636820EE299A93EDF1
:10253000000A29EE009AFFF7CDFE29EE009A204608
:1025400084ED249AFFF75EFF38B1D4ED247AB2EE21
:10255000007A67EE877AC4ED247AF0EE007AF4EE22
:10256000E78AF1EE10FA10D5DFED547AB4EEE7AA5F
:10257000F1EE10FA09D5DFED527A69EEA79AD4EDA3
:102580002A7AE9EEA87AC4ED2A7A9FED4E0A94EDF4
:10259000367ADFED4D7AB0EEC88A28EE008AA7EED3
:1025A000278A84ED368ABDEC068BF8BDFEF7C0FFA6
:1025B00090F80933002B72D02046FFF7A7FE0028C1
:1025C0006DD095F8C42205EB0213196FD4F8E030F2
:1025D0008B4264D0B02606FB025292ED2F7AF0EEC9
:1025E000087AB4EEE77AF1EE10FA58DBCB1AC4F8A9
:1025F000E01008EE903A95F8C4329FED341A94ED4D
:102600001E0ADFED337A06FB0353D3ED309A69EEF1
:10261000819AF8EE688A39EEC00A68EEA78A13F04C
:1026200077FCB0EE409A75F0C5FB94F8BC30B0EE84
:10263000408AF3B1F3EE047AF4EEE78AF1EE10FA91
:1026400017DC95F8C40206FB005595ED2F7AF2EEE3
:10265000027AB4EEE77AF1EE10FAFFF64AAFDFED58
:102660001D7AB0EEC99AB4EEE79AF1EE10FAFFF6D1
:1026700040AF9FED198AD4ED1D0A94ED1C0AB0EE0F
:10268000691A04F1280014F003F8012384ED248A68
:1026900084ED238A84ED228A84F8BC3029E7BDECDE
:1026A000068B04F188009FED0D0ABDE8F84015F097
:1026B000A5BC00BFBD378635CDCC4C3DC2B8B23EBF
:1026C0000AD7233CCDCC4C3ECDCC4C3F35FA8E3C8A
:1026D0006F12833A1904863F00000000EC51783FE6
:1026E00030B50C2303FB010101F1C003144693E84C
:1026F00007008BB004AD85E8070094E8070083E885
:1027000007002846FFF7E4F907AB58B194E8070043
:1027100083E807009DED070ADDED080A9DED091A23
:102720000BB030BD95E80700F2E70000F0B52DEDE5
:10273000028BD0F818318B60D0F81C31CB6085B09B
:1027400004460D4601F0C6FA06460CF083FBA36969
:1027500093F90030022B07464BD1FDF701FC02280C
:1027600047D997F8C432B02202FB0373D3F8B010F4
:102770000022284602F05EFFD4ED4A0A94ED490A91
:10278000284603F013FA94F82C3163B354F03CFC60
:102790009FED228A97F8C4128DED018A01AA0646A0
:1027A00038460BF0DBFBD4F820019FED1D0A361AEA
:1027B00007EE906AF8EE677A4FF4876027EE800A9A
:1027C000B6EE001AF0EE480A13F0B6FBDDED017A22
:1027D00030EE270A04F1F0008DED010A15F054FAED
:1027E000284603F0E3F994F82C0105B0BDEC028B08
:1027F000F0BD707C242303FB006696ED0B8AFEF788
:1028000097FED0ED9C7A9FED077AF8EEE77AE8EE36
:10281000077AFDEEE77A17EE901AA9E700000000AC
:102820006F12833A0000C842F8B5036F0B60436F24
:102830004B60836F8B6000F14C050E46074601F13B
:102840000C040FCD0FC40FCD0FC42B68236007F10C
:10285000B00207CA06F1300383E8070007F19402CB
:1028600007CA06F13C0383E8070007F11C0207CA08
:1028700006F1480383E8070006F160013846FFF7D8
:1028800055FF86F87000F8BD30B589B0044668463B
:102890000D4602F0C9FE69462046FFF797F818B9C1
:1028A0000024204609B030BD04A802F0BDFE204639
:1028B00004A9FFF73BFF04460028F1D004A96846AD
:1028C00003F0CCF885ED000AC5ED010A85ED021A8A
:1028D000E7E700001FB500230C4601A9019302930E
:1028E0000393FFF7D1FF08B1039B236004B010BD31
:1028F00030B585B001AD00230C4629460193029303
:102900000393FFF7C1FF034618B195E8030084E87D
:102910000300184605B030BDF8B506460F4615460B
:10292000FDF7A6F9044690B13946FDF773F970B189
:1029300020463946FDF772F9044640B1FDF798F993
:102940003946FDF76DF985ED000A2046F8BDFEF722
:10295000EFFD90F8083343B13046FFF7D7FC04464B
:1029600018B1D6F84C312B60EFE7D6F84C312B601C
:102970000024EAE770B52DED048B1646FFF7CCFF77
:10298000054670B3FEF7D4FD90F930424CB30CF01D
:1029900061FAFDF7E5FA012823D9E4B207EE904A7F
:1029A000B8EE678A0CF056FA90F8C43296ED009AA9
:1029B000B02202FB0300D0ED2F8AFEF7A7FF38EE0E
:1029C000281A78EEC80A40F2614029EE000A13F096
:1029D000B3FAB0EE408AFEF799FFC8EE007AC6ED72
:1029E000007ABDEC048B284670BD000008B503F0EA
:1029F00071FEBDE8084003F06BBD000010B5044651
:102A000015F054FB50B904F10C0015F04FFB28B938
:102A100004F11800BDE8104015F048BB012010BDBE
:102A200038B500F1280504462846FFF7E7FF28B12E
:102A300020460121BDE83840FFF714BAD4ED107AE2
:102A4000B7EE007AF4EEC77AF1EE10FA06D5BFEED3
:102A5000007AF4EEC77AF1EE10FA12DC2046FFF7A6
:102A60005BFB2846FFF7CAFF0028E1D1D4ED107ABE
:102A7000B2EE047AF0EEE77AF4EEC77AF1EE10FAED
:102A8000D6DC38BD10B5044615F062FE2046BDE820
:102A9000104015F0C7BA00002DE9F04F2DED048B62
:102AA0009FEDC48A95B00446F0EE408A8DED028A0F
:102AB0008DED038A8DED048AFFF7BCFC12F03AFD20
:102AC0000023054695F87921012AA8BF01229342E7
:102AD0003FD20021284611F08FFB01230028F1D0BE
:102AE00008AB0BAA002128468DED0B8A8DED0C8AD0
:102AF0008DED0D8A11F0ACFD9DED080AB5EEC00A12
:102B0000F1EE10FA23DD0BA815F034FA11A904F147
:102B100028008DED110ACDED120A8DED131A13F078
:102B2000EBFB0EA88DED0E0AB0EE680ACDED0F0A94
:102B30008DED101A15F00EFA11A904F1E4008DEDD7
:102B4000110ACDED120A8DED131A15F023FA0123A7
:102B5000B8E795F813130C2303FB015104F1280B7C
:102B600001F5C471584613F0C7FB84ED070A94EDD4
:102B70003F0AC4ED080A70EE288A84ED091AC4EDF4
:102B80003F8A0CF067F90646FEF7D2FC90F809334D
:102B900000932046FFF7BAFB80B13046FDF7E0F91D
:102BA00002280BD996F8C4226169B02303FB0263A3
:102BB00091F9001093F8D20088425FDA94ED3F7AE1
:102BC000DFED7D7AB4EEE77AF1EE10FA5DD4D4ED64
:102BD000538AFEF7A1FF38B1FDF74AF890F84E117D
:102BE000FDF71EF8F0EE408A236C626BA16A139326
:102BF000B0EE680A11A81292119115F0ABF904F524
:102C0000AA7102A88DED020ACDED030A8DED041A1A
:102C100015F0C0F954F0F8F90023074684F8143190
:102C20002046FFF773FB002865D096F8C422B02336
:102C300002FB033232445268C4F8182196F8C422C9
:102C400002FB033333449B68C4F81C3154F0DCF9B5
:102C50000123C4F8200184ED498A84ED4A8A84F86E
:102C60002C31D4F80031002B58D102AB93E8070087
:102C7000C4F80071F03484E8070006E006EB0212A5
:102C8000176FD4F80021BA4204D115B0BDEC048B03
:102C9000BDE8F08FD43393E8070094F814310DF1B8
:102CA000080C8CE807001BB904F1F00383E8070067
:102CB0000123604684F8143104F5AA7115F034F943
:102CC00011A904F14C008DED110ACDED120A8DED24
:102CD000131A13F03FFBB5EEC00AF1EE10FA8DEDBA
:102CE000110AD8BF9FED330ACDED120A8DED131AEC
:102CF00084ED530A94E794ED3F7AD4ED497ADDED03
:102D0000026AE6EE877ADDED036AC4ED497AD4ED16
:102D10004A7AE7EE267AC4ED4A7AA2E7D4ED3F7A02
:102D2000224B8DED058AF5EEC07AF1EE10FA8DEDAD
:102D3000068A0793A9D99FED1E7A94F8143167EE9D
:102D4000877AB7EE007AC7EE279A1BB9009B002B53
:102D500000F0AA80E36804F1F00102A8D3ED008A34
:102D600015F0E2F869EEA88A8DED110A11A8B0EE0F
:102D7000680ACDED120A8DED131A15F0EBF80EA9C5
:102D800005A88DED0E0ACDED0F0A8DED101A15F088
:102D900001F905A8FFF776FE05A815F0A1F9D8B14D
:102DA00054F032F9C4F860016FE700BF000080BF43
:102DB0000AE81C4100000000CDCC4C3ECDCC4C3F7D
:102DC000CDCC4C3D920A06BF920A063FC2B8B23E35
:102DD000728A0E3C5B821839012301930023CDE9EE
:102DE0000833CDE90A33CDE90C335FED0E8A4FF09D
:102DF000FF3A04F1E40895F87921012A1046A8BFAA
:102E00000120834257D20123002AFAD095F83513C6
:102E10000029F6D0B0EE690A404615F0EFF8019BA4
:102E20000DF12C09002B41D0424600212046FFF72E
:102E300057FC8DED0B0ACDED0C0A8DED0D1A4846B1
:102E4000FEF746FE70BB4846FFF71CFE484615F0ED
:102E500047F938BB05A9484615F00CF9484605A9BD
:102E60008DED080ACDED090A8DED0A1A15F0EEF880
:102E700008A8B0EE409A15F06BFCBAF1000F06D12D
:102E8000F4EEC08AF1EE10FAD8BFB0EE680AB5EEE3
:102E9000C09AF1EE10FAF7EE008A58BFF0EE408AC1
:102EA0004FF0000A0123A6E7009B96E798E8070089
:102EB00089E80700C3E7BAF1000F7FF471AF002380
:102EC00084F804312046FFF72FFA38B12046FFF787
:102ED0001DFA002840F025818DED0A8A95F81233FD
:102EE00095F878219A4240F233812B4493F8343399
:102EF000002B00F02D8195F8133395F879219A4233
:102F000040F226812B4493F83533002B00F02081CA
:102F100008A9584613F01EFA8DED080ACDED090AEE
:102F20008DED0A1A08A815F0C1F8002840F01781A5
:102F300008A815F0D5F8002840F011815FED627AFD
:102F400094ED357A68EEA78A5FED647AE7EE278A1A
:102F500004F1B000C4ED358A15F0FAFBA3685FED0B
:102F6000687A93ED007AB4EEE77AF1EE10FAF0EEBB
:102F7000408A00F1F8802046B0EE680AFFF78CF92D
:102F800008A814F0E7FFA3688DED110ACDED120A31
:102F90008DED131A93ED000A11A814F0DBFF204603
:102FA00084ED1F0AC4ED200A84ED211AFFF72AFAE6
:102FB00028B1B2EE000A04F17C0015F01FF8009B66
:102FC000B3B33046FCF7CCFF012831D996F8C402E0
:102FD000B02303FB006696ED2F7AF0EE087AB4EE8C
:102FE000E77AF1EE10FA23D595F813030C2303FBCF
:102FF000005595ED627AF1EE0C7AB4EEE77AF1EED7
:1030000010FA15DBD4ED1D7A1FED927AF4EEC77A33
:10301000F1EE10FA0CDD1FED947AF4EEC77AF1EEC2
:1030200010FA05D5B6EE000A04F17C0014F0E6FFB4
:103030005FED9A7AF4EEE78AF1EE10FA22D51FEDF1
:103040009C0A08A814F086FF0EA88DED0E0A94EDD8
:103050003F0ACDED0F0A8DED101A14F07BFF11A978
:1030600004F1A0008DED110ACDED120A8DED131AB9
:1030700014F090FFD4ED2B7A94ED3F7A77EE877AB7
:10308000C4ED2B7A94ED2B7AF1EE047AB4EEE77A64
:10309000F1EE10FA3BDB12F04DFA5FEDB27A94EDEF
:1030A0002B1A94ED280A21EE271A40F2C530F1EED2
:1030B000410A8DED011ACDED000A12F03DFF9DEDA4
:1030C000011ADDED000A84ED280A40F2C63094EDC5
:1030D000290A12F031FF9DED011ADDED000A84EDA1
:1030E000290A40F2C73094ED2A0A12F025FF04F1B4
:1030F000A00184ED2A0A04F1940014F04BFF84ED42
:103100002A8A84ED298A84ED288A84ED2B8A00237B
:10311000C4F8E430C4F8E830C4F8EC3084ED3F8AF9
:10312000A3E5E368F7EE000A93ED000A12F002FE51
:1031300000283FF4D1AE94ED1C0AB0EEC00A74F042
:1031400039FEDDED0A7A27EE800A8DED0A0AC5E622
:103150008DED0A8A8DED098A8DED088AE2E620461A
:10316000FFF75EFC1CE6C3ED007A04E72DE9F04DA5
:103170002DED048B9EB0044612F0DCF9D0EDC87A38
:1031800090ED618AF4EE487AF1EE10FA48BFB0EEA5
:10319000678ADFED5C7AB4EEE78AF1EE10FA0EDDB5
:1031A0000023C4F8E430C4F8E830C4F8EC3000235D
:1031B000C4F8FC301EB0BDEC048BBDE8F08D204699
:1031C000FEF7EEFD2046FEF7A7FFB0EE480A2046C8
:1031D000FFF762FC2046FFF723FCFEF7A9F914ADC8
:1031E00000F5347204F1280114A813F003F90FCD8F
:1031F00004F14C060FC60FCD0FC62B68336004F1E7
:10320000740204F1780304F1700104F14C0013F02E
:103210009FFA94ED1E8AB0EE480A74F075FC84EDB6
:10322000650AB0EE480A74F0C5FD204684ED640AD4
:10323000FEF7AAFDFEF77CF904F5B471FDF77EFFF9
:1032400053F0E2FED4F89831C31A632BB2D9C4F814
:10325000980133F02FFC9FED2C9A054653F0DCFECD
:10326000D4ED1C7A67EE897A074617EE900A0E466F
:10327000F9F74AF9D4ED1D7A67EE897A824617EE9E
:10328000900A8B46F9F740F994ED1E0A20EE090AE0
:1032900041EC180B12F0BCFDD4F85C0110EE108A62
:1032A000F9F732F9CDE91201D4F85801F9F72CF900
:1032B000CDE91001D4F85401F9F726F9CDE90E0152
:1032C000D4F8D800F9F720F9CDE90C01D4F8D400EE
:1032D000F9F71AF9CDE90A014046F9F715F90B4B50
:1032E00001930B4B0093CDE908018DED068BCDE9E1
:1032F00004ABCDE90276074B074A0849284633F06C
:103300001BF857E7CDCC4C3EE02E65424928090812
:1033100053280908102809081A2809089C260908B2
:1033200008B52DED048BB0EE609AF0EE408A00F007
:1033300011F9B0EE408A89EE280A74F071FEDFEDD3
:103340000B7A20EE270A74F003FEDFED097A38EEDF
:10335000278ADFED087A28EE278AF7EE007A37EE23
:10336000C00A28EE000ABDEC048B08BD41D3423EE2
:1033700033938843A1D81943FFF7D2BF08B52DED89
:10338000048B9FED189AF0EEE07AF4EEC97AF1EE34
:1033900010FAF0EE408AB0EE608A1ED400F0DAF83F
:1033A000DFED117A9FED117A70EE277A9FED100A0A
:1033B000E8EEC77A9FED0F7A27EE800AC8EE007A12
:1033C00087EE270AB4EEC90AF1EE10FA05DBBDEC70
:1033D000048BBDE8084074F003BFBDEC048BB7EE6E
:1033E000000A08BD0000003433938843F4FDD43B49
:1033F00048A18F43CDCC9C3F427CD0ED257A24213F
:1034000001FB020292ED0B0AD2ED090A30EE270A07
:10341000FFF7B4BF38B52DED088BDFED21AA9FED86
:1034200021AA9FED21BA0546B0EE409AF0EE609ACF
:10343000B0EE408A1524013CA4B25CB3F0EE490A18
:103440002846B0EE480AFFF76BFFF0EE490A70EE2F
:10345000698A284638EE2A0AFFF762FFB0EEE87A5A
:1034600070EE697AB4EECA7AF1EE10FA77EEE87A85
:1034700010D468EEAA8A40F2631088EEA70AB0EE74
:103480004B1A38EE400AF0EE4A0A12F055FDB0EE43
:10349000408AD0E7B0EE480ABDEC088B38BD00BFCB
:1034A000CDCCCC3D0AD7233C002474490023436093
:1034B0008360C360036143618361C361002380F85B
:1034C0002030704790F82020531CDBB2062B80F888
:1034D000203000EB820288BF002382ED010A88BF02
:1034E00080F82030704700004FF0FF3310B5436183
:1034F0000E4BC0F8A8300023044680F8C830A8302E
:10350000FFF7D4FF0A4BC4F8A83004F5867052F0D8
:10351000B7FC084B08491C6020462EF03FFFD4F84A
:103520009030C4F89430204610BD00BF702A0908BE
:10353000802A0908645A0020182B090808B5A83009
:1035400035F072FBDFED027A20EE270A08BD00BFDE
:1035500000007A4490ED3C0ADFED057AB0EEC07AC7
:10356000B4EEE77AF1EE10FA48BF90ED3D0A7047ED
:103570000000003473B5D0F8A43004460E4663B1A1
:1035800053F042FDD4F8A430C01A42F20F739842AF
:1035900003D894ED280A02B070BD114B1D687DB1AF
:1035A00095F84E112846FCF739FB48B195F84E11B5
:1035B00001AA2846FCF728FB10B19DED010AEAE7B5
:1035C000242101FB064494ED0A0ADFED067AB4EEED
:1035D000E70AF1EE10FA58BFB0EE670ADBE700BF6A
:1035E0005C5A002000000C4208B561B10378022B40
:1035F00002D9064853F0D6FC5A1C027000EB830037
:103600004160012008BD0846FCE700BF38290908D1
:103610002DE9F84305460E469146002400F13C088A
:103620002B78A34211DD00234A46314601200EF0DB
:1036300081FF242363430746002158F803000EF05E
:1036400089FF874204D00134EAE70020BDE8F8830F
:103650000120FBE7054B1B682BB141694A1C02D0D6
:10366000184633F04DB80020704700BF105D0020B1
:1036700002290BD8242303FB010191F8390030B152
:1036800091F83A0018B191F83B007047002070475C
:103690002DE9F047044653F0B7FCD4F8F86042F245
:1036A0001073861B9E4288BFC4F8F80000274FF0B5
:1036B000240942F2107A237CFDB2AB421CD9294680
:1036C0002046FFF7D5FF70B109FB054898ED0D0ABC
:1036D000D8ED097AD4ED250A30EE270A2046FFF707
:1036E00099FE88ED0C0A564504D909FB0540303097
:1036F0002FF02CF80137DEE7617C2046FFF73AFF18
:1037000084ED3D0ABDE8F08770B5044686B053F0FD
:103710007BFCD4F89830C31AB3F57A7F05464FD3B3
:10372000344B94ED257A1B68DFED336ADB6AD4ED08
:10373000247A93F89C60B0EEC76AB4EEE66AF1EEC4
:1037400010FA32D5B0EEE76AB4EEE66AF1EE10FA9E
:103750002BD502A801F068FF96BBFDF7E9FE02A990
:10376000FDF7ECFC60B3DDED037A9FED247AF8EE13
:10377000E77A67EE877AC4ED257AC4F89850FDF7AA
:10378000D7FEFDF7C3FA2046FFF782FF3CF092FE1A
:103790000546D4F89400F8F7B7FE194ACDE90001C0
:1037A0000621284636F0B2F80AE037EE676AF7EEEF
:1037B000005AB0EEC66AB4EEE56AF1EE10FA01DC2A
:1037C00006B070BDB0EEE76AB4EEE66AF1EE10FA4C
:1037D000F6D4002ECFD02046903080ED007A2EF027
:1037E000B5FF3CF067FE074A012106B0BDE8704016
:1037F00036F08CB8EC250020000000340AD7233CBA
:103800007929090854290908F0B52DED048B85B0F4
:1038100004464FF4537200F5867103A80FF016F8B2
:10382000D4ED227AD4ED236A9FED796A637C37EE7A
:10383000E67A2422B0EEC77AB4EEC67AF1EE10FA38
:10384000C1BF9FED747A67EE877A9FED737AE6EEDB
:10385000877A02FB03430025C4ED237A93F839608D
:103860002378E9B28B4206D904EB8103013558680D
:1038700054F02AFCF4E7DFED698A9FED698A9FED39
:10388000699A0027237CFDB2AB4264D9242303FB51
:10389000054393F83920002A5BD0D3ED0C7AF4EE7F
:1038A000E87AF1EE10FA0BDBF4EE677AF1EE10FA3B
:1038B00006D6F0EEE77AF4EE487AF1EE10FA04DD7F
:1038C000242303FB05435A6A1A63242303FB05439D
:1038D000D3ED090AD3ED0D7A93F8382070EEA70ADC
:1038E000A2B993ED0C0A2046FFF746FDD4ED257AE8
:1038F00030EE670AB4EE400AF1EE10FA16D7242330
:1039000003FB0545002385F83A3022E0012A09BF70
:10391000D3ED0C7A93ED0B0A77EEE00AD4ED3B7A07
:1039200004BF80EE897A87EE270AE3E7F0EEC07ADB
:10393000F4EE487A2423F1EE10FA03FB0545E1DCAE
:10394000012385F83A30D4ED237A37EE800A85EDED
:103950000B0A013796E7627C20461146FFF788FE86
:1039600048B1242101FB024292ED0B0AD16904F116
:10397000A80035F039F994F99C10277C002907DB61
:10398000B94205DACAB211462046FFF771FE68B99E
:1039900000226274D5B2AF4209D929462046FFF70A
:1039A00067FE01320028F5D0657400E0627420469D
:1039B000FFF7AAFE2046FFF74DFE10B1204654F057
:1039C00089FC637C242505FB034393F83930B3421B
:1039D00016D033F06FF84FF6FF7132F091FE78B1E8
:1039E000607C05FB004494F83930002B14BF0022A2
:1039F0000422019233F05EF8019A122132F012FE95
:103A000003A80EF045FF05B0BDEC048BF0BD00BF70
:103A10000AD7233C0AD7A33C48E17A3F0000003490
:103A2000FFFF7F7F002019462DE9F04F0446007C00
:103A30000F4687B004F13A0300220121D5B2A84213
:103A400003F1240305D903F8231C03F8241C0132D5
:103A5000F4E76F4B1E68F06A03685B68984740B1F3
:103A60003CF028FD6B4A062107B0BDE8F04F35F069
:103A70004DBF3CF01FFD684A062135F047FF00238B
:103A800003A904F1880003932FF01EFA0A2553F0CE
:103A9000BBFA80462046FFF7B7FE53F0B5FAA0EB1D
:103AA0000800B0F5FA7F02D95C4800F053FFB06A15
:103AB00003680A215B689847617C2046FFF7D8FDC0
:103AC0000028E7D0B06A036864215B68013D98472D
:103AD00015F0FF05DBD1524B05951B888DF806507C
:103AE000CDE90355ADF80430052553F08DFA804635
:103AF0002046FFF789FE53F087FAA0EB0800B0F5E7
:103B0000FA7FD1D8617C2046FFF7B2FD0028EFD0C4
:103B100094F810B00DF10C08A14601AA4FF0000A6C
:103B20005FFA8AF18B4516D92046FFF7A1FD50B107
:103B3000D8ED007A99ED097A137877EE877A013318
:103B4000C8ED007A13700AF1010A08F1040809F1BE
:103B500024090132E4E7B06A036864215B68013D2F
:103B6000984715F0FF05C0D1A9464FF02408237CE3
:103B70005FFA89F6B34226D906AB334413F8143CF6
:103B800033B908FB064686F83B3009F10109EEE738
:103B9000002FFAD007EE903A06AA02EB8602F8EE62
:103BA000E77A12ED030AD4ED250A204680EE270AB3
:103BB000FFF730FC08FB064002A930308DED020A09
:103BC0002FF082F9E1E7617CDFF85C902046FFF797
:103BD000D1FC002684ED3D0A4FF02408237CF7B287
:103BE000BB420FD908FB074393F83B3043B13CF08D
:103BF00061FC7B1C4A46062135F088FE0135EDB29A
:103C00000136EBE70DB907484FE707B0BDE8F08F85
:103C1000EC25002094290908BF290908D52909089D
:103C200054E50808112A0908EF29090808B5037C9A
:103C3000022B02D9034853F0B5F95A1C02741846F6
:103C400008BD00BF302A090838B5057C02460024AB
:103C5000E1B28D4206D91046FFF70AFD0134002873
:103C6000F6D138BD281E18BF0120FAE770B50D4601
:103C700009780729044606D8027E437E22B901222C
:103C80008A401343437670BD002BFCD00026227877
:103C9000F3B29A42F7D904EB8303294658680368C4
:103CA000DB6898470136F2E737B50D460192FFF71A
:103CB000CBFF0199044630B90448054B00682A46F9
:103CC000C06A0EF0A3FF204603B030BDEC250020F3
:103CD000B32B0A08014B1868704700BF645A0020D4
:103CE00010B50446006810B103685B689847204629
:103CF00010BD000010B50446006810B103685B6891
:103D00009847204610BD000070B5D0ED247A9FED95
:103D1000427AF0EEE77AF4EEC77A0123F1EE10FA78
:103D20008AB00446037609D49030002309A905908F
:103D300009932FF0C9F805982EF008FD0026E663D8
:103D40002666C4F88460762231462046FFF760FC80
:103D5000054600283BD0CDE90666079A0992002364
:103D600009A92046CDE9073354F0DCFD0146204681
:103D7000FFF73AFC09A8FFF7BDFF08A8FFF7BAFF55
:103D800007A8FFF7ADFF15B106A8FFF7A9FF237835
:103D9000032B3FD0237C032B3CD0D4F80031DA0432
:103DA00003D5637E0BB9012363760025637EEB4068
:103DB000DB07EAB21AD40135082DF7D123781BB1FD
:103DC000237C0BB163682BBB144800F0C3FD144B7C
:103DD0001B68596804220B68CDE90102114A009260
:103DE0001E680246762307A8B047B6E7382005923A
:103DF00001F0E8FE064618B1059A214654F0DEFAB5
:103E000031462046FFF7F0FB2378032B02D0237CBA
:103E1000032BD0D10AB070BD00000034442A090839
:103E2000EC250020801A060090F81835934207D937
:103E300002F59E7250F8220010B103689B6A184781
:103E4000002070472DE9F34105466E4686E80C00D8
:103E5000134B45F8043B04460F4600F5C878284646
:103E60002C3500F07DFCA845F9D196E8030004F25A
:103E70001C53C4F8147583E80300089BC4F8243568
:103E8000084920462EF08AFA074B1A6812B10748F3
:103E900053F088F820461C6002B0BDE8F08100BFF6
:103EA000382E0908002D0908685A0020442C0908FA
:103EB0002DE9F041A2B00C4607A92DF0A9FB00287E
:103EC00055D000210D220CA80591ADF818100B91CA
:103ED00076F022FA2B4B611C1F68C9B20BAD012989
:103EE000F86A0A9546D1284B062205A90EF08EFEE7
:103EF000264B019305AB0093002411222946244B45
:103F0000F86A8DF819400EF081FE04AA0DF10F0138
:103F100028468DF83C4004942EF0B4FE38B31D4979
:103F2000DFF86C80482210A876F0ACF9062610ACB9
:103F30002268531E049AC2F3513202EB8312237992
:103F40008DF82430A368019305AB00930892434693
:103F500011222946F86A0EF059FE0021B7EE000A38
:103F600007A82DF005FD013E04F10C04E0D122B0BC
:103F7000BDE8F0810091084B062205A90EF046FE2F
:103F8000B6E700BFEC250020D51B0908752C0908F1
:103F90006F2C090858E50808682C09082DE9F04F2E
:103FA00090F8186585B00446002E48D17F2380F82C
:103FB00028350DF10F01042328308DF80F302EF035
:103FC000BFFF04F5C87504F59E68271D5FFA86F9E2
:103FD0001822FF21284676F09FF985F8579097F927
:103FE00024A0BAF1090F4AD02CDCAAF10303DBB2FA
:103FF000012B37D9D8F8000050B1E96DC5F858A0A9
:1040000031B1254B43F826102EF0D6FB2EF0CCFB19
:1040100058F8040B09F1010A5FFA8AFA40B1036803
:104020009B68984784F818A549462046FFF740FF4B
:104030000136092E05F1600507F12C07C6D105B040
:10404000BDE8F08FBAF10A0FD4D1302001F0BAFDEB
:10405000834688B1CDF800903B462A46214655F06C
:104060000DFB09E0442001F0ADFD834620B13B4645
:104070002A46214654F008FDC8F800B0BAE73820B7
:1040800001F0A0FD83460028F6D03B462A46214693
:1040900055F052F9F0E700BF6C5A002090F818353F
:1040A0008B4283BF602303FB010090F8D501002001
:1040B0007047000090F818358B4283BF602303FBE4
:1040C000010090ED6A0A9FED010A704700000000B0
:1040D00090F818358B4206D901F59E7150F82100F1
:1040E00008B154F065BE9FED010A70470000000062
:1040F00010B490F818458C420A4614D901F59E7404
:1041000050F824407CB1E468246A640603D55DF865
:10411000044BFFF7DDBF602101FB020393ED6A0A48
:104120005DF8044B70479FED010AF9E700000000BD
:1041300090F818358B420BD901F59E7150F821008B
:1041400038B1C3681B6A1A4214BF012000207047AF
:104150000020704770B590F81835934204460E461B
:10416000154601D8002070BD02F59E7350F823005B
:104170000028F7D003689B6998470028F2D0602296
:1041800002FB0544D4F8AC313360ECE770B590F82D
:104190001835934204460E46154601D8002070BDDE
:1041A00002F59E7350F823000028F7D003689B693E
:1041B00098470028F2D0602202FB0544D4ED6C7AC7
:1041C000F4EE677AF1EE10FAE8D6C6ED007AE6E78B
:1041D00070B590F81835934204460E46154601D83E
:1041E000002070BD02F59E7350F823000028F7D020
:1041F00003685B6998470028F2D0602202FB0544FF
:10420000D4F8B4313360ECE790F8183593420ED906
:1042100002F59E7350F823305BB1602303FB02026A
:1042200092F8E40130B1D2F8E0310B607047002021
:10423000704718467047000008299DBF2C2303FBD8
:1042400001004068002070472DE9F04F4B4B2DEDE9
:10425000028B1B68DB6A93F89C3089B00446002B04
:1042600000F08680DFF82CB19FED458A4FF0000901
:1042700094F818355FFA89F5AB4279D905F59E7344
:1042800054F8230000285DD003685B6B98476023D7
:1042900003FB0543074693F8D431834252D20328E7
:1042A00061D8DFE800F04F025259364E4FF0000857
:1042B0003CF000F994F81825AA4284BF602202FB62
:1042C00005424FF0600105F1010301FB05458CBF7C
:1042D000D2F8A82118EE102A8246D5F8B001CDE90F
:1042E0000632F8F711F9079ACDE904011046F8F7FC
:1042F0000BF9069B0096CDE902015A46042150466F
:1043000035F004FB0123204A84F8293585F8D4715F
:10431000D372D4F824354BB3002255B25957481CF8
:1043200003D0414502F10102F7D194F92835AB429F
:1043300008DBD4F82035D4F81C05424631469847AE
:1043400084F8285509F1010992E72C2303FB054362
:104350000E4E93F92B80ABE72C2303FB05430C4E49
:1043600093F92C80A4E70026B046A1E71D46DCE7C0
:1043700009B0BDEC028BBDE8F08F00BFEC2500203A
:1043800000000000892C0908ED5A00201E360A089A
:10439000802C0908982C090890F818358B4207D909
:1043A00001F59E7150F8210010B10368DB691847D0
:1043B0000020704708299CBF602303FB010000F523
:1043C000C870704790F81835934207D902F59E726D
:1043D00050F8220010B103685B6A1847002070474C
:1043E0002DE9F04F002493B005460E4617462146AE
:1043F0002F2206A8059405F59E6975F08DFF05F13D
:10440000280A4FF02C0B05F5F4730BFB04F259F856
:10441000040B1AF90210E5B230B951B90134092C74
:10442000F3D14FF0010813E0602262439A589142A1
:1044300012D01548154B006801930135EDB2009577
:10444000134BC06A324639460EF0E0FB4FF00008CD
:10445000404613B0BDE8F08F05A93322039354F012
:1044600089FD039B804605A90028D7D10648019104
:104470000135EDB200680095054BC06A32463946F9
:104480000EF0C4FBE4E700BFEC250020CE2C0908A9
:10449000C02C09082DE9F04FDFF88090DFF880A0EC
:1044A000DFF880B08DB00646002796F81835FCB2CC
:1044B000A3422ED9602505FB046595F8DC3133B3A2
:1044C00095F8DD1119BB4FF001082022444404A8DF
:1044D00089F8198075F020FF07EE904A4AF21043E0
:1044E000F8EEE77A03AA4C21ADF828305046242391
:1044F000CDED037A37F00AF93BF0DCFF9BF8003092
:10450000054A0094042135F001FA85F8DD81013770
:10451000CBE70DB0BDE8F08FD82C0908ED5A00208C
:104520009D5D0020282300202DE9F04F2F4B1E68B1
:1045300085B0044646B1D0F81415304632F0E0F8A4
:1045400010B1304631F0A0F852F05EFD4FF0000897
:1045500001904FF02C0A4FF0600B94F818355FFA79
:1045600088F5AB4239D904EB8507D7F8F00488B356
:104570000AFB05430BFB054993F92820D9F8E811FC
:104580008A4227D132B30268D2689047D7F8F00444
:104590000268126B904799F8D52112B1019BC9F8B6
:1045A000D831BEB1D4F81415304632F0A9F888B12C
:1045B00052F032FDCDE9021002460B46D7F8F00466
:1045C000294654F0CDFEDDE90232D7F8F004294641
:1045D00054F044FF08F10108BFE72046FFF734FE1E
:1045E000204605B0BDE8F04FFFF754BF105D002036
:1045F0002DE9F0474FF000082DED028B0446894667
:10460000B0EE408A474601264FF0600A94F818350C
:104610005FFA88F5AB421AD929FA05F3DB070AD508
:1046200005F59E7354F8230078B10368B0EE480A8C
:104630009B6B984706400AFB054508F1010895F871
:10464000D4319F4238BF1F46E0E70646F3E727B95B
:104650007F23A4F82835034BDF72BDEC028B304674
:10466000BDE8F087ED5A002090F818358B4207D945
:1046700001F59E7150F8210010B10368DB6B1847FB
:10468000002070470B46114690F818259A4207D92A
:1046900003F59E7350F8230010B103681B6C184794
:1046A0007047000070B504460E46002594F8183592
:1046B000E9B28B4205D932462046FFF7E3FF0135C8
:1046C000F4E770BD2DE9F84390F818550246002430
:1046D00000F128062C2700F5F4784FF06009E1B2CC
:1046E0008D420FD907FB04F309FB04F0F35658F889
:1046F0000000834209D11BB11046FFF7CFFC10B177
:104700000134ECE70120BDE8F8830020FBE700005E
:1047100010B590F818258A42044617D9602202FB8A
:10472000010393F8D431022B03D004D9032B18BF13
:104730000023184610BDFFF797FF48B92046FFF742
:10474000C1FF00280CBF06230123F2E70023F0E796
:104750000623EEE7014B1868704700BF685A002037
:1047600010B5034904462DF019FE204610BD00BFC8
:10477000B02E090810B50446203044F0EFFE044B7B
:1047800004491C6020462DF009FE204610BD00BFE4
:10479000905A0020343009082DE9F3410022B7EE89
:1047A000000A022105462DF0FBF9284654F0B0FF1F
:1047B00044F0B8FF234B1E680446F06A03685B6A46
:1047C00098470B46022102460091204644F0DCFE49
:1047D000B5F94A70002F13DDD6F82C80D8F80030D8
:1047E00040465B68BCB2984728B198F84D3013B189
:1047F000C92FA8BFC824B06A036821465B689847E0
:1048000095F949002022002111F0D4FBC4B245F0F3
:10481000D9FD45F03DFD70B9B06A036801345B68AD
:10482000E4B205219847072CF1D9074802B0BDE84A
:10483000F04151F01DBD072CF7D885F8494002B072
:10484000BDE8F081EC250020A02F090810B5044632
:1048500054F02CFF2046BDE8104054F057BF000034
:104860002DE98048284BDFF8A490DFF8A4A0DFF8FA
:10487000A4B01446012293B005460E461A704FF0BC
:10488000000852F0C1FBD9F800300393A0EB0802F6
:1048900041F287339A4207461FD9CDE90056039863
:1048A0005346342205A9C06A0EF0B0F9214605A886
:1048B000049451F0CDFCCDE9005603985B463422B8
:1048C00005A9C06A0EF0A2F904943BF0F3FD049B25
:1048D00005AA022135F000F8B8463BF0EBFD3AF0AE
:1048E000E7FE3BF0E7FD3CF0EFFC0A2105A80DF0E8
:1048F00093FF039B986A036805215B68984705A8A6
:104900000DF096FFBDE700BF945A0020EC25002073
:104910003DA209080D460A080FB400B595B016AAC5
:10492000002152F8043B039205A83C220193049114
:1049300075F0F2FC054A019B402104A851F030FCBF
:10494000039A034804A9FFF78BFF00BFB82F09089B
:10495000CE2F09080FB407B504AA034852F8041B68
:104960000192FFF77DFF00BFE02F09080146D0E963
:10497000070300B11847002BFCD17047B0F9023093
:1049800002889A4314BFC3F3C000002070470000A0
:1049900038B507230380022200230525C0E905322C
:1049A000C0E90D33C0E91033C0E92C330C49036270
:1049B000C0F89C5004462DF0F1FC0A4B196811B167
:1049C000094852F0EFFA94F910001C602A4611F0E1
:1049D000F1FA637C207403F010036361204638BD54
:1049E00084310908985A0020C43009080123436122
:1049F0000423C36470470000002343610423C3649D
:104A0000704700000123C364704700000223C364A1
:104A1000704700000323C3647047000010B5C369EA
:104A200093B190F9514090F950309C4207DA074B0E
:104A300007480068C06A0EF0E9F8002010BD036A5C
:104A4000012B01D8034BF3E70120F7E7E030090819
:104A5000EC250020EC300908F8B504463CF0ACFF2A
:104A60003CF096FF3DF054FE07463CF0A5FF3CF0BD
:104A700099FF3DF04DFE06463CF09EFF3CF074FF72
:104A80003DF046FE05463CF097FF3CF077FF3DF0D9
:104A90003FFE0246606C50B101285FD1012E5DD10E
:104AA000012A5BD1012D14BF00200820F8BD012F81
:104AB00028D176B9012A61D1012D63D1627CD70753
:104AC00005D494F9511094F95020914210DA022043
:104AD000ECE7022E16D1012A50D1012D52D1627C71
:104AE000D60741D494F9511094F9502091423BDB00
:104AF0006269216C8A421AD0002A33D0012A08BF89
:104B00000A20D3E7002D3BD0012E0BD1012A09D179
:104B1000022DEDD12046FFF731FF002814BF0420FD
:104B20000320C3E7E2B1022AE2D10620BEE7E26C2D
:104B3000A16B8A42BAD0012A1DD1617C0D0715D420
:104B4000617C490710D4022A12D1617C0B070DD475
:104B5000627C12F0040F18BF0220A7E70020A5E72F
:104B60000520A3E70920A1E701209FE710469DE764
:104B7000042A9BD1ECE7032AE5D1E1E7002DD1D14E
:104B8000072093E7002DB3D1FAE700004B6A022B10
:104B90004FF0000303D080F84830436470478A68C0
:104BA000032A05D0042A05D0002380F84830704736
:104BB0004364F9E70B680A7B5B78012A03F00F0373
:104BC00005D0022AF0D1002BEED00262ECE7002BD8
:104BD000EAD005230362E7E7FFF7D8BF037C033B76
:104BE000022B94BF0120032070470000037C033B8D
:104BF000022B94BF0120042070470000C06910B14F
:104C000003681B6A1847704770B50446C06903689B
:104C100000215B6C9847E069036801219B6C984711
:104C2000E06903680021DB6B9847E5692B6828463B
:104C3000D3E90D63984740F4407081B22846B047ED
:104C40000A23E0691A464FF4E1310DF0ABFEE0694A
:104C50000368BDE870401B6A184700000339042947
:104C60009ABF024B58560020704700BF7C3109089C
:104C7000F7B5C36904466BB3E2B9012915BF002338
:104C8000012303270427CC208DF804008DF805109C
:104C90000BB18DF80620002630467D1EF3B2AB42E4
:104CA00006F1010609DA02AA134413F8041C11F0F4
:104CB0002DFAF3E701230427E5E702AB1D443A464A
:104CC00005F8040CE069036801A9DB689847E0690E
:104CD0000DF0C4FE03B0F0BD10B5C4693CB18469E9
:104CE000012C06D1C262CAB22146FFF7C1FF20469D
:104CF00010BD0020FCE70000042910B5044604DCC8
:104D000002290DDC01290ED010BD0A29FCD1FFF7C4
:104D100065FFE26801462046FFF7DEFF032306E059
:104D2000437C9B07F0D5FF23A4F852300423236271
:104D3000EAE7000010B590F8513080F85030044692
:104D400044F042FE20B100F58050002380F8843406
:104D50006369012B0DD163885B060AD52046FFF7F6
:104D60003DFFE26801462046FFF7B6FF03232362BA
:104D700010BD0223FBE70000013938B504460629BF
:104D800069D8DFE801F0042031688B8BB60090F918
:104D90005030002B5FDC013380F85030C2680221B4
:104DA000FFF79AFF94F95030002B0ADD44F00CFE17
:104DB00020B100F58050012380F88434052323625C
:104DC00049E00423FBE790F95030002B08DD013B5C
:104DD000C26880F850300221FFF77EFF0623EEE71D
:104DE000BDE83840FFF7A6BF90F9503090F9521057
:104DF000012B20DD90F91000484D421EC2EBC2028B
:104E0000AB18AA5C2AB353FA81F394F853205B7869
:104E1000013B9A421DD105281BD0A26800212046E3
:104E2000FFF75AFF002384F8533094F85030013BC9
:104E300084F850300FE00CD190F910203748531E01
:104E4000C3EBC303C35C23B1013B994201D1052AE3
:104E500002D100290BDA38BDE26800212046FFF7B5
:104E60003BFF94F85030013B84F85030B6E794F99A
:104E700010302A4A013BC3EBC30313440B445B7855
:104E8000002BE8D0A26800212046FFF725FF94F907
:104E900050300133022BA8BF0223C9E701218268E9
:104EA000FFF71AFF94F950301C49012B94F9103088
:104EB00011DD013B94F8520094F85320C3EBC30377
:104EC0000B44034401325B78B2FBF3F103FB112284
:104ED00084F85320BFE7013BC3EBC30394F952208E
:104EE000CB5C013292FBF3F103FB112284F85220D8
:104EF000B1E790F95030002B09DD013B80F85030CC
:104F00000023C26880F853300221FFF7E5FE94F9D0
:104F10005030002B9FD194F85130A5E70D2200208E
:104F200010B54369012B044610D143885B060ED5AA
:104F3000437CD90607D4FFF751FEE26801465200D0
:104F40002046FFF7C9FE0323236210BD0BB10223E5
:104F5000FAE743885A06FAD5437CDB06F7D5FFF714
:104F600045FEE268014652002046FFF7B5FEEEE737
:104F7000042910B5044604DC02290DDC01290ED0F9
:104F800010BD0929FCD1FFF731FEE2680146204639
:104F9000FFF7A2FE02230EE0437C9B07F0D52046DC
:104FA000FFF724FEE26801462046FFF795FEFF2347
:104FB000A4F8523004232362E2E7000010B504464F
:104FC00052F022F8A36AE26AC31A934207D3226A14
:104FD000A0620023022AE36202D0032A10D010BD8F
:104FE0006269012A0AD1638813F0400F0CBF0021C7
:104FF0000A212046BDE81040FFF77EBE1946F8E7BB
:10500000616949B9638813F0400F18BF0921204630
:10501000BDE81040FFF7ACBF1946F8E773B50B6861
:105020005B78836143885B045EBF0B685B88438069
:10503000B0F90230002B04461ADD012303623BF075
:1050400039FA05462046B4F90260FFF797FC68B9C3
:105050002388B3430CBF022300230093094A33463D
:105060000621284634F052FC02B070BD0523F4E757
:105070003BF020FA044A042102B0BDE8704034F04D
:1050800045BC00BF0031090831310908FFF7C6BF30
:1050900070B50446D0F8B8000E46E8B1D4F8A83090
:1050A00023B1D4F8A420CB1A934221D3B4F8AC5046
:1050B0009DB12046FFF7A8FDD4E9260194F8A02071
:1050C000FFF7D6FDB4F8AC30C4F8A8600020013B6F
:1050D00084F8A100A4F8AC3070BD042304F194005E
:1050E000C4F8B830FFF742FCC4F8B8502846F3E7DC
:1050F0000120F1E738B50024054620466B7BA3422A
:1051000005DD2B68195D11F001F80134F6E738BDB3
:105110002DE9F041C3690446002B43D051F074FFE0
:1051200001462046FFF7B4FF00283BD0E069036842
:105130005B699847402828BF40200025064604F1B7
:105140009407A846AE422DD051F05EFF014620469E
:10515000FFF79EFF30B3E06903689B69984794F8B6
:10516000A130C0B20BB9CC281AD1D4F89420D054B5
:1051700094F8A13094F8A2200133DBB29A4284F86B
:10518000A1300DD13846FFF7B5FF00280CBF022330
:105190000323C4F8B8303846FFF7E8FBC4F8B880FA
:1051A0000135CFE7BDE8F081074A002352F833000C
:1051B000884203D102EBC303187970470133042BF3
:1051C000F4D10020704700BF3022002038B50373AF
:1051D00000234373049B03611546BDF814308560BA
:1051E00001F154020446C0E90021038300F11C03CD
:1051F000DDE9060183E803000123636251F004FF47
:10520000294660612046FFF7CFFFA073204638BDD6
:105210002DE9F0438FB016AC064634F8049B0F46D8
:1052200090461D46FFF7EAFC94E8030002AB83E8D2
:1052300003003A46CDE900594346314604A804AC80
:10524000FFF7C4FF0FCC06F194050FC50FCC0FC5B7
:1052500094E80300424685E80300394630460FB023
:10526000BDE8F043FFF704BD10B586B0094B0593C8
:10527000049006AA12E9030001AB83E803000022B0
:105280004FF6FF73009311464FF47A63FFF7C0FFA8
:1052900006B010BD8D50010813B51A4B04461868AE
:1052A00020B100221A212EF049FEE061E36953B1DA
:1052B00001230DF1070104F110008DF807302DF0E6
:1052C0003FFE2DF071FA94F9103013B9E36102B08A
:1052D00010BDE269002AFAD0022B01D0052B03D1C0
:1052E0004FF6FF73A4F850302046FFF78DFC51F0C5
:1052F0008BFE6368A0622046E36202B0BDE8104006
:10530000FFF7B2BFBC5B002030B587B004AB83E8C9
:105310000600054693E8030001AC022384E805007B
:105320000421009301224FF4C8732846FFF770FF51
:1053300007B030BD30B587B004AB83E80600054642
:1053400093E8030001AC84E80500022200924FF4C8
:10535000C87304212846FFF75BFF07B030BD00008B
:1053600010B586B006AC04E90C0061B101244464B8
:1053700001AC84E80C000224CAB200944FF4C87354
:105380002146FFF745FF06B010BD000070B586B09E
:1053900004AB83E8060002254564044693E8030055
:1053A00001AE86E805004FF4C87300950022032182
:1053B0002046FFF72DFF06B070BD000010B5012399
:1053C00080F848304B1E88B00446C262072B31D8A3
:1053D000DFE803F0040E181818181825164B009073
:1053E0001A460146019308B0BDE81040FFF78CBF94
:1053F000114B02901A460146039308B0BDE81040D5
:10540000FFF798BFFFF72AFC0B4B04940146224696
:105410002046059308B0BDE81040FFF7A1BF064B3A
:105420000793069008AB13E9060008B0BDE81040EA
:10543000FFF7ACBF08B010BDD94B01084B1E10B52B
:105440000446092B20D8DFE803F00C233636363625
:1054500036053636642208212046BDE81040FFF7A5
:10546000ADBF90F9503083B944F0AEFA20B100F5E9
:105470008050012380F88434642201212046FFF704
:105480009DFF012384F8503010BD64220321E3E71F
:1054900090F95030002BF7DD44F096FA20B100F57A
:1054A0008050002380F88434642202212046FFF7D4
:1054B00085FF0023E6E76422CEE7000013B504462B
:1054C0000191FFF75BFA019928B1204602B0BDE8CF
:1054D0001040FFF7B3BF2388B4F90220934305D1EE
:1054E000204602B0BDE81040FFF746BC02B010BD38
:1054F00070B5044651F088FD94F8482022B9A36A9B
:10550000E16AC31A8B4202D20023236370BDC4E94F
:105510000A022046FFF7A0FA236B62698342014624
:10552000236AE06C0ED1656BAB420BD1A56B854253
:1055300008D194F93C6094F95050AE4202D1256CE8
:105540009542E3D0C4E90C13A063013B94F85000EA
:1055500084F83C002264052BD8D8DFE803F0030868
:105560000D1213182046BDE87040FFF7D9BC204645
:10557000BDE87040FFF7C0BB2046BDE87040FFF7B4
:10558000F7BC01212046BDE87040FFF797BF02211C
:10559000F8E7000010B50D4B1B68DB6A93F89C30F0
:1055A000044623B12046BDE81040FFF707BD44F094
:1055B0000BFA28B100F5805393F86434032BF1D82B
:1055C0002046BDE81040FFF793BF00BFEC25002048
:1055D00038B5C36904467BB190F9103063B1FFF769
:1055E00097FD51F011FD636AC31A642B054603D978
:1055F0002046FFF7CFFF656238BD0000014B1868F9
:10560000704700BF985A002008B50449102274F072
:1056100029FEB0FA80F0400908BD00BF9C5A002066
:105620001022002174F078BE10B50446FFF7F8FF91
:10563000204610BD0378416023F00D03022A037059
:1056400008D0032A0AD0012A03D1DBB243F00103B8
:1056500003707047037843F00803F9E7037823F0F9
:10566000050343F00503F3E773B504460E461546FC
:105670000193FFF7D5FF2046C4E90265069A019918
:10568000FFF7D8FF02B070BD0078420704D40307CB
:1056900004D400F0010070470320704702207047D7
:1056A000F0B587B004461546FFF7EEFF88420F4677
:1056B000064605D163682B600126304607B0F0BD71
:1056C00000230328019301D0032913D12EF0EAFF10
:1056D00008B90026F1E7012301AA21462EF01EFE9B
:1056E0000028F6D0DDED017A9FED337A67EE877AF8
:1056F000CDED017A032E32D8DFE806F00209162438
:105700006468032FE5D8DFE807F02C2E3C49FBF74F
:105710000FFF90F87C32DB07DBD56468FBF708FFEE
:10572000D0F870321C44ECE702A8FFF779FFFBF7D2
:10573000FFFE02A9FBF702FD06460028BDD0646803
:10574000039BEFE7D4ED017A9DED017AF8EEE77A5D
:1057500077EE877AFDEEE77A17EE904AD1E70024DC
:10576000CFE72C60A8E7FBF7E3FE90F87C6216F029
:105770000106AED0FBF7DCFED0F87032E41A2C60E4
:105780009BE702A8FFF74CFFFBF7D2FE02A9FBF74D
:10579000D5FC0646002890D0039BEFE707EE904A21
:1057A0009DED017AF8EEE77A77EEC77AFDEEE77ABB
:1057B000C5ED007A80E700BF0000C84273B501AABA
:1057C00005460E46FFF76CFF044620B101993246AC
:1057D0002846FFF72FFF204602B070BD13B51446D0
:1057E00001AAFFF75DFF48B1DDED017A9FED047A74
:1057F000F8EEE77A67EE877AC4ED007A02B010BD62
:105800000AD7233C07EE900A9FED090AF8EEE77AE3
:1058100008B527EE800A72F077F9DFED067AB4EE6C
:10582000E70AF1EE10FAD8BFB0EE670A08BD00BF74
:1058300050E0EF300AD7233C10B50446806810F0E2
:105840000DFD20B1E068BDE8104010F01BBD10BD9B
:105850000D4B83424FF000038B4106DA00F12550D7
:1058600000F5311000F5E0507047084B98424FF0BA
:10587000FF3371EB0303BEBF00F1564000F5130088
:1058800000F52440704700BF00D2496B002EB6944B
:1058900090EA010F01D4401A7047C317401A63EB16
:1058A000E1710D4B83424FF000038B4106DA00F1AA
:1058B000255000F5311000F5E0507047074B984235
:1058C0004FF0FF3371EB0303BEBF00F1564000F50C
:1058D000130000F52440704700D2496B002EB694A7
:1058E00070B52DED028B84B0044668460D46FFF777
:1058F00097FEFBF71DFE6946FBF720FC064608B342
:10590000A368029ADFED128A03999B1A07EE903A78
:10591000F8EEE77A67EEA87AC5ED007AE068FFF75F
:10592000B7FF08EE100AA068024402EBD272B8EE8C
:10593000C88A5010FFF766FF28EE288A28EE000A72
:1059400085ED010A304604B0BDEC028B70BD00BF8E
:10595000F67C8E3F37B500230C4601AA022105468E
:105960000193FFF79DFE10B9002003B030BD214622
:105970002846FFF7B5FF0028F6D0DDED017AF8EEF6
:10598000E77AC4ED027AF0E738B52DED028B0C46CC
:105990000246C168E068FFF77BFF9568A46808EEDF
:1059A000100A601900EBD0704010641BFFF72AFF4B
:1059B00007EE904AF8EEE77AF8EEC80A87EE807AAA
:1059C000BDEEC70A10EE103A5B4200EE103AB8EE98
:1059D000C00A72F0BBFADFED087A30EE270ABDECA0
:1059E000028BB5EEC00AF1EE10FA44BFDFED037A88
:1059F00030EE270A38BD00BFDB0FC93FDB0FC940BF
:105A000030B52DED028B0B4685B08C68D0E9025184
:105A1000D868FFF73DFF08EE100A601900EBD07060
:105A20004010FFF7EFFE641B07EE904AF0EE400ACD
:105A3000B8EEC88A9FED060AF8EEE77A28EE008AEB
:105A400027EE800A68EE200A05B0BDEC028B30BD5F
:105A50008262363C82B002B0FFF7D2BFF0B52DEDC6
:105A6000028B0D4689B08C680646D0E90271E86861
:105A7000FFF70EFF08EE100AE01900EBD07040109F
:105A8000FFF7C0FE73686A689FED0E1A9B1A07EE57
:105A9000903AE41BB8EEE77AF0EE400A07EE904A3F
:105AA0009FED090AB8EEC88AF8EEE77A28EE008A78
:105AB00027EE011A27EE800A68EE200A09B0BDEC35
:105AC000028BF0BD0AD7233C8262363C10B52DED27
:105AD000028B84688A680B46111B08EE901AC16815
:105AE000D868FFF7D5FE224402EBD27208EE100A06
:105AF0005010FFF787FEB8EEC88AF8EEE88A28EE65
:105B0000000A20EE000AA8EEA80A72F069FBBDECBC
:105B1000028BDFED027A20EE270A10BD8262363C4E
:105B2000094B984206DDC0F1D64000F5930000F520
:105B3000A4407047054B9842BEBFC0F1144000F529
:105B4000360000F53850704700E9A43500175BCAED
:105B5000F8B52DED028BDFED148A076820EE280AD8
:105B60000646FDEEC07A0D4617EE904A04EBD4705F
:105B700007EB6000B0EE608AFFF744FE28EE288A4B
:105B80003819C8EE007AFFF7CBFF306017EE900AA5
:105B9000F7F7E4F92B68C01841EBE371FFF758FE03
:105BA000BDEC028B2860F8BD02AAB34200F10C01E3
:105BB0000830FFF7CDBF00000148FFF731BD00BF3F
:105BC0009C5A00200121884238BF084670F006B96F
:105BD000FFF7F8BF08B170F005B97047FFF7FABFDB
:105BE00000214FF0FF3310B500220363044601602B
:105BF0000171C0F80510417280F8251000F13C03D6
:105C000000F50B70D9709A60DA601A615A619A6176
:105C1000DA611A625A629A62DA631A645A649A649E
:105C2000DA641A655A659A65DA65DA661A675A6738
:105C30007C339842E6D1214604F5167007F0AAFAA3
:105C4000044B1A6822B904491C6020462CF0A6FBBC
:105C5000204610BDAC5A0020BC33090873B5D0F8FB
:105C60003C3201919942044613D0D0F84032994217
:105C700018D0D0F844328B4216D102200AE0D4F872
:105C8000343253B3D4F838324BB34FF0030002B080
:105C900070BD002094F822308342F8D8431C84F869
:105CA0002230F4E70120F5E7D0F83062002EE6D18B
:105CB00094F841233546B6009AB1A319C3F83012BF
:105CC000A319019AC3F83C2294F82230AB429CBF3E
:105CD0006B1C84F822302846D9E70126E8E7022623
:105CE000E6E704F50C7001A930442DF0FBF9E7E775
:105CF00038B504460D462DF06BF9291D201D2DF0F9
:105D000067F905F1080104F108002DF03BFA05F1EF
:105D1000140104F114002DF035FA05F1200104F10D
:105D200020002DF02FFA05F12C0104F12C002DF0AC
:105D3000E3F805F1300104F130002DF0EBF905F145
:105D40003C0104F13C002DF01DFAAB6BA3636B6BBF
:105D5000636338BD2DE9F043A1B00023002500F1B5
:105D60003C0706468DF8075003930493059306936A
:105D70000793089309930A930B931093119312932B
:105D80001393149315931693179318931C931D93C1
:105D90001E9300F50F78B94658F8043BF3B1F26E44
:105DA000934223D0D6F8E820934221D0D6F864213C
:105DB000934213D10221EBB299420FD0C1EB4111B2
:105DC00009EB8104214601A8FFF792FF39462046DE
:105DD000FFF78EFF01A93846FFF78AFF0135032D33
:105DE00007F17C07D8D121B0BDE8F0830021E2E7BC
:105DF0000121E0E72DE9F04706460F4615468046AB
:105E000004464FF0000A39463046FFF727FF626F1D
:105E1000BA425FFA8AF90ED1C3B2022B0BD87C22A8
:105E200002FB0A66012086F83E0086F83F3085F8BE
:105E30000090BDE8F0870AF1010ABAF1030F04F1FE
:105E40007C04E0D1002439463046FFF707FFD8F83C
:105E50006C205FFA84F912B9C3B2022B22D9013443
:105E6000032C08F17C08EED100244FF07C0906F1E8
:105E70003E0A39463046FFF7F1FE034609FB04F0BF
:105E80005FFA84F81AF8002012B9DBB2022B12D99B
:105E90000134032CEDD196F82300042814D91948B5
:105EA00051F080F87C2000FB0464012084F83E005F
:105EB00084F83F30BBE70644012086F83E0086F8B0
:105EC0003F3085F80080B4E706F54371002251F8B1
:105ED000043BBB42D4B208D1A04202D8631C86F86E
:105EE000233003342C700020A3E73BB9421C06EB9F
:105EF000800086F82320C0F80C73F2E70132052AEF
:105F0000E5D1F0E7F4310908C9B200EB8101D1F81D
:105F10003C3253B1026F93420AD0D0F8EC20934246
:105F200008D0D0F86821934206D04FF003007047A4
:105F300000207047012070470220704759B190F847
:105F40002030032B07D05A1C80F8202000EB830060
:105F50004161012070470020704700002DE9F8439F
:105F60000F469146044600F5BA7894F83E5035B98C
:105F70007C344445F9D100252846BDE8F883002348
:105F80004A46394601200CF0D5FA00210646E06E5B
:105F90000CF0E0FA8642EBD1EEE700002DE9F04389
:105FA000DFF87C8085B0044600F50F7600257C275D
:105FB000B14656F80C3CD9F800209342E9B206F1FC
:105FC000040619D1C3B12046FFF79EFFC0B207FBFC
:105FD000004090F83E307BB903A9A9F10C0003936F
:105FE0002DF080F83AF066FA56F8043C00934246E9
:105FF0002B46012133F08AFC0135032DD8D104F161
:106000006C0504F5F074296821B9AB6813B1284612
:106010002BF01AFB7C35A542F5D105B0BDE8F08325
:106020001032090838B504461546FFF76DFFC0B2B7
:10603000022808D87C2303FB004029465030BDE8E5
:1060400038402DF08FB838BD38B504461546FFF7F7
:106050005BFFC0B2022808D87C2303FB004029461E
:106060005C30BDE838402DF07DB838BD37B50D4601
:1060700004468DED010AFFF747FF022D07D8C0B295
:106080007C2303FB004001A968302CF01DFF03B006
:1060900030BD000038B50546FFF736FFC4B2022C0C
:1060A00013D8C4EB4414A4003C3504F10800284480
:1060B00000212BF0C9FA04F1340104F13000294425
:1060C0002844BDE838402DF00DB838BD70B5054600
:1060D0000E461446FFF718FFC3B2022B0DD87C20E2
:1060E00000FB035394E80700443383E8070031467C
:1060F0002846BDE87040FFF7CDBF70BD37B50446F8
:106100001546FFF701FFC0B2022809D87C2303FB24
:1061100000400DF1070140308DF807502CF058FF7A
:1061200003B030BD10B500210446FFF7B3FF204691
:106130000121FFF7AFFF20460221BDE81040FFF725
:10614000A9BF00001FB590F92C30044623B390F985
:1061500021300BB36846FFF767FAFBF7E9F96946A8
:10616000FAF7C8FFC0B1DDED037A9FED0C0AF8EE37
:10617000E70ADDED027AF8EEE77A0123C0EE800A45
:1061800084F83D3387EE800A07F046FADFED047AA3
:1061900020EE270A84ED0A0A04B010BD8096184B41
:1061A00035FA8E3C024690F9210058B192F840032E
:1061B00040B1114491F92C0220B192F92400033826
:1061C00018BF01207047000038B590F8223005460E
:1061D0005BB100242346E1B22846FFF7E3FF08B194
:1061E0000133DBB20134032CF5D1184638BD000071
:1061F00090ED0A0A7047000038B50C46D1ED066AEA
:1062000011460546FFF780FEC3B27C2000FB035316
:10621000D4ED087AD3ED260A94ED076AD3ED255A1A
:1062200093ED245A26EE600A67EEA00AA5EEA70AAF
:10623000F0EE607AE5EE867AB7EE007AA6EEE67AC0
:1062400067EEE60AB1EE400AE5EE070A71F07EFE5F
:106250009FED071ADFED070A40F61C000FF06CFEF9
:10626000D5ED0A7ABDE8384030EE270A0FF050BE6F
:10627000DB0F4940DB0F49C02DE9F04190F8223097
:106280008B4204460D4602D20020BDE8F081FFF7A4
:106290003BFEC0B204F13C06C0EB401006EB8000B0
:1062A000083012F055FADFED157AB0EEC00AB4EE00
:1062B000E70AF1EE10FAE7D429462046FFF724FE5C
:1062C000C5B27C2000FB05473B6F002BDCD0032DC3
:1062D000DAD000FB05603030D7F86C802CF034F950
:1062E000D7E91B32934201D1984505D07C2000FBB1
:1062F0000544C4F86C80C7E70120C6E700000034FD
:106300002DE9F74F04460E46174600F50F7A4FF079
:10631000000B5AF8049B5FFA8BF8B9F1000F26D0F6
:1063200041462046FFF73EFF08B341462046FFF7AF
:10633000EBFD7C23C0B203FB004090F83E505DB9FA
:1063400008F101031B4ADBB2394630464FF028FF03
:10635000284603B0BDE8F08F5AF8102C914506D0BE
:10636000154A394630464FF01BFF0025F0E70BF188
:10637000010BBBF1030FCCD14FF0000894F8223091
:106380005FFA88F18B420DD920460191FFF774FF27
:10639000054620B901992046FFF704FF20B908F10E
:1063A0000108EBE70125D3E7044A394630464FF0B0
:1063B000F7FECDE7383209084D3209087232090874
:1063C0002DE9F0412DED048B90F842139FED348AB6
:1063D000DFED348A9FED349A82B00646FFF794FDD4
:1063E00006F13C07C5B27C2000FB057554354FF023
:1063F000000896F822205FFA88F39A424ED919468F
:106400003046FFF7CFFE10B908F10108F1E7194651
:106410003046FFF779FDC4B27C2000FB0474D4ED54
:10642000157AF0EEE77AF4EEC87AF1EE10FA04F19C
:1064300054040ED5D4ED017AF0EEE77AF4EEC87A82
:10644000F1EE10FA05D5002002B0BDEC048BBDE8DA
:10645000F0812946204612F093F9B4EEE80AF1EEF5
:1064600010FAF0DC2946204611F0B2FCB4EEC90A5D
:10647000F1EE10FAE7DC2146284611F0F5FB6846FC
:106480008DED000ACDED010A11F08EFCDFED077AEB
:10649000B4EEE70AF1EE10FAB6DDD4E70120D3E757
:1064A00000000034DB0FC93F920A863F00004843DA
:1064B000022910B5044608D8FFF726FD7C23C0B298
:1064C00003FB004494F83D0010BD0020FCE70000F1
:1064D00013B590F8421301910446FFF7E9FF30B17C
:1064E0000199204602B0BDE81040FFF75BBE02B044
:1064F00010BD0000F7B590F921500446002D73D06F
:1065000090F84053002D6FD090F84213FFF7D0FF62
:1065100094F83D33064613B92046FFF713FE0025D5
:1065200094F82020EBB29A4207D904EB830301359B
:10653000586903689B689847F2E750F065FD0027AB
:10654000224604F5BA7140F2F315D2F89C30C31A12
:10655000AB428CBF0023012382F83D307C32914254
:1065600047EA0307F1D194F92430032B07D194F8BB
:106570003C33002B3BD0D4F83803002849D167B115
:10658000236B013309D030F095FA216B30F0B8F865
:1065900018B130F08FFA2FF08BF994F92C32002BD0
:1065A0003AD194F92D32CBBB94F92E3213B1022398
:1065B00084F8423394F842132046FFF779FF86426D
:1065C000054611D030F076FA4FF6FF7130F098F8AA
:1065D00050B1002D14BF00220422019230F06AFA5B
:1065E000019A032130F01EF8284603B0F0BD0123C4
:1065F00084F83C330420FFF7E5FA054610B1214644
:1066000006F05EFE94F92430C4F83853032BB2D060
:10661000B5E706F063FEB2E70023C9E70123C7E749
:1066200038B590F921300446D3B190F84053BDB14C
:10663000FFF76AFCC0B2022812D87C2303FB004497
:10664000D4ED1A7A9FED087AF4EEC77AF1EE10FADB
:1066500006D4B7EE087AF4EEC77AF1EE10FA00DD50
:106660000025284638BD00BFABAA2A3F70B5D0F838
:10667000085315F4003504460E460DD190F840330A
:106680005BB90A78072A07D8012303FA02F290F8C7
:106690003F33134380F83F3370BD94F82020EBB2B2
:1066A0009A42F9D904EB8303314658690368DB68E1
:1066B00098470135F1E7000038B505466C242B59A1
:1066C0001BB1002128192AF0BFFF7C34B4F5F07FFC
:1066D000F5D138BD014B1868704700BFAC5A002097
:1066E0002DE9F04FAA4BD3F800800446D8F80400F7
:1066F00003688DB09B689847002507464FF0010955
:1067000009FA05F33B4240F082820135202DF7D192
:10671000D8F804000368DB689847002507464FF067
:10672000010909FA05F33B4240F0B3820135202DFF
:10673000F7D1D8F8040003689B68984700250746FE
:106740004FF0010909FA05F33B4240F0E1820135BF
:10675000202DF7D1D8F80400DFF840B203689B6819
:10676000984700250490049A0123AB40134240F05F
:106770000B830135202DF6D1D8F80400DFF81CB2C8
:106780000368DB68984700250490049A0123AB4016
:10679000134240F0C9830135202DF6D1D8F804000A
:1067A0000368DB689847002507464FF0010909FA9E
:1067B00005F33B4240F083840135202DF7D1D8F812
:1067C00004000368DB689847002507464FF001097D
:1067D00009FA05F33B4240F0B1840135202DF7D191
:1067E000D8F8040003689B689847002507464FF0D7
:1067F000010909FA05F33B4240F0DF840135202D01
:10680000F7D1D8F8040003689B689847002507462D
:106810004FF0010909FA05F33B4240F00E850135BE
:10682000202DF7D1D8F8040003689B68984700250D
:1068300007464FF0010909FA05F33B4240F03D8558
:106840000135202DF7D1D8F804000368DB6898479C
:10685000002507464FF0010909FA05F33B4240F0D5
:1068600068850135202DF7D14A4B089308AF0425E0
:10687000D8F8040003689B689847002683460123E4
:10688000B34013EA0B0F40F08F850136202EF6D16E
:10689000D8F804000368DB68984700268346012384
:1068A000B34013EA0B0F40F0C4850136202EF6D119
:1068B000013D15F0FF0507F10107D9D1D8F8040013
:1068C00003689B6898474FF00109074609FA05F3EA
:1068D0003B4240F0F2850135202DF7D1D8F8040075
:1068E0000368DB689847002507464FF0010909FA5D
:1068F00005F33B4240F01D860135202DF7D1D8F835
:10690000040003689B689847002507464FF001097B
:1069100009FA05F33B4240F048860135202DF7D1B6
:10692000D8F804000368DB689847002507464FF055
:10693000010909FA05F33B4240F073860135202D29
:10694000F7D1154B0793D8F8040003689B68984764
:10695000002583460123AB4013EA0B0F42D00027EA
:106960005FFA85F9D4F8083313F4803A32D107ABD3
:106970004946DB5D04931A462046FFF7EFFA049B75
:106980000646002800F08986CDE908AA08E000BF85
:10699000EC2500200C0D0E0F20212223801A06006A
:1069A000099B0B93002201210BA8CDE9092204F0D9
:1069B00003FE01462046FFF7C1FA0BA8FDF79AF93E
:1069C0000AA8FDF797F909A8FDF78AF916B108A8F2
:1069D000FDF786F994F82330052B00F04881013744
:1069E000042FBFD10135202DB4D1D8F8040003689D
:1069F000DB689847002583460123AB4013EA0B0F61
:106A000038D000275FFA85F9D4F8083313F4803AB8
:106A100028D107AB4946DB5D04931A462046FFF7B1
:106A20009DFA049B0646002800F04686CDE908AA98
:106A30000022099B0B9311460BA8CDE9092204F013
:106A4000BBFD01462046FFF779FA0BA8FDF752F986
:106A50000AA8FDF74FF909A8FDF742F916B108A8F1
:106A6000FDF73EF994F82330052B00F00081013743
:106A7000042FC9D10135202DBED1D8F804000368F8
:106A80009B689847002682460123B34013EA0A0F09
:106A900031D010255FFA86F9D4F8083313F0080BCB
:106AA00020D12A4649462046FFF758FA07460028D3
:106AB00000F01186CDE909BB0A9B002201210BA839
:106AC000CDE90A2301F00AFC01462046FFF736FA19
:106AD0000BA8FDF705F90AA8FDF702F917B109A8F7
:106AE000FDF7FEF894F82330052B00F0C080013547
:106AF000EDB2142DD0D10136202EC5D1D8F8040026
:106B000003689B689847002682460123B34013EA36
:106B10000A0F34D014255FFA86F9D4F8083313F439
:106B2000001B24D12A4649462046FFF717FA07469C
:106B3000002800F0E385CDE908BB099B0B930022F8
:106B400001210BA8CDE9092201F0DAFF0146204618
:106B5000FFF7F4F90BA8FDF7CDF80AA8FDF7CAF87E
:106B600009A8FDF7BDF817B108A8FDF7B9F894F822
:106B70002330052B7BD00135EDB2182DCDD1013658
:106B8000202EC2D1D8F804000368DB68984700269D
:106B900082460123B34013EA0A0F34D014255FFA6A
:106BA00086F9D4F8083313F4001B24D12A46494649
:106BB0002046FFF7D3F90746002800F0AF85CDE95E
:106BC00008BB0022099B0B9311460BA8CDE90922B3
:106BD00001F096FF01462046FFF7B0F90BA8FDF73C
:106BE00089F80AA8FDF786F809A8FDF779F817B122
:106BF00008A8FDF775F894F82330052B37D0013538
:106C0000EDB2182DCDD10136202EC2D12FE0D4F80F
:106C1000083313F0010A25D15FFA85FB1E2259467D
:106C20002046FFF79BF9064620B3CDE908AA099A4A
:106C30000B920023082201210BA8CDE9093303F0B0
:106C400089FA01462046FFF779F90BA8FDF752F8BB
:106C50000AA8FDF74FF809A8FDF742F816B108A8F1
:106C6000FDF73EF894F82330052B7FF44EAD0DB0C0
:106C7000BDE8F08FD8F8041004220B68CDE90102BA
:106C8000A84A0092D3F800A05A461E2309A8D0476C
:106C9000CDE7D4F8083313F0010A24D15FFA85FB5D
:106CA0001E2259462046FFF759F9064608B3CDE99A
:106CB00008AA099B0B93062200210BA8CDE9091114
:106CC00003F048FA01462046FFF738F90BA8FDF714
:106CD00011F80AA8FDF70EF809A8FDF701F816B19A
:106CE00008A8FCF7FDFF94F82330052B7FF41EADB8
:106CF000BDE7D8F8041004220B68CDE90102894AE7
:106D00000092D3F800A05A461E2309A8D047D0E726
:106D1000D4F8083313F4805A21D15FFA85FB0D2291
:106D200059462046FFF71AF90646F0B1CDE909AAFF
:106D30000A9B0022CDE90A23012108220BA804F0B6
:106D400077FA01462046FFF7F9F80BA8FCF7C8FFD1
:106D50000AA8FCF7C5FF16B109A8FCF7C1FF94F813
:106D60002330052B7FF4F3AC81E7D8F8041004221C
:106D70000B68CDE901026B4A0092D3F800A05A4695
:106D80000D230AA8D047D3E7D4F8083313F480774B
:106D90003FD15FFA85F90C2249462046FFF7DEF81D
:106DA0000646002800F08480CDE90677079B0A9309
:106DB0004FF0000A692249462046CDF81CA0FFF793
:106DC000CDF80746002800F08180CDE908AA099B8C
:106DD0000B9300221A2309920BA901220AA801F0A1
:106DE00005F801462046FFF7A9F80BA8FCF778FF45
:106DF00009A8FCF775FF17B108A8FCF771FF0AA8EE
:106E0000FCF76EFF07A8FCF76BFF16B106A8FCF7AE
:106E100067FF94F82330052B3FF429AFD4F80833EB
:106E200013F480777FF4A5AC5FFA85F90C2249460C
:106E30002046FFF793F80646002856D0CDE906779E
:106E4000079B0A934FF0000A682249462046CDF876
:106E50001CA0FFF783F80746002854D0CDE908AA04
:106E6000099B0B9300221A2309920BA901220AA85D
:106E700000F0BCFF01462046FFF760F80BA8FCF7C6
:106E80002FFF09A8FCF72CFF17B108A8FCF728FF73
:106E90000AA8FCF725FF07A8FCF722FF16B106A8F1
:106EA000FCF71EFF94F82330052B7FF462ACDEE67E
:106EB000D8F8041004220B68CDF800B0CDE9010227
:106EC0004A461F6807A80C23B8476FE7D8F8041094
:106ED00004220B68CDF800B0CDE901024A46D3F890
:106EE00000A009A86923D04771E7D8F8041004224C
:106EF0000B68CDF800B0CDE901024A461F6807A82B
:106F00000C23B8479CE7D8F8041004220B68CDF88E
:106F100000B0CDE901024A46D3F800A009A86823D1
:106F2000D0479DE7801A0600D4F8083313F4807721
:106F30003DD15FFA85F90C2249462046FFF70EF84D
:106F40000646002800F08180CDE90677079B0A936A
:106F50004FF0000A692249462046CDF81CA0FEF7F2
:106F6000FDFF074600287ED0CDE908AA099B0B93B8
:106F700000221A230BA90AA8099200F037FF014644
:106F80002046FEF7DBFF0BA8FCF7AAFE09A8FCF7DA
:106F9000A7FE17B108A8FCF7A3FE0AA8FCF7A0FEFD
:106FA00007A8FCF79DFE16B106A8FCF799FE94F819
:106FB0002330052B3FF45BAED4F8083313F480770D
:106FC0007FF4E9AB5FFA85F90C2249462046FEF7CB
:106FD000C5FF0646002855D0CDE90677079B0A93E2
:106FE0004FF0000A682249462046CDF81CA0FEF763
:106FF000B5FF0746002853D0CDE908AA099B0B939B
:1070000000221A230BA90AA8099200F0EFFE0146FC
:107010002046FEF793FF0BA8FCF762FE09A8FCF7D9
:107020005FFE17B108A8FCF75BFE0AA8FCF758FE44
:1070300007A8FCF755FE16B106A8FCF751FE94F818
:107040002330052B7FF4A7AB11E6D8F804100422F7
:107050000B68CDF800B0CDE901024A461F6807A8C9
:107060000C23B84772E7D8F8041004220B68CDF857
:1070700000B0CDE901024A46D3F800A009A869236F
:10708000D04773E7D8F8041004220B68CDF800B09D
:10709000CDE901024A461F6807A80C23B8479DE7BF
:1070A000D8F8041004220B68CDF800B0CDE9010235
:1070B0004A46D3F800A009A86823D0479EE7D4F831
:1070C000083313F0200A24D15FFA85FB1C225946AD
:1070D0002046FEF743FF064608B3CDE908AA002282
:1070E000099B0B9311460BA8CDE9092203F030FC54
:1070F00001462046FEF722FF0BA8FCF7FBFD0AA87D
:10710000FCF7F8FD09A8FCF7EBFD16B108A8FCF7A1
:10711000E7FD94F82330052B7FF44EABA7E5D8F8B4
:10712000041004220B68CDE90102B84A0092D3F89A
:1071300000A05A461C2309A8D047D0E7D4F808334A
:1071400013F0200A24D15FFA85FB1E2259462046FF
:10715000FEF704FF064608B3CDE908AA0022099B02
:107160000B9311460BA8CDE9092203F0F1FB014670
:107170002046FEF7E3FE0BA8FCF7BCFD0AA8FCF7CF
:10718000B9FD09A8FCF7ACFD16B108A8FCF7A8FDED
:1071900094F82330052B7FF420AB68E5D8F8041071
:1071A00004220B68CDE90102984A0092D3F800A0AE
:1071B0005A461E2309A8D047D0E7D4F8083313F065
:1071C000200A25D15FFA85FB1C2259462046FEF78E
:1071D000C5FE064610B3CDE908AA099A0B92002312
:1071E000022201210BA8CDE9093303F0B1FB0146CE
:1071F0002046FEF7A3FE0BA8FCF77CFD0AA8FCF7CF
:1072000079FD09A8FCF76CFD16B108A8FCF768FD2C
:1072100094F82330052B7FF4F1AA28E5D8F8041060
:1072200004220B68CDE90102784A0092D3F800A04D
:107230005A461C2309A8D047CFE7D4F8083313F0E7
:10724000200A25D15FFA85FB1E2259462046FEF70B
:1072500085FE064610B3CDE908AA099A0B920023D1
:10726000022201210BA8CDE9093303F071FB01468D
:107270002046FEF763FE0BA8FCF73CFD0AA8FCF7CE
:1072800039FD09A8FCF72CFD16B108A8FCF728FD6C
:1072900094F82330052B7FF4C2AAE8E4D8F8041050
:1072A00004220B68CDE90102584A0092D3F800A0ED
:1072B0005A461E2309A8D047CFE7D4F8083313F065
:1072C000400A21D15FFA85FB0C2259462046FEF781
:1072D00045FE0646F0B1CDE909AA0A9B0022CDE998
:1072E0000A23012106220BA800F046FD0146204694
:1072F000FEF724FE0BA8FCF7F3FC0AA8FCF7F0FC51
:1073000016B109A8FCF7ECFC94F82330052B7FF4A8
:1073100097AAACE4D8F8041004220B68CDE9010266
:107320003A4A0092D3F800A05A460C230AA8D04744
:10733000D3E7D4F8083313F0400A20D15FFA85FB75
:107340000C2259462046FEF709FE0646E8B1CDE973
:1073500009AA00220A9B11460BA8CDE90A2300F0D6
:107360000BFD01462046FEF7E9FD0BA8FCF7B8FC33
:107370000AA8FCF7B5FC16B109A8FCF7B1FC94F813
:107380002330052B7FF46DAA71E4D8F80410042291
:107390000B68CDE901021D4A0092D3F800A05A46BD
:1073A0000C230AA8D047D4E7D4F8083313F0800A96
:1073B00026D13B78F1B21A462046CDE90413FEF7F8
:1073C000CDFDDDE90413814610B3CDE909AA0A9B7E
:1073D0000022CDE90A2301210C220BA803F086F933
:1073E00001462046FEF7AAFD0BA8FCF779FC0AA887
:1073F000FCF776FCB9F1000F02D009A8FCF770FC8D
:1074000094F82330052B7FF440AA30E4801A06005C
:10741000D8F80400B84AD0F800E000924FF0040C0D
:10742000CDE9019C0A46DEF800A001460AA8D04733
:10743000CDE7D4F8083313F0800A26D13B78F1B2B7
:107440001A462046CDE90413FEF788FDDDE9041352
:10745000814608B3CDE909AA0A9B0022CDE90A2397
:1074600000210C220BA803F041F901462046FEF74B
:1074700065FD0BA8FCF734FC0AA8FCF731FCB9F158
:10748000000F02D009A8FCF72BFC94F82330052B41
:107490007FF40BAAFFF7EBBBD8F80400964AD0F8AC
:1074A00000E000924FF0040CCDE9019C0A46DEF8A2
:1074B00000A001460AA8D047CEE7D4F8083313F459
:1074C000004A20D15FFA85FB0C2259462046FEF780
:1074D00045FD0646F0B1CDE909AA0A9B002201212B
:1074E0000BA8CDE90A2302F077FF01462046FEF7FC
:1074F00025FD0BA8FCF7F4FB0AA8FCF7F1FB16B17D
:1075000009A8FCF7EDFB94F82330052B7FF4E3A9E1
:10751000FFF7ADBBD8F8041004220B68CDE90102D7
:10752000754A0092D3F800A05A460C230AA8D04707
:10753000D3E7D4F8083313F4004A20D15FFA85FB6F
:107540000C2259462046FEF709FD0646F0B1CDE96A
:1075500009AA00220A9B11460BA8CDE90A2302F0D2
:107560003BFF01462046FEF7E9FC0BA8FCF7B8FB01
:107570000AA8FCF7B5FB16B109A8FCF7B1FB94F813
:107580002330052B7FF4B8A9FFF771BBD8F804109E
:1075900004220B68CDE90102574A0092D3F800A0FB
:1075A0005A460C230AA8D047D3E7D4F8083313F47B
:1075B000007A20D15FFA85FB302259462046FEF73B
:1075C000CDFC0646F0B1CDE909AA0A9B00220121B3
:1075D0000BA8CDE90A2303F087FC01462046FEF7FD
:1075E000ADFC0BA8FCF77CFB0AA8FCF779FB16B1F5
:1075F00009A8FCF775FB94F82330052B7FF48DA9BF
:10760000FFF735BBD8F8041004220B68CDE901025E
:10761000394A0092D3F800A05A4630230AA8D0472E
:10762000D3E7D4F8083313F4007A20D15FFA85FB4E
:10763000302259462046FEF791FC0646F0B1CDE9CE
:1076400009AA00220A9B11460BA8CDE90A2303F0E0
:107650004BFC01462046FEF771FC0BA8FCF740FBF3
:107660000AA8FCF73DFB16B109A8FCF739FB94F812
:107670002330052B7FF462A9FFF7F9BAD8F804107C
:1076800004220B68CDE901021B4A0092D3F800A046
:107690005A4630230AA8D047D3E7D8F8041004206C
:1076A0000A68CDE9016014480090D2F800A009A84A
:1076B0004A46D047FFF774B9D8F8041004200A6886
:1076C000CDE901600C480090D2F800A009A84A4614
:1076D000D047FFF7ADB9D8F8041004220B68CDE904
:1076E0000102054A0092D3F800B04A462B460AA888
:1076F000D847FFF7E1B900BF801A0600D8F8041098
:1077000004220B68CDE901020C4A0092D3F800B0C4
:107710004A462B4609A8D847FFF70FBAD8F80410F5
:1077200004220B68CDE90102044A0092D3F800B0AC
:107730004A462B4609A8D847FFF743BA801A0600E5
:1077400073B50446FEF7CCFF94F82330052B32D0F6
:10775000002594F83F33EB40DA07E9B216D401353F
:10776000082DF6D194F82330052B24D094F820303E
:1077700013B194F82230F3B9104B11491B68986982
:1077800003681B6802B0BDE870401847D4F808339E
:107790009B030CD42C200191FEF714FA064610B17D
:1077A000019903F019FC31462046FEF7C7FB94F817
:1077B0002330052BD3D102B070BD00BFEC250020D3
:1077C0008C3209082DE9F04F90F9213089B0044638
:1077D000002B00F00481012300F50C7580F8413383
:1077E000024600F50F712B462E46D06E002859D068
:1077F000002384F8413394F94030642B5BD094F932
:10780000BC30642B00F08D8094F93831642B00F08B
:107810008A80D4F830722FBB01A9204629F0F8FEE7
:1078200000B30C230593012306978DF81830714B94
:1078300007936946BDF80430049704A8ADF81030EA
:107840008DF800702AF064F89DF9001051B10229FA
:1078500008DC38B1C9B27C2303FB01416C312846F6
:107860002BF058FC94F841B3BBF1000F5DD0E36EF0
:107870006367D4F8E830C4F8F030D4F86431C4F861
:107880006C3194F8233003F1C30204EB820200212F
:10789000042B7CD852F8040B1061013342F8041C0D
:1078A000DBB2F5E753F8040B0028A1D18B4202F1BB
:1078B0007C029AD19FE7002066238DF810307C234C
:1078C00003FB004004A940302BF068FB04A92046CC
:1078D00029F09EFE00289CD004238DF81830002348
:1078E000CDE90133039331230593694604A82AF0B7
:1078F0000FF8059B28B108AA02EB8302009942F811
:10790000E01C0133332B0593EFD94CF0CFFF9DEDF5
:10791000031ADDED020A9DED010A66214CF084FF99
:1079200077E70120C8E70220C6E70127A94655F8F6
:10793000043B23B1AB600137042FF7D197E7AA4688
:10794000B8465FFA88F3022BF5D8DAF8002055F82C
:10795000043C9A4205D104A95046CDF810B02BF052
:10796000D9FB5AF8043B08F101020BB99046E8E74D
:1079700004A906EB88000193CDF810B02BF0CAFBE8
:10798000019BAB6001A948462BF0C4FBD3E794F8F8
:10799000413313B92046FEF7DDF994F822300BB3DA
:1079A000154B1B68986A036864215B6898472046FA
:1079B000FEF7A0FD94F83E3003B9E36694F8BA30C0
:1079C0000BB9C4F8E83094F836310BB9C4F8643117
:1079D000F9F7AEFDF9F736FE0123A4F8403309B0FC
:1079E000BDE8F08F2046FFF7ABFE94F82230002B65
:1079F000E0D0D5E7BCCB0908EC250020704700009B
:107A00000120704701207047436898687047000064
:107A100010B5054B03600446806A10B103685B68CB
:107A20009847204610BD00BF5037090840680368DA
:107A30005B6A184733B46C46406884E80C000368FE
:107A40009D6A94E80C00AC4602B030BC6047000070
:107A500010B50446FFF7DCFF2046FEF7BBF82046D2
:107A600010BD000040680AF0A5BC0000406801237A
:107A70000AF0A0BC40680AF079BC000040680A2205
:107A80000AF01EBC40680AF033BC000040680AF0EF
:107A9000B5BC000090F82E2022B190F82D100022E5
:107AA00001F06EB97047000073B504460525002645
:107AB000A06A8DF8076003680DF10702DB680121F9
:107AC000984778B19DF807300C2B09D0102B05D0C2
:107AD000092B07D184F8303002B070BD1523F9E7C7
:107AE0001423F7E7013DE3D12846F5E710B4806A97
:107AF00003681C690822A44601235DF8044B312168
:107B00006047000010B4806A03681C690122A44623
:107B100000235DF8044B322160470000F0B50446B5
:107B2000806A036885B05B6998470546002800F0C5
:107B30008480A06A03685B69984703689B689847DC
:107B4000A06A03689B69984760B93D4B3D491B6833
:107B5000986903681B6898472B682846DB68984734
:107B6000002667E02046FFF7CDFF0028F4D020462E
:107B7000FFF79AFF0028EFD0A06A03680121DB6AB3
:107B800098472046FFF7B2FF30B92D4B2E491B68AE
:107B9000986903681B68DEE7A06A0368DB69984799
:107BA00030B9274B29491B68986903681B68D2E7DD
:107BB000A06A94F83010012784F82E7003685B6A7D
:107BC0009847A06A03689B6A984704F12D02014612
:107BD000204601F023F906460028BDD0A06A94F89B
:107BE0002D10036801919B6A98470199024620462F
:107BF00001F018F994F82C302BB194F82D103A4676
:107C0000204601F023F994F82F2094F82D102046F7
:107C100001F03EF92B682846DB689847A06A029479
:107C200003681D6A0A4B039304AB13E90C0042F28C
:107C30001071A847304605B0F0BD0646FAE700BF10
:107C4000EC250020BC360908E2360908013709088E
:107C5000497D010870B5002586B0CDE900550023A7
:107C60000446806A8DF808500593039304930368D3
:107C70006A469E6810210923B047A0B19DF80030E4
:107C800013F0010615D194F831300133DBB2052B26
:107C900084F8313007D12046FFF734FF2046FFF744
:107CA00025FF84F83160A06A03681B6B984706B013
:107CB00070BD9DF8083084F831501B07F3D4BDF92E
:107CC00001309FED1F6A06EE903ABDF9033007EED2
:107CD000103ABDF90530F8EEE66A07EE903ACDEDC0
:107CE000036AF0EEE66AB8EEC77AF8EEE77AF4EEE9
:107CF000C66AF1EE10FA8DED047ACDED057A0DD558
:107D0000B0EEC77AB4EEC67AF1EE10FA06D5F0EE10
:107D1000E77AF4EEC67AF1EE10FAC4D49FED090AC0
:107D200003A810F06BF9B2EE040A03A810F066F98C
:107D300094F82D200A2303A9204601F00FF9B2E799
:107D4000000000349A99193EFFF784BF10B5044B28
:107D5000044640F8043BFBF7C3FF204610BD00BFBC
:107D60006837090810B50446FFF7F0FF2046FDF715
:107D700031FF204610BD0000F7B503680F461646D8
:107D80001BB90024204603B0F0BD00240460082085
:107D90000193FDF717FF054620B1124B0360019BCD
:107DA0004360019401A8FBF79BFF002DE9D034202C
:107DB000FDF708FF04460028E3D000F0E1FE0A4B7F
:107DC000A562236084F82C7084F82F602046FFF7AA
:107DD000A5FE05460028D5D1236820465B68984754
:107DE0002C46CFE768370908503709082DE9F74FC7
:107DF000046806460D4690469946002C6CD00B68E8
:107E0000002B49D0236820465B6A984703689B682B
:107E10009847012328680DEB030200210AF0CAFAF3
:107E200098B39DF80130EA2B2FD1DFF8F0B04FF076
:107E3000060A28680023802206210AF097FA20B358
:107E4000DBF80070B86A03680A215B689847002372
:107E500028681A4606210AF089FAB0B1B86A0368A0
:107E60000A215B689847012328680DEB030206216D
:107E70000AF0A0FA48B19DF8014014F040042FD058
:107E80000AF1FF3A1AF0FF0AD3D1306803685B6A3F
:107E900098470368DB68984700241DE002222346C8
:107EA0000F2128680AF062FAB86A036801215B684A
:107EB0009847306803685B6A98470368DB689847AF
:107EC000336834604A46414601A80193FFF754FFE6
:107ED000044601A8FBF704FF204603B0BDE8F08F7D
:107EE000224623460F2128680AF040FAB86A036840
:107EF00001215B6898470223214630680DEB03029D
:107F00000AF058FA04460028C8D0B8690249036844
:107F10001B689847B9E700BF28370908EC250020FF
:107F200090F82C10002200F02BBF000070B5044622
:107F30008CB00426013E76B2731C4AD0A06A152389
:107F40006A465D210AF036FA0028F3D0A06A1523AC
:107F500006AA5D210AF02EFA05460028EAD015226D
:107F600006A9684672F07EF90028E3D19DF800303A
:107F700084F82E309DF8073084F830309DF81430A6
:107F800084F83A309DF813309DF8102084F83B3087
:107F90009DF80F3043EA0223A3879DF8013084F84F
:107FA0002F309DF8083084F83130039B9DF80C2069
:107FB000C3F30F2363869DF80B3043EA0223A386A5
:107FC000049BC3F30F23E386019BC3F30F23238793
:107FD00007E0054B05491B68986903681B689847CB
:107FE000002528460CB070BDEC2500209C37090800
:107FF0002DE9FF4104460023806A8DF807300368AD
:10800000DFF868815B6A984703689B689847A06AB5
:1080100003680A219B6C9847A06A0A2204210AF08F
:108020004FF90425013D6DB26B1C32D000234B216A
:10803000A06A82220AF09AF9D8F800600746B06A6E
:10804000036802215B689847002FEBD001231A4692
:108050004B21A06A0AF08AF90746B06A0368022138
:108060005B689847002FDDD0A06A01230DF107025D
:1080700040210AF09FF90028D4D09DF80720322A29
:1080800010D0002DCED1B069364903681D68322367
:10809000A847A06A03685B6A98470368DB6898474B
:1080A00000255BE02046FFF741FF0028F1D0A06AE1
:1080B0000123172251210AF059F90028E9D0522250
:1080C000A06A012311460AF051F90028E1D0A06A04
:1080D000012338224C210AF049F90028D9D0A06A9E
:1080E00003685B6A98470368DB689847A06A0521C4
:1080F0000AF0FEF8A36A04F12C029968204600F009
:108100008DFE054650B3A36A94F82C109A68204659
:1081100000F088FE94F8442094F82C10204600F0DB
:10812000B7FE94F845302BB194F82C10012220466C
:1081300000F08CFEA06A036802219B6C9847A06A3D
:10814000029403689E6A084B039304AB13E90C0086
:1081500044F21B11B0474EF057FF2064284604B08C
:10816000BDE8F081C4370908D9820108EC25002058
:1081700070B5858F90F93B60AD03B5FBF2F2A2F5C7
:10818000804404FB04F2D51190F83A200498D201FF
:10819000624306FB05225212A03002F580124243D0
:1081A00012134A43DB0003EB623000B270BD0000E3
:1081B00010B5448E53005C43B0F93830C91A838F30
:1081C000D31AB0F93620B0F93400534304F5004413
:1081D0009B10C3EBC13300EB2440044993FBF0F048
:1081E0004FF400420DF0D6FE00B210BD0080FFFF3C
:1081F00010B52DED028B8AB004460823806A05AACB
:1082000042210AF0D7F818B1BDF81A20D30719D4C3
:10821000A06A0AF0F3F84EF0F7FE236CC31AFA2BAB
:108220000CD92064002382224B21A06A0AF09EF818
:108230000123A06A1A464B210AF098F80AB0BDEC57
:10824000028B10BDBDF9141094F9303000939208E0
:1082500094F92E300392C9102046FFF789FFBDF92B
:10826000161094F93130039A009308EE900A94F9AD
:108270002F30C9102046FFF77BFFBDF91810039A75
:10828000491008EE100A2046FFF792FF07EE900A09
:10829000F8EEE88AF8EEE77AB8EEC88AB3EE000A9C
:1082A00007A8CDED097ACDED078A8DED088A0FF08C
:1082B000B9FEB2EE040A07A80FF0A0FE4EF0A4FE2D
:1082C00094F82C2020640A23204607A900F046FEDB
:1082D000A06A0AF093F8B1E7FFF78ABFF7B5036821
:1082E0000D4616461BB90024204603B0F0BD0027FA
:1082F00007604820CDE90073FDF764FC044650B1E7
:1083000000F03EFC0E4B2360019BA362019784F8B2
:10831000446084F8455001A8FBF7ECFC6846FBF785
:10832000E9FC002CDFD02046FFF762FE054600285E
:10833000DAD1236820465B6898472C46D4E700BF13
:10834000FC37090810B5044B044640F8283BFBF7FE
:10835000D1FC204610BD00BFFC37090810B504460B
:10836000FFF7F0FF2046FDF735FC204610BD00006A
:1083700090F82C10002200F003BD0000F8B5044670
:108380000D4617461E4600F0FBFB094B23602B6889
:10839000A362002200232A6084F82D7084F82E60E6
:1083A00023656365A365E365236663662046F8BDC0
:1083B00014380908F8B51C4609331646DB086A4626
:1083C000A2EBC30300AF9D46806AA31C6A4609F076
:1083D000F1FF054628B122460DF10201304671F049
:1083E00051FF2846BD46F8BD2DE9F34106460F462C
:1083F00014464EF009FE114BD3F800800546D8F81C
:108400002800036801215B68984701230DF10702EA
:1084100007213046FFF7CEFF60B19DF80730DA073D
:1084200002D4B7EB531F05D04EF0EEFD431BA34221
:10843000E5D3002002B0BDE8F08100BFEC250020AC
:108440002DE9F041DFF8608292B0044602AF0026C9
:1084500046F02002A06A0023D2B2502109F086FF24
:10846000002800F00C810325013D6DB26A1C00F06C
:108470000681D8F80030986A03684FF496719B68BB
:10848000984701230DF1060255212046FFF792FF80
:10849000002800F0F4809DF8063013F0E00F40F063
:1084A000EE80DB07E0D502230DF1060252212046C3
:1084B000FFF780FF002800F0E280BDF806300136AB
:1084C0005BBA202E27F8023BC2D1BDF824309DF8BC
:1084D00026109FED6D7ADFED6D6A9FED6D6A43F3B7
:1084E0000B0207EE902A1B0903F47063BDF82620E7
:1084F000F8EEE77A0B4343F30B03C4ED0C7A07EE77
:10850000903A02F470639DF82820F8EEE77A13435E
:1085100043F30B03C4ED0D7A07EE903A9DF9223038
:10852000F8EEE77AC4ED0E7A07EE903A9DF929301D
:10853000F8EEE77A67EE877A07EE103AB8EEC77A78
:108540009DF92A30C4ED0F7A27EE267ADFED517AB5
:1085500084ED107A07EE103AB8EEC77A9DF92B3009
:10856000E7EE267AC4ED117A07EE903AF8EEE77A54
:108570009DF9233067EEA67ADFED476AC4ED127AE3
:1085800007EE903A9DF92C3007EE103AB8EEC77A14
:108590009DF92E3027EE267AF8EEE77A84ED147AEC
:1085A00067EE867A07EE103A9DF93030C4ED137A03
:1085B00007EE903AF8EEE77A9DF92D3067EEA67A4D
:1085C000B8EEC77AC4ED167A27EE267A07EE903A0F
:1085D00084ED157AF8EEE77A9FED307A9DF92F3029
:1085E00067EE877AC4ED177A07EE903A9DF931303D
:1085F000F8EEE77A06EE903A67EE877AF8EEE66AEA
:10860000C4ED187ADFED267ABDF93830E6EE877AC8
:1086100007EE103A9DF93230C4ED197AB8EEC77AF8
:10862000F3EE077AE7EE067A07EE103ADFED1D6A01
:10863000C4ED1A7AB8EEC77A27EE267A84ED1B7A53
:108640009DF9333007EE103AB8EEC77A9DF9343011
:1086500027EE267A84ED1C7A07EE103A9DF9353024
:1086600007EE903AB8EEC77AF8EEE77A27EE267A68
:1086700067EEA67A84ED1D7AC4ED1E7A00E0002034
:1086800012B0BDE8F08100BFCDCC4C3E0000803B75
:108690000000003B0AD7233C0000003D000080386A
:1086A00017B7D1B80AD7A33AEC25002073B5012338
:1086B0000E460DF1070206210446FFF77BFE18B9AE
:1086C0000025284602B070BD9DF80730013B012B04
:1086D0000CD80023A06A1A46062109F047FE00289C
:1086E000EED0062200212046FFF77EFEA06A00237E
:1086F0003246062109F03AFE05460028E0D026223F
:1087000031462046FFF770FEDBE7000013B501237A
:108710000DF1070207210446FFF74CFE10B90020B7
:1087200002B010BD9DF807301B070CD50023A06ACE
:108730001A46062109F01AFE0028F0D00622002170
:108740002046FFF751FEA06A00230722062109F008
:108750000DFE0028E3D0132207212046FFF744FE38
:108760000028DCD0A06A00230522062109F0FEFDC6
:108770000028D4D0172205212046FFF735FE002817
:10878000CDD001212046FFF791FFC9E7F7B5044698
:10879000806A5B4F03685B6A984703689B689847E9
:1087A000A06A03680A219B6C9847A06A0A220421E8
:1087B00009F086FD0525013D6DB26B1C00F0968029
:1087C000A06A0023B6227E2109F0D0FD0028F2D055
:1087D0003B68986A036818215B686E4698470123D6
:1087E000324600212046FFF7E5FD0028E3D09DF842
:1087F0000030332BDFD12046FFF722FE002875D052
:10880000A06A00238022502109F0B0FD00286DD01D
:108810002046FFF77BFF002868D0A06A002386224D
:108820002E2109F0A3FD002860D0A06A0023242295
:10883000042109F09BFD002858D0A06A00230222E1
:10884000062109F093FD002850D014220221204671
:10885000FFF7CAFDA06A00230722052109F086FD63
:10886000002843D001212046FFF720FF00283DD0FB
:10887000A06A036803219B6C9847A06A03685B6A3F
:1088800098470368DB689847A06A172109F030FD14
:10889000A36A04F12C029968204600F0BFFA05464D
:1088A00008B3A36A94F82C109A68204600F0BAFA2C
:1088B00094F82E2094F82C10204600F0E9FA94F851
:1088C0002D302BB194F82C100122204600F0BEFA76
:1088D000A06A03689F6A0B4B0094019396E80C0012
:1088E00042F21071B847284603B0F0BDA06A036891
:1088F0005B6A98470368DB6898470025F3E700BF89
:10890000EC250020FD8A010810B586B00C236A46CC
:1089100031210446FFF74EFD002800F0DF809DF86E
:1089200001309DF80020DFED717ADFED715A1B04F4
:1089300003EB02239DF8022003EB02631B1206EEF9
:10894000903A9DF804309DF803201B0403EB0223AA
:108950009DF8052003EB02631B1207EE103A9DF809
:1089600007309DF806201B0403EB02239DF8082026
:1089700003EB02631B1206EE103A9DF80A309DF8D5
:1089800009201B0403EB0223F8EEE66AB8EEC77A6F
:108990009DF80B2066EEA76A27EE277AB8EEC66A26
:1089A000DFED547A03EB02631B1226EE276A07EE13
:1089B000903AF8EEE77A67EEA57AF5EEC07AF1EE36
:1089C00010FA40F38D80DFED4C5A77EEE57AD4ED66
:1089D000134A94ED0F5A94ED1C4AD4ED1D3A94F8C5
:1089E0002C20F7EE005A74EEA54AF0EE632AA4EEAE
:1089F000A75A0A2303A9D4ED107AD4ED0C4A77EED6
:108A0000A57A2046E7EEA64AD4ED1A7A75EE677A83
:108A100094ED145AF0EE646AD4ED174AE5EE276A35
:108A2000B0EE655AA7EEA45AC6EE854A94ED115AE7
:108A3000D4ED0D6A35EE255AE5EE076A94ED157A08
:108A4000E7EE876A94ED187AB0EE655AA7EE875A7A
:108A500086EE857A94ED125AD4ED0E6A35EE255ADB
:108A6000E5EE066A94ED166A94ED195AE7EE866A09
:108A7000B0EE656AA7EE856AF0EE657A86EE863A14
:108A800094ED1B6AF0EE646AE6EE447AE6EE476A1D
:108A900086EEA75AF0EE476AE4EE646AC6EEA75A7D
:108AA000D4ED1E6AD4EE262AE6EE636AB2EE046ABC
:108AB00027EE667A65EE066AA2EEA47ACDED036A29
:108AC00065EE866ACDED046AC7EE276A76EE837A94
:108AD00067EE867ACDED057A00F040FA06B010BD5B
:108AE00044BFDFED055A77EEA57A70E747ABE73B69
:108AF0005B9E803AF61BEB3B85EBCB41FFF704BF57
:108B000030B51346026885B00D461AB900242046D8
:108B100005B030BD002101607C2001930392FDF778
:108B200051F8044620B1019B2A4603A9FFF726FC11
:108B300003A8FBF7DFF8002CE8D02046FFF726FE5D
:108B400005460028E3D1236820465B6898472C46F9
:108B5000DDE7000010B5044B044640F8283BFBF766
:108B6000C9F8204610BD00BF1438090810B50446E6
:108B7000FFF7F0FF2046FDF72DF8204610BD00005E
:108B8000064B10B503600446FDF7A4FD606004F1D8
:108B900008004DF075F9204610BD00BF2C380908BB
:108BA00073B50646144675687C2303FB0253C4EB79
:108BB000441405EB8404084693F8A41001900FF0C8
:108BC000B3FA94F93C3001983BB9736893F82510D7
:108BD00002B0BDE870400FF0A7BA94F84010F7E774
:108BE00037B5446801917C2505FB024595F83F3077
:108BF00004EB8304D4F84C325BB14EF005FAC5F8AF
:108C00009C000199D4F84C0203B0BDE8304003F059
:108C100079BE03B030BD00002DE9F04FC2EB421425
:108C200047684FEA840881460E4607F13C0B08F17D
:108C300008018BB01546594430460FF0ABF9D9F80E
:108C4000040029460BEB8404FDF7EAFC38B17C23D1
:108C500003FB057393ED1A0A30460FF0CFF97C231E
:108C600003FB057393ED146ADFED3A7AD3ED156AD1
:108C7000B0EEC67AB4EEE77AF1EE10FA0FD5B0EEA8
:108C8000E67AB4EEE77AF1EE10FA08D594ED077AB9
:108C9000B0EEC77AB4EEE77AF1EE10FA1BD47C237B
:108CA00003FB0573D86D196E5A6E9B6D029003918C
:108CB0000490079101A831468DED016ACDED056A5A
:108CC0000692089209930DF017FB86ED000AC6ED97
:108CD000010A86ED021A7C2303FB05770023C7F8FF
:108CE0008C30C7F88830C7F88430D9F8040090F980
:108CF0005C3208F13C0A08F14808DA44D84463B110
:108D00005DB9414600F5167004F0B4FA41463046AC
:108D10000BB0BDE8F04F0FF03DB990F93430012BA6
:108D20000BD190ED0E0A50460FF014F984ED120AA3
:108D3000C4ED130A84ED141AE8E7022BE6D1FBF721
:108D400009FD002201A9FBF705FA0028DED09DED00
:108D5000010AE8E70000003410B543687C2404FBF6
:108D6000023407C904F1900383E807004EF04CF980
:108D7000C4F89C004EF03CF9C4F8A00010BD0000FF
:108D8000F0B5074685B00D46164600F10801A92248
:108D900003A809F05BFD7C687C2303FB0543D3F843
:108DA000B42022B903A809F073FD05B0F0BDBEB12F
:108DB00096ED007AD3ED2A7A67EE877AC3ED2A7AA8
:108DC00096ED017AD3ED2B7A67EE877AC3ED2B7A95
:108DD00096ED027AD3ED2C7A67EE877AC3ED2C7A82
:108DE0007C2607EE902A06FB0541A831B8EE670AFB
:108DF000084601910FF016F901992A463846FFF707
:108E0000ABFF06FB05410023C1F8B030C1F8AC3020
:108E1000C1F8A8300023C1F8B430C3E74068FCF7BC
:108E2000E9BF0000F7B50646406801927C2707FBC2
:108E300001000D466C3001A914462AF04BF9716807
:108E400007FB05152C6703B0F0BD000007B54068AF
:108E50007C2303FB010393F93C30022B0BD000F180
:108E60003C03C1EB411003EB80000DF107018DF8CD
:108E700007202AF089F803B05DF804FB43687C22E0
:108E800002FB013191F93C00003818BF0120704706
:108E900043687C2000FB013181F8A420704700006A
:108EA000F8B5054608460F460FF01AF910B1002430
:108EB0002046F8BD38460FF0F9F804460028F6D1F0
:108EC0006B6893F934637EB138460FF041FC95ED41
:108ED000087ADFED1F7AF0EEC76AF4EEE76AF1EE8A
:108EE00010FA03D585ED080A0124E1E777EE407A10
:108EF00030EE076AF0EEE77AC7EE866AF6B207EE62
:108F0000906A9FED146AF8EE677A26EE866AF4EEB0
:108F1000C67AF1EE10FA48BFB2EE046ADFED0E7ABF
:108F200045BF6B6A66EE866AB0EE676A87EEA66A30
:108F300046BF01336B620124F7EE007A77EEC67A02
:108F400020EE060AA7EE270A85ED080AB0E700BF63
:108F50000000003400004843CDCCCC3D2DE9F74360
:108F600004460E4615461F46FFF71AFE2A463146AE
:108F70002046FFF735FE314620462A46FFF74CFED5
:108F800031462046FFF78CFF28B39B2204F10801ED
:108F900001A809F05BFC64684FF07C0909FB0548F7
:108FA00008F1A808314640460EF0F4FF09FB0542DF
:108FB000D2F8B4100131C2F8B4104FB1B94207D39E
:108FC0004908C2F8B410B0EE000A40460FF02AF883
:108FD00001A809F05DFC03B0BDE8F08310B50446BC
:108FE000FCF792FFC0B23C34C0EB401004EB8000B1
:108FF00010BD0000F8B50A4E044600F5167704F5DA
:10900000137555F8040B08B103F0B0FFBD42F8D159
:109010003368986A036801215B689847EFE700BFEF
:10902000EC25002008B5FFF7E5FF0000F0B5144E71
:1090300000EB810773780446D7F84C026FF34103C5
:1090400087B00D467370C8B102F07EFB68B17378CB
:1090500043F0100373702C440023A372D7F84C0222
:1090600007B0BDE8F04002F0F3BAD7F84C126846FA
:1090700002F09AFB009B012BEDD1E8E707B0F0BDB1
:109080000C5B002070B506460D46002445FA04F33B
:10909000DB07E1B202D53046FFF7C8FF0134032CED
:1090A000F4D170BDFF21FFF7EDBF000030B500F532
:1090B000137587B000F5167455F8041B21B9A54245
:1090C000FAD1002007B030BD684602F06DFB009B6E
:1090D000013B022BF3D80120F4E700002DE9F04713
:1090E0002DED028B88B004460D469046B0EE408AC6
:1090F000FDF7DEF930B90026304608B0BDEC028B32
:10910000BDE8F08729462046FDF74CF806460028C2
:10911000F1D004EB8507D7F83C22D7F830329A42D9
:1091200006D037F0C7F95C4A032130F0EFFBE2E7E5
:10913000D7F84C3283B94FF49870FCF743FD814661
:1091400008B103F017F8C7F84C92B9F1000F03D13A
:1091500037F0B0F9514AE7E7B4F84A32D90711D5E8
:1091600005F078FE90F8082390F8C43232B9B022A6
:1091700002FB030090F8A130012B03D837F09AF9D5
:10918000474AD1E72046FFF791FF20B9454A537877
:1091900043F00203537094F9353053B32946204607
:1091A000FFF71CFF90F90030002B53D029462046D2
:1091B000FFF714FF90F80490B9F12B0F19D8294646
:1091C0002046D7F84CA2FFF709FF94F9353090F903
:1091D0000020022BD4BF00210121012BD4BF00238A
:1091E0000123003A009118BF01224946504602F07F
:1091F00043FA631900229A7275B3D4EDC10AB4F828
:109200004822D7F84C0270EEA00A2B46B0EE480A6E
:10921000414602F051FA94F83E33002B31D1224AF4
:10922000069412680127E773906A0268156D1F4A59
:109230000792029309224FF40063CDE9003208AA95
:1092400012E906001A4BA847C8B937F033F9194A92
:1092500002216AE79946B2E729462046FFF7BEFE9B
:1092600090F90030002BC8D0D4EDC10AB4F84822E0
:10927000D4F84C022B46B0EE480A4146C9E784F8C0
:109280003E7300230DF1170104F124008DF817300F
:1092900029F084FE30E700BF3C3809086E38090821
:1092A000913809080C5B0020EC250020259001086E
:1092B000AF380908BA3809082DE9F0412DED028BC5
:1092C000002443739DF82030837305460F46904673
:1092D000B0EE408A264647FA04F3DB07E1B210D528
:1092E000B0EE480A42462846FFF7F8FE064640B967
:1092F00039462846FFF7C6FEBDEC028B3046BDE876
:10930000F0810134032CE6D1F6E70000F8B5002423
:109310002DED028B05460F46B0EE408A42738373F3
:109320002646E1B2B0EE480A3A462846FFF7D6FE96
:109330000134002818BF0646032CF2D1BDEC028B85
:109340003046F8BDF0B500EB81030D46D3F84C1262
:109350009BB0044611B900201BB0F0BD0BA802F071
:1093600007FA6319987A0028F6D10B9A002A48D098
:10937000042AF0D101229A720DAA07CA02AB83E82F
:10938000070010AA07CA05AF87E8070013AA07CA93
:109390009DED180A08AE86E807001A4629462046C1
:1093A0008DED010AFCF792FE3A4629462046FCF76D
:1093B00039FE324629462046FCF746FE9DED010A5D
:1093C00029462046FCF752FE9DF8643083B12946B9
:1093D0002046FFF703FE90F900304BB194F9353089
:1093E000012B05DD9DF85D2029462046FCF786FE11
:1093F0002046FFF75BFE20B9034A537843F004038D
:1094000053700120A8E700BF0C5B00202DE9F0415C
:109410000546884600F513770024012657F8043BDB
:10942000E1B26BB148FA04F3DB0709D52846FFF730
:1094300089FF002857F8040C08BF002602F008F93D
:109440000134032CEAD13046BDE8F0812E4B2DE9E2
:10945000F04F1F68FB6A93F89C8087B00446B8F110
:10946000000F38D1DFF8A8A000F5137600F1030B48
:10947000054656F8040BA5EB04095FFA89F9E8B133
:1094800002F04EF928B19AF8013043F008038AF847
:10949000013056F8040C02F057F9F8B9637B6BB150
:1094A000AB7A5BB956F8041C684602F07DF9009B64
:1094B000042B03D149462046FFF744FF01355D45A3
:1094C000D7D1124B204683F81280FFF7EFFD0546F7
:1094D00030B10123237407B0BDE8F08F8046EDE77B
:1094E000237C002BF7D0A37B002BF4D0B86A036851
:1094F0004FF47A715B689847B86A03689B6B29469A
:1095000007B0BDE8F04F1847EC250020ED5A0020C9
:109510000C5B0020F0B5002587B000F513762C46D3
:10952000012756F8041B41B1684602F03DF9009B43
:109530001BB107FA05F31C43E4B20135032DF0D14A
:10954000204607B0F0BD00002DE9F04F2DED028B55
:1095500003270E7C9FED348A91B005468846B946B4
:10956000AC5D0134E4B2B4FBF9F303EB4303E41A5A
:10957000E4B205EB8403D3F84C1209B9AC554CE0C6
:1095800003A802F011F9DDF80CB00BF1FF33022B48
:10959000F4D8304631F048F98246304632F048F887
:1095A00000F11B039A4508D2304630F0B9FB002089
:1095B00011B0BDEC028BBDE8F08FAC55284698F891
:1095C00010A0FFF7A7FFDDED057A8DF83100FCEE66
:1095D000E77A9DF810208DF8332017EE903A8DF839
:1095E000343006AB03CB1B88ADF83D305C221B2327
:1095F000CDE90032CDF83500CDF8391009AABF21E8
:1096000050468DED098A8DED0A8A8DED0B8A8DF815
:1096100030408DF832B031F071F9013F17F0FF079B
:109620009ED10120C4E700BF000000002DE9F04FEB
:109630000F7CA1B006468846032500EB070999F880
:1096400005400134E4B20323B4FBF3F303EB43031B
:10965000E41AE4B206EB8403D3F84C1211B989F88A
:1096600005400AE011A802F083F8DDF844A0BAF141
:10967000030F08DCBAF1000FF1DA013D15F0FF0528
:10968000DDD1012012E0AAF10402032AF5D8384600
:1096900031F0CAF88346384631F0CAFF00F136028D
:1096A000934506D2384630F03BFB002021B0BDE8A0
:1096B000F08F89F80540304698F810B0FFF72AFF80
:1096C000DDF848E0CDF80CE0DDF84CE0CDF810E036
:1096D000DDF850E0CDF814E0DDF854E0CDF818E006
:1096E000DDF858E0CDF81CE0DDF85CE0CDF820E0D6
:1096F000DDF860E0CDF824E03219DDF864E01C9B71
:10970000CDF828E0DDF868E092F80AC09DF8741002
:109710009DF87520CDF82CE00E93DDF86CE01E9BD3
:109720008DF835008DF83C108DF83D20CDF830E0F7
:109730008DF834408DF836A08DF837C02422CDF84E
:109740003E303623CDE90032C0212C2303AA5846EF
:1097500031F0D4F891E700007FB58A8B0B464AF2CE
:10976000B9518A4205465FD04AF2BA518A4274D052
:109770004AF2B8518A420BD1474A1268D26A92F82B
:109780009C203AB136F096FE444A052130F0BEF8EE
:10979000042479E0D3ED007AF5EEC07AF1EE10FA08
:1097A000F6D49FED3F7AF4EEC77AF1EE10FAEFDCD3
:1097B00093ED017ADFED3B6A1C6993ED030AB0EE8D
:1097C000C77AB4EEE67A93ED027AFCEEE77AB0EE71
:1097D000C77AF1EE10FAB4EEE67A17EE903A54BF7B
:1097E00001260026F1EE10FA54BF01220022003CAF
:1097F00018BF012413F0FF0110D18DED030A02926E
:10980000FCF7CCFB9DED030A029A2346314628461D
:10981000FFF77CFD0028BBD0002435E01346009400
:109820003246FFF749FDF5E7D3ED007AF5EEC07A51
:10983000F1EE10FAACD49FED1A7AF4EEC77AF1EE9D
:1098400010FAA5DCFCEEE77A17EE903A13F0FF0170
:1098500008BFFF21FFF7DAFDDCE7D3ED007AF5EE74
:10986000C07AF1EE10FA93D49FED0D7AF4EEC77A38
:10987000F1EE10FA8CDCFCEEE77A17EE904A14F069
:10988000FF0404D1FFF70EFC204604B070BD214652
:10989000FFF7F8FBC0E700BFEC250020EC38090813
:1098A00000007F4300000034F0B58BB00E46144634
:1098B0000746FFF793FB543007C884E8070031469A
:1098C0003846FFF78BFB90ED057ADFED267AB0EE98
:1098D000C77AB4EEE77AF1EE10FA054611D590EDAD
:1098E000067AB0EEC77AB4EEE77AF1EE10FA08D550
:1098F00090ED077AB0EEC77AB4EEE77AF1EE10FA9F
:1099000024D431463846FFF769FB016A426A836A0C
:10991000E869D5F814E0D5F818C0099001A8CDF889
:1099200004E0029103920491CDF814C006930792CB
:1099300008930CF08DFE98B1214601A80CF0DCFCD8
:1099400084ED000AC4ED010A84ED021A314638465E
:10995000FFF744FB00F1080120460EF035FB012023
:109960000BB0F0BD000000342DE9F0472DED048B65
:10997000ACB0B0EE608A0546B0EE409A0F46F0EE0D
:10998000418A9046FCF70AFBDFED8B7AB0EEC87A8D
:10999000B4EEE77AF1EE10FA4BD5B0EEE87AB4EE19
:1099A000E77AF1EE10FA44D523AC2046FBF73CFEF3
:1099B000F7F7BEFD2146F7F79DFB064658BB05F0BD
:1099C00049FA90F8083390F8C42233B1B02303FB6E
:1099D000020393F8A130012B07D84FF0B00909FB1F
:1099E000020090F8A130022B0BD836F063FD734AC9
:1099F00003212FF08BFF30462CB0BDEC048BBDE86B
:109A0000F08705F027FA90F8C43209FB0300AC3068
:109A10000FC884E80F00DDED257A9FED691AB8EED6
:109A2000E78ADDED267AF8EEE78A28EE018A68EE0D
:109A3000818A04AA03A902A8F0EE680AB0EE480AD7
:109A400003F0D4FC064618B936F034FD5D4ACFE782
:109A50009FED5D7ADDED027A9FED5C8ADFED5C8A39
:109A60008DED068A67EE877A2422002111A8CDEDBC
:109A7000057A8DED078A70F04FFC9DED031ADDED40
:109A8000040ADFF858A121EE281A68EEE00AB0EEC9
:109A9000480A11A80CF0FCFD05A911A80CF02CFC3B
:109AA000242200211AA8CDED060A8DED071A8DEDAE
:109AB000050A70F031FCF7F73BFD90ED810A8DED62
:109AC000010AF7F735FD29EE281AD0ED820A9DED3F
:109AD000010A1AA80CF0DCFD1AA923A80CF0FAFC64
:109AE00005A923A80CF008FC4FF000098DED050A2C
:109AF000CDED060A8DED071A95F822305FFA89F44C
:109B0000A3427FF678AF1FB127FA04F3DB071AD51B
:109B10002B1993F92C32B3B1B8F1000F0DD02146B7
:109B20002846FCF7C5FC88B936F0C4FC294A234610
:109B300003212FF0EBFE00265DE721462846FCF7C7
:109B400031FB0028EBD109F10109D5E708AA21462C
:109B500028468DED088A8DED098A8DED0A8AFFF77A
:109B6000A3FE20B936F0A6FC1B4A2346E0E708A96D
:109B700005A80EF0D9F90BAA214628468DED0B0A4F
:109B8000CDED0C0A8DED0D1AFCF7A0FA9AE807004E
:109B90000EAB83E807001A4621462846FCF742FA36
:109BA00023AA214628468DED238A8DED248A8DED4A
:109BB000258AFCF749FAC6E7000000341039090885
:109BC00095BFD6332B39090800007A440000000005
:109BD00035FA8E3C4039090854390908A0E50808CF
:109BE0000120704701207047436898687047000063
:109BF000406803689B6C184710B5054B036004462A
:109C0000806A10B103685B689847204610BD00BFAA
:109C10003C3A0908406803685B6A184733B46C46ED
:109C2000406884E80C0003689D6A94E80C00AC4628
:109C300002B030BC6047000010B50446FFF7DCFFFF
:109C40002046FBF7C7FF204610BD0000406808F023
:109C50004FBB0000406808F0ADBB00004068012326
:109C600008F0A8BB4068002308F080BB90F84420AF
:109C7000D20705D590F8421000F12C02FFF780B80A
:109C800070470000F8B504461E460F461546FEF71D
:109C900077FF084B23600023E3622363636394F838
:109CA0004430A76265F3410384F8436084F844308C
:109CB0002046F8BD3C3A090810B50D4B83630446B5
:109CC000806A036898221B690021984770B1A06AD6
:109CD000036820221B690121984738B1A06A0368F4
:109CE000BDE810401B69012202211847002010BD69
:109CF000C5DC6A3F37B50446806A03686A469D68DA
:109D000003210623A847D0B1BDF80020BDF80410F8
:109D100052BA95B249BAB5F5704F0BB211D013F5DE
:109D2000805F0ED0BDF802305BBA9DB2B5F5704FC2
:109D300007D052425B42A287E187A4F8403003B0CB
:109D400030BD0020FBE70000806A036801221B6928
:109D50000221184730B585B00446FFF7CBFF054612
:109D60002046FFF7F1FF6DB3B4F93C3094ED0E0AD5
:109D700006EE903AB4F93E3007EE103AB4F94030AE
:109D800007EE903AF8EEE66AB8EEC77AF8EEE77AB0
:109D900001A8CDED016A8DED027ACDED037A0EF0CA
:109DA0002DF994F842102046FFF768F818B1022107
:109DB00001A80EF0B9F994F842200E2301A920461B
:109DC000FFF7CCF805B030BDFFF7C4BF13B5806A0C
:109DD000036801AA9C680A210323A04738B10549FA
:109DE000032201A870F03EFAB0FA80F0400902B0F8
:109DF00010BD00BF743909082DE9F84300252DED89
:109E0000028BDFF888819FED5D8A04462E462F463F
:109E1000A06A036811221B690021013798470028B6
:109E20007BD0D8F80090D9F82800036832215B680D
:109E30009847A06A036860221B690121984700289F
:109E40006BD0A06A036801221B6902219847002891
:109E500063D0D9F82800036832215B689847204610
:109E6000FFF748FF002858D00135022FEDB256DD2C
:109E7000B4F93C309FED425A9FED426A07EE903AAA
:109E8000F8EEE77AC5EE276AF0EEE66AF4EEC66A07
:109E9000F1EE10FA41DDF4EEC86AF1EE10FA3CD5AD
:109EA000B4F93E30DFED385A07EE903AF8EEE77A33
:109EB00085EEA77AB0EEC77AB4EEC67AF1EE10FA64
:109EC0002BDDB4EEC87AF1EE10FA26D5B4F94030A5
:109ED00005EE903AF8EEE55AC5EE257AF0EEE77A0F
:109EE000F4EEC67AF1EE10FA17DDF4EEC87AF1EE70
:109EF00010FA12D594ED0B6A76EE266A0136C4ED9F
:109F00000B6AD4ED0C6A36EE877A84ED0C7A94ED08
:109F10000D7A77EE277AC4ED0D7A192F02D0052E2F
:109F20007FF476AFA06A036810221B69002198476E
:109F3000052E18D1D4ED0B6AF1EE047A86EEA77ADD
:109F40000120D4ED0C6A84ED0B7A86EEA77AD4ED6D
:109F50000D6A84ED0C7A86EEA77A84ED0D7ABDEC5D
:109F6000028BBDE8F8834FF07E53052DE362236337
:109F7000636394BF00200120F1E700BFCDCCAC3F6C
:109F800000002E443333333F00002244EC250020F0
:109F9000F0B50446806A036885B05B69984705465A
:109FA00048B9504B50491B68986903681B6898472B
:109FB000284605B0F0BD03689B689847A06A03680F
:109FC0000A21DB6A9847A06A03689B69984760B9D1
:109FD000444B46491B68986903681B6898472B687F
:109FE0002846DB6898470025E2E72046FFF7EEFEAB
:109FF0000028F4D02046FFF7FFFE30B9394B3C492A
:10A000001B68986903681B68E8E72046FFF754FE61
:10A010000028E4D0A06A0368DB69984730B9314B67
:10A0200034491B68986903681B68D7E794F8443083
:10A03000A06A43F0010384F8443003680321DB6A1B
:10A0400098472B682846DB689847236820469B681A
:10A050009847A06A036807215B6A9847A06A03686B
:10A060009B6A984704F1420201462046FEF7D6FE5D
:10A07000054600289CD0A06A94F84210036801911C
:10A080009B6A9847019902462046FEF7CBFE94F85A
:10A09000432094F842102046FEF7FAFE94F844302C
:10A0A0009B0705D594F8421001222046FEF7CEFE0C
:10A0B000A06A029403681E6A0F4B039304AB13E972
:10A0C0000C0043F21541B047064BA06A1B689E691D
:10A0D00033681F6803689B6A984708490246304600
:10A0E000B84765E7EC250020783909089E3909084A
:10A0F000C4390908E9390908C99D0108173A09084E
:10A1000010B5084B036004460023086860600B60CC
:10A11000037A03F00703022B02D1C02108F008FAEA
:10A12000204610BD543A090810B5044B044640F8C7
:10A13000043BF9F7DFFD204610BD00BF543A090883
:10A1400010B50446FFF7F0FF2046FBF743FD20461D
:10A1500010BD0000F7B503680E4617461BB9002472
:10A16000204603B0F0BD0022026008200193FBF7F7
:10A1700029FD054610B101A9FFF7C2FF01A8F9F7B3
:10A18000B9FD002DEBD04820FBF71CFD044600284C
:10A19000E5D029463B463246FFF774FD2046FFF7DF
:10A1A000F7FE05460028DBD1236820465B68984708
:10A1B0002C46D5E790F82D100022FEF7E1BD0000F7
:10A1C000F0B50446806A036889B05B6A9847036803
:10A1D0009B689847A06A03680A219B6C9847A06A0D
:10A1E00001230DF11702002108F0E4F8002838D00F
:10A1F0009DF81730082B34D14E4F0525002301223E
:10A20000A06A322108F0B2F83B689B6A1A6852686B
:10A2100040B90A2118469047013D15F0FF05EDD1E0
:10A2200045481CE018461421904706AEFF238DF8E0
:10A230001830A06A01233246322108F0BBF800280A
:10A24000EAD09DF8183013F00103E5D1A06A03931A
:10A250000822322108F08AF8039B58B937484CF09D
:10A2600007F8A06A03685B6A98470368DB68984749
:10A2700000255CE0A06A03931A46342108F076F8C2
:10A280000028EBD0039BA06A2422412108F06EF83D
:10A290000028E3D0039BA06A0822312108F066F869
:10A2A0000028DBD0A06A036803219B6C9847A06A52
:10A2B00003685B6A98470368DB689847A06A1021C7
:10A2C00008F016F8A36A04F12D0299682046FEF7FB
:10A2D000A5FD054658B3A36A94F82D109A68204648
:10A2E000FEF7A0FDA36A16481A7A597A00919B6876
:10A2F0001449D2084BF0BCFF94F82C2094F82D1090
:10A300002046FEF7C5FD94F82E302BB194F82D10A1
:10A3100001222046FEF79AFDA06A03689F6A0A4B55
:10A320000694079396E80C0042F21071B84728464D
:10A3300009B0F0BDEC250020E43A0908843A090888
:10A34000BB3A0908B33A0908D5A3010810B586B08D
:10A3500004460123806A0DF10302102108F02AF857
:10A3600098B39DF80330DB072FD5A06A062301AA16
:10A37000112108F01FF840B3BDF904309FED146AB5
:10A3800094F82D2006EE903ABDF9063007EE103A0B
:10A39000BDF808305B421BB207EE903AF8EEE66A71
:10A3A000B8EEC77AF8EEE77A66EE866A27EE067AA6
:10A3B00067EE867A0A2303A92046CDED036A8DED68
:10A3C000047ACDED057AFEF7C9FD06B010BD00BFD9
:10A3D00085EBC13FFFF7BABFF7B503680D461646D8
:10A3E0001BB90024204603B0F0BD002707603020D1
:10A3F000CDE90073FBF7E6FB044650B1FEF7C0FB66
